:100000000C94A70B0C94D80B0C94D80B0C94D80B15
:100010000C94D80B0C94B8750C94C34C0C94688752
:100020000C94D80B0C94D80B0C94D80B0C94D80BC4
:100030000C94D80B0C94D80B0C94D80B0C94D80BB4
:100040000C94D80B0C94F85D0C948C770C94A99EAE
:100050000C94D80B0C94D80B0C94D80B0C94D09E09
:100060000C94D80B0C9446A30C947CA30C94D80B42
:100070000C94D80B0C94D80B0C94D80B0C94D80B74
:100080000C94B7650C94D80B0C94D80B0C94D80B2B
:100090000C94F1A30C9427A40C94D80B0C94089EF8
:1000A0000C94D80B0C94D80B0C94D80B0C94D80B44
:1000B0000C94D80B0C9488800C94D80B0C94D80B0F
:1000C0000C94D80B0C94D80B0C94D80B0C949CA4C7
:1000D0000C94D2A40C94D80B0C9447A50C947DA539
:1000E0000C94D80BE21ABA1A921A041B631B231B36
:1000F000581B411BFE1BD61BAE1B201CA51C3F1C06
:100100009A1C831C631E8E1EB91EE31E8A1FB71F16
:10011000E41F1020BD20BD20BD20BD20BD20BD207E
:10012000BD20BD20BD20BD20BD20BD20BD20BD20E7
:10013000BD20BD20BD20BD20BD20BD20BD20BD20D7
:10014000BD20BD20BD20BD20BD20BD20BD200D1F78
:10015000371F611F3C206820942073267A26812651
:1001600088268F2696269D26A426AB26B226B9265B
:10017000C026C726CE26D526DC26E326EA26F1268B
:10018000F826FF2606270D2714271B2722272927B5
:10019000302737273E2745274C2753275A276827DC
:1001A0006F2776277D2784278B27BC27C327CA275D
:1001B000D127D827DF27E627ED27F427FB270228BA
:1001C0000928102817281E2825282C2833284F28CE
:1001D00056285D2864287E28832888288F2894281C
:1001E00099289E28A328A828AF28B628BD28C42867
:1001F000CB28D228D928E028E728EE28F528FC28A3
:100200000329612792279927A027A727AE27B5277B
:100210003A28412848286B28722879280A29112968
:10022000B273C773DD73F173057419742D7441745F
:100230005574727486749A74B674C974027B0E7B9A
:100240001A7B267B327B3E7B4A7B9F7B567B627B85
:100250006E7B7A7B867B927BB87BC27BCC7BD67BAA
:10026000E07BEA7BF87B387C067C107C1A7C247C63
:100270002E7C967F9F7FA77FBB7FC17FDF7FEA7F3A
:10028000E290E290EA90E290F190F99001910A9167
:100290002CA031A036A040A04AA0C3A054A05CA0CE
:1002A00064A06EA078A082A091A09BA0C3A0A5A0EE
:1002B000AFA0B9A0E5A0E8A0D7A0DBA0E1A01FA156
:1002C000ECA0F0A0F6A0FAA0FEA004A108A10CA149
:1002D0001FA112A116A11AA146756E6374696F6EF3
:1002E000202300202D3E200020736563005475728A
:1002F000726574206D6F76656D656E742064656CD3
:1003000061793A2020004E6F6E6500596573005484
:10031000757272657420737469636B2066756E63A1
:1003200074696F6E733A200046554E4354494F4EE0
:100330002054524947474552530076206375746FE5
:10034000666629002028004C564320456E61626C89
:1003500065643A202020202020007600566F6C74BF
:100360006167653A2020202020202020202000598D
:100370006573004E6F004261747465727920446544
:100380007465637465643A2000424154544552597F
:100390000053657269616C20332054782042617586
:1003A000643A2020004175782053657269616C20A1
:1003B000426175643A202020004D6F746F722053A3
:1003C000657269616C20426175643A200055534240
:1003D0002053657269616C20426175643A20202067
:1003E0000042415544205241544553004952202671
:1003F0002054616E6B20426174746C696E67204496
:10040000697361626C656400207365632072656363
:100410006F766572792900207365632072656C6F51
:1004200061642C2000204D4720686974732C2000E3
:100430002063616E6E6F6E20686974732C200028D3
:100440000057656967687420436C6173733A2020B4
:100450002020200044616D6167652050726F6669DD
:100460006C653A20202000596573202800416363A1
:10047000657074204D472044616D6167653A2000C6
:1004800059657320280053656E64204D47204952FA
:1004900020436F64653A2020004E2F410052657062
:1004A00061697265642062793A2020202020200052
:1004B0004E2F41004869742050726F746F636F6CE7
:1004C00020323A20202000290020285465616D2028
:1004D00000466972652050726F746F636F6C3A20CA
:1004E00020202000466972652050726F746F636F20
:1004F0006C3A202020200049732052657061697297
:100500002054616E6B3F20202000424154544C45E2
:1005100020494E464F002900202D2041646A757302
:1005200074656420746F2000202853656E736974AD
:10053000697669747920002900202D2041646A754C
:100540007374656420746F2000202853656E73698E
:10055000746976697479200053656E736F72206ECA
:100560006F74206465746563746564210048696C08
:100570006C205068797369637320456E61626C65A5
:10058000643A202020202020202020004261727226
:10059000656C2053746162696C697A6174696F6E0D
:1005A00020456E61626C65643A200053656E736F1E
:1005B000722064657465637465643A20202020208D
:1005C00020202020202020202059657300494E45FE
:1005D000525449414C204D4541535552454D454E8D
:1005E0005420554E495400536F756E6420636172F8
:1005F000643A2000534F554E44204341524400205A
:10060000736563005265636F696C2064656C617922
:100610003A202020202020202020202020202020C0
:1006200020202020002500596573202D20004261E4
:100630007272656C20456C65766174696F6E2053CB
:1006400070656564204C696D697465643A200025A5
:1006500000596573202D2000547572726574205204
:100660006F746174696F6E205370656564204C69A6
:100670006D697465643A20200054555252455420E7
:1006800053455454494E4753004E2F4120666F72D4
:100690002076656869636C652074797065005475AF
:1006A000726E206D6F64653A20202020202020206B
:1006B000202020202020004E2F4120666F722076BF
:1006C000656869636C652074797065002500202D6C
:1006D00020004E65757472616C207475726E2061B5
:1006E0006C6C6F7765643A2020200020736563008E
:1006F0005472616E736D697373696F6E2064656C9B
:1007000061793A2020202020002073656300456E27
:1007100067696E652070617573652074696D653AEF
:100720002020202020200020736563005368696624
:10073000742074696D653A2020202020202020201C
:1007400020202020002500596573202D20005265AF
:100750007665727365205370656564204C696D69B8
:100760007465643A2020002500596573202D20000F
:10077000466F7277617264205370656564204C69BE
:100780006D697465643A202000206D73290025206E
:100790007468726F74746C6520666F722000202814
:1007A000004D6F746F72204E7564676520456E61F1
:1007B000626C65643A202020200029004E6F6E652F
:1007C000004E6F6E65002C205072657365743A2080
:1007D000002900202841646A757374656420746F71
:1007E000200020284C6576656C3A200044656365DE
:1007F0006C2052616D7020456E61626C65643A20B8
:10080000202020200029004E6F6E65004E6F6E651F
:10081000002C205072657365743A2000290020284E
:1008200041646A757374656420746F200020284CDD
:100830006576656C3A2000416363656C2052616D9A
:100840007020456E61626C65643A20202020200093
:100850004163746976652044726976696E672050D9
:10086000726F66696C653A200056656869636C65ED
:1008700020547970653A202020202020202020203C
:10088000200044524956452053455454494E47533D
:10089000004D656368616E6963616C207265636FAA
:1008A000696C00416972736F6674004D65636861BD
:1008B0006E6963616C2042617272656C3A2000203F
:1008C000284D31290020284D3229002028422900B6
:1008D00042617272656C20456C65766174696F6EF9
:1008E0003A20200020284D30290020284D312900B1
:1008F000202841290054757272657420526F74610A
:1009000074696F6E3A202020004472697665204D2C
:100910006F746F72733A202020202020004D4F54B6
:100920004F52205459504553004368616E6E656CB8
:1009300073207574696C697A65643A200043686154
:100940006E6E656C732064657465637465643A20CB
:10095000004E4F54204445544543544544004947B4
:100960004E4F52454400416E616C6F6700446967A9
:100970006974616C00417578204368616E2E202097
:10098000204D696E20202020204D617820202020DD
:10099000205479706500417A696D75746820202053
:1009A0002000456C65766174696F6E202000547577
:1009B000726E20202020202020005468726F7474F2
:1009C0006C6520202000537469636B202020202058
:1009D00020204D696E2020202043656E74657220B2
:1009E00020204D6178202020204465616462616E82
:1009F00064202052657665727365640052414449F3
:100A00004F20494E464F202D20004649524D574118
:100A100052452056455253494F4E3A20005761697E
:100A200074696E6720666F7220726164696F2E2E22
:100A30002E200025004E6F005965730046414C532F
:100A4000450054525545002000202D20002D004126
:100A50006E616C6F6720557365722046756E6374A6
:100A6000696F6E2032202D2000416E616C6F67200F
:100A7000557365722046756E6374696F6E20312000
:100A80002D2000557365722046756E6374696F6E14
:100A9000203200557365722046756E6374696F6EFF
:100AA0002031005365742048696C6C2053656E7367
:100AB000697469766974793A2000536574204261DB
:100AC0007272656C2053656E7369746976697479A6
:100AD0003A200053657420446563656C2052616D53
:100AE00070204C6576656C3A200053657420416334
:100AF00063656C2052616D70204C6576656C3A20A0
:100B0000005661726961626C650020286F6620354D
:100B100029003320286F66203329003220286F6691
:100B2000203329003120286F662033290032202805
:100B30006F66203229003120286F6620322900504C
:100B40006F732000417578204368616E6E656C207C
:100B5000005661726961626C65004F6E004F666697
:100B6000004200410045787465726E616C20496EE8
:100B700070757420005475727265742053746963C3
:100B80006B202D2000536574205475726E204D6FBC
:100B900064653A203100536574205475726E204D9F
:100BA0006F64653A203200536574205475726E206C
:100BB0004D6F64653A2033005573657220536F752D
:100BC0006E64200034202D2053746F700034202D6B
:100BD00020537461727420526570656174696E6728
:100BE00000340033202D2053746F700033202D20EB
:100BF000537461727420526570656174696E670028
:100C0000330032202D2053746F700032202D20537A
:100C10007461727420526570656174696E67003228
:100C20000031202D2053746F700031202D2053741B
:100C300061727420526570656174696E670031007D
:100C400053657420766F6C756D653A2000536D6F37
:100C50006B65722064697361626C656400536D6FCB
:100C60006B657220656E61626C65640052657665C5
:100C7000727365643A2020004D61782050756C7362
:100C8000653A20004D696E2050756C73653A2000FE
:100C9000456E642056616C75657300456E64205224
:100CA00065636F696C20536572766F205365747548
:100CB0007000456E6420456C65766174696F6E20C6
:100CC000536572766F205365747570005365727644
:100CD0006F20756E2D72657665727365640053655D
:100CE00072766F2072657665727365640052657600
:100CF00065727365643A2020004D61782050756CF0
:100D000073653A20004D696E2050756C73653A200A
:100D10000053746172742056616C75657300494E9E
:100D200056414C494420534552564F2E204E4F2099
:100D300053455455502E00536574757020526563A9
:100D40006F696C20536572766F00536574757020FF
:100D500054757272657420456C65766174696F6E46
:100D60002050616E20536572766F00526164696F26
:100D7000205265616479202D2000524144494F2062
:100D80004641494C534146450053746F70205265AB
:100D9000766F6C76696E6720417578204C6967685C
:100DA00074005374617274205265766F6C76696E4C
:100DB0006720417578204C696768740053746F70C0
:100DC00020417578204F757470757420426C696E7F
:100DD0006B696E6700537461727420417578204F9F
:100DE000757470757420426C696E6B696E67004132
:100DF0007578204F757470757420466C61736865E2
:100E00006400417578204F75747075742050726558
:100E10007365742044696D00417578204F75747056
:100E20007574204F66660053746F70205265766F3C
:100E30006C76696E6720417578204C69676874002C
:100E400053746F7020417578204F757470757420DD
:100E5000426C696E6B696E6700417578204F7574DE
:100E6000707574204F6E0052756E6E696E67204CFF
:100E70006967687473204F66660052756E6E696E9E
:100E800067204C6967687473204F6E004C6967680F
:100E9000742032204F6666004C69676874203220E7
:100EA0004F6E004C696768742031204F6666004CB5
:100EB000696768742031204F6E004C564320457896
:100EC0006974202D20566F6C7461676520526573BC
:100ED000746F726564007629004C56432074687202
:100EE0006573686F6C642072656163686564212056
:100EF0002800494F20506F72742042204F75747043
:100F00007574202D204F666600494F20506F727413
:100F10002042204F7574707574202D204F6E00494B
:100F20004F20506F72742041204F7574707574207B
:100F30002D204F666600494F20506F72742041206B
:100F40004F7574707574202D204F6E0048696C6C5D
:100F500020506879736963733A205475726E6564C2
:100F6000204F46460048696C6C205068797369636D
:100F7000733A205475726E6564204F4E0042617260
:100F800072656C2053746162696C697A6174696F0F
:100F90006E3A205475726E6564204F464600426179
:100FA0007272656C2053746162696C697A617469EC
:100FB0006F6E3A205475726E6564204F4E00456E18
:100FC00061626C65204E65757472616C2054757237
:100FD0006E730044697361626C65204E657574724E
:100FE000616C205475726E7300456E67696E652082
:100FF0004175746F2053687574646F776E00447226
:101000006976696E672050726F66696C65207365DA
:101010007420746F202300436F6D6D7320636861CB
:101020006E67656420746F2055534200436F6D6D89
:1010300073206368616E67656420746F2053657206
:1010400069616C2031004869676820496E74656E7B
:101050007369747920466C61736820556E697420D9
:101060002D204D616E75616C2054726967676572E1
:1010700000536572766F205265636F696C202D2076
:101080004D616E75616C2054726967676572004DC1
:10109000656368616E6963616C205265636F696C3A
:1010A000202D2044697361626C656400416972732C
:1010B0006F6674202D2044697361626C6564004D15
:1010C000656368616E6963616C205265636F696C0A
:1010D000202D20456E61626C656400416972736FFA
:1010E0006674202D20456E61626C6564004D6563F9
:1010F00068616E6963616C205265636F696C202D55
:10110000204D616E75616C2054726967676572006D
:10111000416972736F6674202D204D616E75616C2C
:101120002054726967676572004D472053746F7071
:10113000004D472053746172740046697265204304
:10114000616E6E6F6E0046697265205265706169EE
:1011500072205369676E616C0053746F70706564C0
:10116000004E65757472616C205475726E004D6F1F
:1011700076696E672052657665727365004D6F768D
:10118000696E6720466F7277617264004272616BAC
:10119000696E670054414E4B20524553544F52459F
:1011A000440025004865616C7468204C6576656C68
:1011B0003A200056454849434C4520524550414944
:1011C0005220434F4D504C4554450054414E4B2006
:1011D00044455354524F5945440025004865616CBD
:1011E0007468204C6576656C3A20002900564548A5
:1011F00049434C4520524550414952205354415295
:10120000544544202800524550414952204F5045F2
:10121000524154494F4E2043414E43454C4C454466
:101220000029004D414348494E452047554E20482E
:10123000495421202800524550414952204F5045E1
:10124000524154494F4E2043414E43454C4C454436
:1012500000290043414E4E4F4E204849542120283A
:101260000054757272657420656C65766174696F7F
:101270006E206973206E6F74206F662074797065BC
:1012800020536572766F2E204E6F207365747570D3
:1012900020617661696C61626C652E0021200046D8
:1012A0004143544F52592052455345542120000781
:1012B0000809090B0C0C0B0C0C69427573005342A6
:1012C00075730050504D004E6F6E65204465746517
:1012D0006374656400426F74746F6D20526967684F
:1012E0007400426F74746F6D2043656E7465720094
:1012F000426F74746F6D204C656674004D69646450
:101300006C65205269676874004D6964646C65207F
:1013100043656E746572004D6964646C65204C654C
:10132000667400546F7020526967687400546F705F
:101330002043656E74657200546F70204C6566744E
:1013400000556E6B6E6F776E00556E6B6E6F776EBD
:101350000044657461636865642F4E4100526563A3
:101360006F696C20536572766F0050616E20536513
:1013700072766F00536572766F2F455343004F6E40
:10138000626F617264204D6F746F7220447269766F
:101390006572004F70656E2050616E7A65722053E1
:1013A000636F75742053657269616C204553430007
:1013B0005361626572746F6F7468205365726961FE
:1013C0006C00506F6C6F6C752053657269616C00B6
:1013D000536572766F203100536572766F2032004C
:1013E000536572766F203300536572766F20340038
:1013F000536572766F203500536572766F20360024
:10140000536572766F203700536572766F2038000F
:10141000446973656E67616765205472616E736DB0
:10142000697373696F6E00456E67616765205472FA
:10143000616E736D697373696F6E005475726E209F
:10144000456E67696E65204F6666005475726E2042
:10145000456E67696E65204F6E0054616E6B202883
:10146000444B4C4D207479706529004361720048EB
:10147000616C66747261636B0054616E6B00554EF3
:101480004B4E4F574E003A2000426974200047618E
:10149000703A20003400330032004E6F6E65005306
:1014A0006F6E790052435441204D616368696E65E7
:1014B0002047756E00436C61726B204D61636869F3
:1014C0006E652047756E005243544120526570612D
:1014D0006972004942552052657061697200436C1F
:1014E00061726B20526570616972004F70656E5059
:1014F000616E7A657200567354616E6B00464F568A
:101500000054616967656E0048656E67204C6F6EB8
:10151000670054616D69796120312F333500546162
:101520006D69796120322D53686F740054616D6963
:10153000796100556E6B6E6F776E00102788139877
:101540003A1027401F7017D007A00FA00FDC05D05E
:1015500007C4096C023A026C023A026C023A026C4D
:1015600002B036384A5C121C255C125C121C255CE9
:1015700012BC7FC7F2C07887A5B7C5A00F8813B883
:101580000B401FB80BB80B7017401F554E4B4E4FFA
:10159000574E0042656965722055534D2D52432DBB
:1015A000320054616967656E20536F756E64204325
:1015B000617264004F70656E2050616E7A657220B2
:1015C000536F756E6420436172640042656E65649A
:1015D000696E6920544253204D696E6900556E6BE7
:1015E0006E6F776E004F70656E2050616E7A657217
:1015F0000054616D697961205370656300556E6BAD
:101600006E6F776E004865617679004D6564697527
:101610006D004C6967687400437573746F6D0000EA
:10162000000A0B02090C0D0E08070304010000005C
:1016300000000000000000000000000000000000AA
:101640000000000000000000000000121110000067
:10165000000000000000000000000000000000008A
:101660000000000000010210202008081020401097
:101670002040800201020108040201010204081056
:101680002040808040201008040201800402018074
:10169000402010080402010804020101020408109D
:1016A0002040800102040810204080050505050740
:1016B0000508080808020202020A0A0808040404CD
:1016C00004010101010101010103030303030303F9
:1016D00003040707070C0C0C0C0C0C0C0C02020288
:1016E0000206060606060606060B0B0B0B0B0B0B7B
:1016F0000B000020002300260029002C002F0032C0
:10170000000001000003010601090100002200257C
:101710000028002B002E00310034000201000005DB
:101720000108010B0100002100240027002A002DE0
:10173000003000330001010000040107010A01002C
:10174000B54BC58EB194AEA359A404A5AFA5112481
:101750001FBECFEFD1E2DEBFCDBF00E00CBF18E06F
:10176000A0E0B2E0E9EEFFE701E00BBF02C00790A6
:101770000D92A031B107D9F725E1A0E1B8E001C091
:101780001D92AD32B207E1F717E1CEE4D7E100E0F8
:1017900006C022970109FE010BBF0E94D8ADC034DC
:1017A000D10780E00807A9F70E941EAB0C943AB15C
:1017B0000C940000089508950895089508950895DB
:1017C0000895089508950895089508950895089531
:1017D000089508951092E2080895809193098093E6
:1017E0009409089502960C94E38102960C947981F1
:1017F00002960C94798102960C941D8102960C94A9
:101800004D8102960C94848102960C9491810296EB
:101810000C94C08202960C94EF8202960C94F38290
:1018200002960C94C48202960C94C88202960C9480
:10183000EB8202960C94CC8202960C94D58202968E
:101840000C94C98202960C94DD8202960C94E68276
:1018500002960C94DA8202960C94FA8202960C9408
:10186000F78202960C94038302960C9407830296E7
:101870000C940B8302960C940C8302960C941083A8
:1018800002960C94148302960C94158302960C9481
:10189000198302960C941D830C94268302960C9453
:1018A000C08302960C943E8302960C944183029668
:1018B0000C94678302960C948D8302960C944A8351
:1018C00002960C94708302960C94968302960C9464
:1018D0001E8302960C9422836091290970912A0933
:1018E00085E999E00E94D564882341F06091290937
:1018F00070912A0985E999E00E94896360E088E097
:101900000E9459A1809194098823D1F080912809DF
:10191000882319F060E47EE00DC0809127098823B8
:1019200019F067E27EE006C080918F09811108C03E
:1019300068E17EE080919109909192090E9474A6DD
:1019400010922809109227090895C6CFCF9360916D
:101950000A0289E30E9459A160910A02C1E06C2742
:101960008AE30E9459A180910A028C2780930A027F
:10197000CF9108954F925F926F927F92AF92BF92F4
:10198000CF92DF92EF92FF920F931F932C01612C65
:10199000712C1F921F921F928FEF8F93A12CB12C4D
:1019A0006501EE24EA9413E0F12E00E010E020E05F
:1019B00030E0A901C301B2010E94BDA888E00E94E5
:1019C00008A01F921F921F9284E68F9320E030E0C0
:1019D000A901C301B2010E94BDA88DB79EB70896A8
:1019E0000FB6F8949EBF0FBE8DBF80911012681382
:1019F000609310121F910F91FF90EF90DF90CF90A6
:101A0000BF90AF907F906F905F904F9008956091DE
:101A10001B0870E088E00E9408A089E180931A0802
:101A200090910C0280911B08992311F08D5F01C0E9
:101A3000835080931B0880911B08873970F099238D
:101A400021F08FEF80931B0808C08D3D30F086E9B0
:101A500080931B0888E780931A0880911B088F3FAA
:101A600019F410920C0205C08A3118F481E08093B9
:101A70000C0240911A0850E060E070E027E03DE081
:101A800085E999E00E946D6390932A098093290962
:101A900008952091F108222369F0A091FE08B091E9
:101AA000FF08ED91FC9111970190F081E02DBC01B0
:101AB000CD01199408952091F008222369F0A09196
:101AC000FC08B091FD08ED91FC9111970190F08117
:101AD000E02DBC01CD01199408952091EF08222337
:101AE00069F0A091FA08B091FB08ED91FC91119773
:101AF0000190F081E02DBC01CD0119940895209151
:101B0000EE08222369F0A091F808B091F908ED9150
:101B1000FC9111970190F081E02DBC01CD01199449
:101B200008952091ED08222369F0A091F608B09164
:101B3000F708ED91FC9111970190F081E02DBC0127
:101B4000CD01199408952091EC08222369F0A09109
:101B5000F408B091F508ED91FC9111970190F08196
:101B6000E02DBC01CD01199408952091EB082223AA
:101B700069F0A091F208B091F308ED91FC911197F2
:101B80000190F081E02DBC01CD01199408952091C0
:101B9000E608222369F0A091E908B091EA08ED91E6
:101BA000FC9111970190F081E02DBC01CD011994B9
:101BB00008952091E508222369F0A091E708B091EB
:101BC000E808ED91FC9111970190F081E02DBC01A6
:101BD000CD01199408952091F108222339F0BC0118
:101BE00080910C0990910D090C94E45B089520916B
:101BF000F008222339F0BC0180910A0990910B0969
:101C00000C94E45B08952091EF08222339F0BC0185
:101C100080910809909109090C94E45B0895209142
:101C2000EE08222339F0BC01809106099091070942
:101C30000C94E45B08952091ED08222339F0BC0157
:101C400080910409909105090C94E45B089520911A
:101C5000EC08222339F0BC0180910209909103091C
:101C60000C94E45B08952091EB08222339F0BC0129
:101C700080910009909101090C94E45B0895AF9262
:101C8000BF92CF92DF92EF92FF920F931F93CF9369
:101C9000DF93BC0180918F11811132C0E0910E0958
:101CA000F0910F090190F081E02DC081D18180E099
:101CB00090E01F921F921F922FEF2F93A12CB12C17
:101CC0006501EE24EA9413E0F12E00E010E020E03C
:101CD00030E0A9010E94BDA80F900F900F900F90C7
:101CE00080910E0990910F09FE01DF91CF911F9114
:101CF0000F91FF90EF90DF90CF90BF90AF9019942D
:101D0000DF91CF911F910F91FF90EF90DF90CF90D7
:101D1000BF90AF90089580919309882361F00E944D
:101D20004B53029741F06DE17AE0809191099091D7
:101D300092090C9474A608950E94EB67882379F0A9
:101D400080E00E94E86780919409882341F063ED68
:101D50007FE080919109909192090C9474A6089566
:101D60008091AE11833099F00E94EB6781110FC012
:101D700081E00E94E86780919409882341F06EEB2E
:101D80007FE080919109909192090C9474A6089536
:101D90000E94EB67882319F080E090E0CDCF80E0CF
:101DA00090E0DECF0E94E567833079F083E00E9407
:101DB000DE6780919409882341F067EA7BE0809197
:101DC0009109909192090C9474A608950E94E56778
:101DD000823079F082E00E94DE6780919409882346
:101DE00041F066E97BE080919109909192090C9411
:101DF00074A608950E94E567813079F081E00E9421
:101E0000DE6780919409882341F065E87BE080914A
:101E10009109909192090C9474A60895CF93DF9341
:101E2000EC0180911208909113088C179D07D9F04E
:101E3000D0931308C093120880919409882399F0D5
:101E400069E67AE080919109909192090E9438A602
:101E50004AE050E0BE018091910990919209DF9192
:101E6000CF910C947AA7DF91CF910895CF93DF9310
:101E7000EC0180911008909111088C179D07D9F002
:101E8000D0931108C093100880919409882399F089
:101E90006FE47AE080919109909192090E9438A6AE
:101EA0004AE050E0BE018091910990919209DF9142
:101EB000CF910C947AA7DF91CF910895FC0180898E
:101EC000918993878287828993899587848784897A
:101ED00095899787868708950E943A86809194090C
:101EE000882341F061E371E1809191099091920919
:101EF0000C9474A60895F0CF0E948886809194096E
:101F0000882341F069E271E18091910990919209F1
:101F10000C9474A60895F0CF0E94FA8680919409DB
:101F2000882379F0209181118091910990919209F3
:101F3000222319F060E171E102C06DEE70E10C94B2
:101F400074A60895E9CF81E00E94AF85809194093D
:101F5000882379F0209181118091910990919209C3
:101F6000222319F06BED70E102C06FEB70E10C946D
:101F700074A60895E8CF80E00E94AF85809194090F
:101F8000882379F020918111809191099091920993
:101F9000222319F06CEA70E102C06FE870E10C9442
:101FA00074A60895E8CF0E94B2858111E4CFCBCF0B
:101FB000FACFE0911009F091110982810E949C5F93
:101FC00080919409882341F061E770E18091910943
:101FD000909192090C9474A60895EBCF0E9401870A
:101FE00080919409882341F066E470E18091910921
:101FF000909192090C9474A60895F0CF833079F0F3
:1020000030F4813051F0823091F48BE30BC0843096
:1020100041F0853061F482E405C08CE303C080E4C4
:1020200001C081E40E948EA121E0892B09F420E007
:10203000822F089585E0E2CF0F931F9380916B0864
:1020400081110DC00E941A9F609327087093280881
:102050008093290890932A0881E080936B088091EF
:102060000E028A3AC9F4E6DF882361F00E94C39524
:1020700082E593E190939209809391098FEF809389
:102080000E020AC00E94CA9585EB92E190939209D4
:102090008093910910920E020E941A9F00912708C6
:1020A000109128082091290830912A08601B710B93
:1020B000820B930B633371058105910508F443C0CE
:1020C0000E941A9F6093270870932808809329081C
:1020D00090932A08AFDF882321F080910E02882395
:1020E00041F0A8DF81112FC080910E028F3F59F57A
:1020F00016C00E94C39582E593E190939209809364
:10210000910980919409882331F06CE270E182E5B5
:1021100093E10E9474A68FEF80930E0214C00E9478
:10212000CA9585EB92E190939209809391098091F1
:102130009409882331F067E170E185EB92E10E9418
:1021400074A610920E021F910F91089557DF91E02F
:102150008927089581E0FADF882331F082E0F6DFF5
:10216000882311F080E0089581E0F0DF882321F0DA
:1021700082E044DF811113C08CE30E948EA1892B81
:1021800021F082E0E3DF81110CC08CE30E948EA17C
:10219000892B21F082E032DF811105C0089581E0B2
:1021A000089582E0089583E0089583E0CFDF8823D7
:1021B00031F084E0CBDF882311F081E0089583E0E3
:1021C000C5DF882321F084E019DF811111C083E08D
:1021D00015DF882321F084E0B9DF81110BC083E093
:1021E0000DDF882321F084E009DF811105C0089507
:1021F00082E0089583E0089584E00895EF920F93BC
:10220000CF93C82F823069F4E090A21100919F1102
:102210002091A3114091A0116091A11180919E1174
:102220000CC0E0909C110091991120919D1140915A
:102230009A1160919B11809198110E944E65809136
:102240001702C817D1F0C093170280919409882310
:10225000A1F06EEF7FE080919109909192090E9428
:1022600038A64AE050E06C2F809191099091920934
:10227000CF910F91EF900C9460A7CF910F91EF90B9
:10228000089581E0BBCF82E0B9CF80911702813001
:1022900011F482E001C081E0B1CFF7CF6091E30893
:1022A0007091E40885E999E00E94D564882341F0A3
:1022B0006091E3087091E40885E999E00E948963E0
:1022C0001092E4081092E30808958091B311909160
:1022D000B411A091B511B091B611181619061A06CD
:1022E0001B0654F50E947569882329F16091E30863
:1022F0007091E40885E999E00E94D564882341F053
:102300006091E3087091E40885E999E00C94B86461
:102310004091B3115091B4116091B5117091B61103
:1023200020E832E285E999E00E946D639093E40829
:102330008093E3080895B2CF089510922E098091FA
:102340003309811112C0EFEFF0E180819181845651
:1023500091098436910530F0339681E1E737F8072B
:10236000A1F703C081E080932E0910923509809176
:102370003A09811112C0EFEFF0E180819181885C10
:1023800091098436910530F0339681E1E737F807FB
:10239000A1F7089581E080933509089580910701A0
:1023A000869581700895FADF882399F061E08FE3C4
:1023B0000E9459A181E08093320980919409882379
:1023C00041F066E37FE080919109909192090C942D
:1023D00074A60895E8CFE2DF882391F060E08FE3F0
:1023E0000E9459A11092320980919409882341F0EA
:1023F0006FE17FE080919109909192090C9474A60D
:102400000895E9CF80912608882311F0E4DF01C008
:10241000CADF8091260891E08927809326080895D5
:10242000F1CFCF93DF93BADF81112AC0C0912F097A
:10243000D091300980913409882371F08FE30E9494
:10244000E39F813092402CF01092300910922F09B6
:102450000AC081E090E003C08FE30E94E39F909365
:10246000300980932F0980912F09909130098C17A2
:102470009D0719F41092310903C081E0809331095E
:10248000DF91CF9108958091070181700895FBDF5E
:10249000882399F061E08EE30E9459A181E0809346
:1024A000390980919409882341F069E07FE08091A7
:1024B0009109909192090C9474A60895E8CFE3DFF6
:1024C000882391F060E08EE30E9459A110923909AF
:1024D00080919409882341F062EF7EE08091910918
:1024E000909192090C9474A60895E9CF80912508E3
:1024F000882311F0E4DF01C0CADF8091250891E054
:102500008927809325080895F1CFCF93DF93BBDF10
:1025100081112AC0C0913609D091370980913B09B9
:10252000882371F08EE30E94E39F813092402CF06B
:1025300010923709109236090AC081E090E003C07A
:102540008EE30E94E39F9093370980933609809130
:102550003609909137098C179D0719F410923809A4
:1025600003C081E080933809DF91CF910895809175
:102570002E09811156DF809135098111C6CF08954A
:102580002DEC3EE340ED57E060E070E085E999E036
:102590000E946563909399088093980808958F929C
:1025A0009F92AF92BF92CF92DF92EF92FF9285E41B
:1025B0000E94E39FBC01882777FD8095982F0E9499
:1025C00033AC20E030E040E85AE30E94E7AC20E082
:1025D00030E040EA50E40E94E7AC6B017C0180915E
:1025E0000D02882351F0C0922108D0922208E09277
:1025F0002308F092240810920D0226E636E646E6FD
:102600005FE36091210870912208809123089091E6
:1026100024080E94E7AC4B015C0120ED3CEC4CEC43
:102620005DE3C701B6010E94E7AC9B01AC01C501A7
:10263000B4010E9430AB609321087093220880930C
:102640002308909324082DE33CE248E450E40E94E0
:10265000E7AC2AE939E949E95EE30E9430ABFF9033
:10266000EF90DF90CF90BF90AF909F908F900895A4
:1026700096DF20E030E040E050E40E9494AB881FF9
:102680008827881F08958BDF20E030E04AE754E474
:102690000E94E7AC0E9405AC41E020910512309108
:1026A00006126217730708F040E0842F089561E076
:1026B00085E30E9459A18091230990912409DC01AE
:1026C000ED91FC9106A0F7A1E02D19958091940958
:1026D000882341F06FEA7EE0809191099091920900
:1026E0000C9474A60895E3CF60E085E30E9459A19D
:1026F0008091230990912409DC01ED91FC9106A0C1
:10270000F7A1E02D199580919409882341F063EA9F
:102710007EE080919109909192090C9474A608959D
:10272000E3CF80912008882311F0DEDF01C0BFDFF6
:102730008091200891E08927809320080895F1CFA7
:1027400061E085E00E9459A180919409882341F0BD
:1027500068E97EE080919109909192090C9474A6A9
:102760000895EECF60E085E00E9459A18091940920
:10277000882341F06CE87EE0809191099091920964
:102780000C9474A60895EECF80911F08882311F051
:10279000E9DF01C0D5DF80911F0891E08927809390
:1027A0001F080895F1CF81E080932D0961E084E056
:1027B0000C9459A110922D0980912C09811104C00B
:1027C00060E084E00C9459A160912B0970E084E0F2
:1027D0000C9408A081E080932C0980912D0981112F
:1027E00006C060912B0970E084E00E9408A08091EF
:1027F0009409882341F06AE77EE0809191099091E5
:1028000092090C9474A60895E5CF10922C0980913A
:102810002D09811104C060E084E00E9459A18091DB
:102820009409882341F067E67EE0809191099091B8
:1028300092090C9474A60895E8CF80911E0888230D
:1028400011F0E3DF01C0C6DF80911E0891E0892707
:1028500080931E080895F1CF61E088E00E9459A19D
:1028600080919409882361F080912809811108C022
:1028700069E57EE080919109909192090C9474A68B
:102880000895EACF60E088E00C9459A1809128096E
:10289000811110C021D881E080932809809194098A
:1028A000882341F065ED7DE0809191099091920936
:1028B0000E9474A680911C08882311F0E3DF01C0F8
:1028C000CBDF80911C0891E0892780931C08882326
:1028D00029F040910C1250910D1204C040910E123B
:1028E00050910F1260E070E026E434E185E999E050
:1028F0000E946D6390932A09809329090895C6CF99
:1029000080911D08882319F00E946C0C01C0A4DF7F
:1029100080911D0891E0892780931D080895F0CFCC
:102920006091101270E088E00E9408A080919409E4
:10293000882341F062E07EE08091910990919209B4
:102940000C9474A60895ECCF87DF40910A12509141
:102950000B1260E070E02CE63CE085E999E00E9413
:102960006D6390932A0980932909809194098823A3
:1029700041F06FEE7DE080919109909192090C9465
:1029800074A60895E1CF80912809882311F10E944F
:102990006C0C109228096091290970912A0985E927
:1029A00099E00E94D564882341F0609129097091D3
:1029B0002A0985E999E00E94896380919409882316
:1029C00049F06CEB7DE080919109909192090C9413
:1029D00074A65CCF0895D7CF80912709811129C0B3
:1029E00060E088E00E9459A11092280960912909AD
:1029F00070912A0985E999E00E94D564882341F005
:102A00006091290970912A0985E999E00E948963FA
:102A100081E08093270980919409882341F062EA3C
:102A20007DE080919109909192090E9474A60C9486
:102A3000070D0895D1CF80912709882321F11092A5
:102A4000270960E088E00E9459A1609129097091EE
:102A50002A0985E999E00E94D564882341F06091B4
:102A6000290970912A0985E999E00E94896380917A
:102A70009409882349F069E87DE08091910990915B
:102A800092090C9474A6A8CF0895D5CF729A089590
:102A900072980895CF9360910B0289E30E9459A127
:102AA00060910B02C1E06C278AE30E9459A16091FA
:102AB0000B0285E30E9459A160910B026C2785E00F
:102AC0000E9459A160910B026C2784E00E9459A1D9
:102AD00060910B0287E00E9459A10E946C0CC0918A
:102AE0000B02CC2311F0D4DF01C0D0DF81E08C27B2
:102AF00080930B02CF91089561E089E30C9459A172
:102B000060E089E30C9459A161E08AE30C9459A137
:102B100060E08AE30C9459A10F931F93CF93DF9346
:102B20008C01C1E0D0E00C171D079CF0E5DF64E6E6
:102B300070E080E090E00E94499FE2DFC017D1077B
:102B400034F46AE570E080E090E00E94499F2196AD
:102B5000EACFDF91CF911F910F91089581E090E02E
:102B6000DBCF0F931F93CF93DF938C01C1E0D0E0B5
:102B70000C171D079CF0C8DF64E670E080E090E071
:102B80000E94499FC5DFC017D10734F46AE570E0A1
:102B900080E090E00E94499F2196EACFDF91CF919B
:102BA0001F910F91089581E090E0DBCF60E089E311
:102BB0000E9459A160E08AE30E9459A160E085E388
:102BC0000E9459A160E085E00E9459A160E084E084
:102BD0000E9459A160E087E00E9459A10E946C0CFC
:102BE00057CF60918D0970918E0985E999E00E9417
:102BF000D564811116C0DADF80911212882319F092
:102C00002AE435E102C026EA3CE042E350E060E01D
:102C100070E085E999E00E94656390938E09809346
:102C20008D09089560E089E30E9459A160E08AE37C
:102C30000E9459A160E085E30E9459A160E085E00F
:102C40000E9459A160E084E00E9459A160E087E001
:102C50000E9459A11DCF60918D0970918E0985E95F
:102C600099E00E94D564882369F060918D09709184
:102C70008E0985E999E00E94896310928E0910926D
:102C80008D09D0CF08958091190881110DC010923F
:102C900018081092170881E090E09093160880932E
:102CA00015088093190836C080911708909118086C
:102CB000863191057CF18F38910534F480911508A7
:102CC00090911608019609C08D3521E0920754F4C1
:102CD000809115089091160802969093160880939B
:102CE000150818C0863222E0920734F48091150846
:102CF000909116080496F1CF883E93403CF4809161
:102D00001508909116088A5B9F4FE7CF109216081E
:102D100010921508BFDE4091170850911808493EDF
:102D200083E0580754F0109219087CDF2AEB36E153
:102D300048EE53E060E070E006C0662757FD6095FE
:102D4000762F23E436E185E999E00E946D63909344
:102D50009708809396088091170890911808209101
:102D6000150830911608820F931F909318088093CE
:102D70001708089580919A08811185CF609196086F
:102D80007091970885E999E00E94D564882341F005
:102D9000609196087091970885E999E00E9489638F
:102DA00041CF8F929F92AF92BF92CF92DF92EF92DC
:102DB000FF920F931F93CF93DF9381E08093F108ED
:102DC0008093F0088093EF088093EE088093E608E4
:102DD0008093E5089091AE119150943050F080931B
:102DE000AE1141E050E060E571E08AE192E10E94BD
:102DF0002F949091AE112DEF290F809177112230F1
:102E000008F0B1C18A3079F03CF4883009F465C02B
:102E1000893009F456C14AC18B3009F4B0C08C30F6
:102E200009F4F1C043C182E290E00E942CABEC01B6
:102E300033E5832E32E0932E9982888288E090E0F9
:102E40009B838A83AA24A394BB24BA94BD82AC82B8
:102E5000CC24CA94D12CDF82CE8219861886188E93
:102E60004FEE53E163E8CE0149960E9427626FE777
:102E7000E62E63E0F62EF982E8820CEF11E119A349
:102E800008A3D0931D09C0931C09CE010E942A5C9F
:102E900082E290E00E942CABEC019982888289E06A
:102EA00090E09B838A83BD82AC82DF82CE821986CA
:102EB0001886188E4FEE53E163E8CE0149960E94C2
:102EC0002762F982E88219A308A3D0931909C09355
:102ED0001809CE010E942A5CE7C280E290E00E94BD
:102EE0002CABEC0183E5A82E82E0B82EB982A88233
:102EF00088E090E09B838A83CC24C394DD24DA9419
:102F0000DD82CC82EE24EA94F12CFF82EE821986D7
:102F10001886188E4FEE53E16AE0CE0149960E9462
:102F20000F6107E913E019830883D0931D09C0934B
:102F30001C09CE010E94B55780E290E00E942CABA4
:102F4000EC01B982A88289E090E09B838A83DD82CC
:102F5000CC82FF82EE8219861886188E4FEE53E1DE
:102F60006AE0CE0149960E940F6119830883D093CD
:102F70001909C0931809CE010E94B55795C289E17D
:102F800090E00E942CABFC0188E090E09383828368
:102F9000EE24E394FF24FA94F582E4820FEF10E02C
:102FA0001783068311861086108EC3EAD3E0D1837F
:102FB000C083F0931D09E0931C09CF010E94E857DC
:102FC0001092E6088091AE11843009F06DC289E15B
:102FD00090E00E942CABFC0189E090E09383828317
:102FE000F582E4821783068311861086108ED183C2
:102FF000C083F0931909E0931809CF010E94E857A4
:103000001092E50851C289E190E00E942CABEC01DE
:10301000A3E5AA2EA2E0BA2EB982A88287E090E0AA
:103020009B838A83CC24C394DD24DA94DD82CC8212
:10303000EE24EA94F12CFF82EE8219861886188E0F
:10304000CE010E94FC5F0BEB13E019830883D09341
:103050001D09C0931C09CE010E9448581092F10826
:103060008091AE11843009F01FC289E190E00E9486
:103070002CABEC01B982A88286E090E09B838A8326
:10308000DD82CC82FF82EE8219861886188ECE01F0
:103090000E94FC5F19830883D0931909C093180913
:1030A000CE010E9448581092F008FEC189E080933A
:1030B000771149E050E069E171E08AE192E10E9414
:1030C0002F9480E290E00E942CABEC0173E5A72ED8
:1030D00072E0B72EB982A88288E090E09B838A8351
:1030E000CC24C394DD24DA94DD82CC82EE24EA94ED
:1030F000F12CFF82EE8219861886188E4FEE53E16E
:1031000060E8CE0149960E947D600BE813E01983C8
:103110000883D0931D09C0931C09CE010E947757E4
:1031200080E290E00E942CABEC01B982A88289E099
:1031300090E09B838A83DD82CC82FF82EE821986B7
:103140001886188E4FEE53E160E8CE0149960E9432
:103150007D6019830883D0931909C0931809CE01A3
:103160000E947757A1C18A3079F03CF4883009F485
:103170005BC0893009F437C12BC18B3009F49AC088
:103180008C3009F4D0C024C182E290E00E942CABC4
:10319000EC0133E5832E32E0932E9982888288E019
:1031A00090E09B838A83AA24A394BB24BA94BD8213
:1031B000AC82CC24CA94D12CDF82CE8219861886A8
:1031C000188E4FEE53E163E8CE0149960E942762C4
:1031D0006FE7E62E63E0F62EF982E8820CEF11E14C
:1031E00019A308A3D0931F09C0931E0982E290E09F
:1031F0000E942CABEC019982888289E090E09B834D
:103200008A83BD82AC82DF82CE8219861886188EB0
:103210004FEE53E163E8CE0149960E942762F9829E
:10322000E88219A308A326C180E290E00E942CAB9B
:10323000EC0183E5A82E82E0B82EB982A88288E04E
:1032400090E09B838A83CC24C394DD24DA94DD82CE
:10325000CC82EE24EA94F12CFF82EE821986188645
:10326000188E4FEE53E16AE0CE0149960E940F613D
:1032700007E913E019830883D0931F09C0931E093F
:1032800080E290E00E942CABEC01B982A88289E038
:1032900090E09B838A83DD82CC82FF82EE82198656
:1032A0001886188E4FEE53E16AE0CE0149960E94CF
:1032B0000F61DEC089E190E00E942CABFC0188E048
:1032C00090E093838283EE24E394FF24FA94F582C2
:1032D000E4820FEF10E01783068311861086108EAC
:1032E000C3EAD3E0D183C083F0931F09E0931E09A2
:1032F00089E190E00E942CABFC0189E090E093838F
:103300008283F582E4821783068311861086108EED
:10331000D183C083F0932109E09320091092E6083D
:103320001092E508ABC0923059F481E08093AE1161
:1033300041E050E060E571E08AE192E10E942F9463
:1033400089E190E00E942CABEC01A3E5AA2EA2E05B
:10335000BA2EB982A88287E090E09B838A83CC242E
:10336000C394DD24DA94DD82CC82EE24EA94F12C3D
:10337000FF82EE8219861886188ECE010E94FC5FAD
:103380000BEB13E019830883D0931F09C0931E0928
:1033900089E190E00E942CABEC01B982A88286E022
:1033A00090E09B838A83DD82CC82FF82EE82198645
:1033B0001886188ECE010E94FC5F19830883D09373
:1033C0002109C09320091092F1081092F00856C00C
:1033D00089E08093771149E050E069E171E08AE18A
:1033E00092E10E942F9480E290E00E942CABEC01CD
:1033F00073E5A72E72E0B72EB982A88288E090E02C
:103400009B838A83CC24C394DD24DA94DD82CC822E
:10341000EE24EA94F12CFF82EE8219861886188E2B
:103420004FEE53E160E8CE0149960E947D600BE8C3
:1034300013E019830883D0931F09C0931E0980E20B
:1034400090E00E942CABEC01B982A88289E090E068
:103450009B838A83DD82CC82FF82EE821986188666
:10346000188E4FEE53E160E8CE0149960E947D60D0
:1034700019830883D0932109C093200980912009E2
:1034800090912109DC01ED91FC910280F381E02D06
:10349000199580911E0990911F09DC01ED91FC9115
:1034A0000280F381E02D19958091AE118250823017
:1034B00040F589E190E00E942CABEC0183E592E0BD
:1034C0009983888386E090E09B838A8381E09FEFE5
:1034D0009D838C838FEF90E09F838E83198618865F
:1034E000188ECE010E94FC5F8BEB93E0998388835A
:1034F000D0931B09C0931A09CE010E94485810921C
:10350000F00880917811992787FD9095A92FB92F00
:10351000FC013897E830F10508F0CAC0EE58FF4FBB
:103520000C94C2AD82E290E00E942CABEC0183E5EA
:1035300092E09983888388E090E09B838A8381E08E
:103540009FEF9D838C838FEF90E09F838E831986FE
:103550001886188E4FEE53E164E8CE0149960E941A
:1035600027628FE793E0998388838CEF91E199A399
:1035700088A323C080E290E00E942CABEC0183E59D
:1035800092E09983888388E090E09B838A8381E03E
:103590009FEF9D838C838FEF90E09F838E831986AE
:1035A0001886188E4FEE53E167E8CE0149960E94C7
:1035B0007D608BE893E099838883D0931709C0934B
:1035C0001609A6C080E290E00E942CABEC0183E5D6
:1035D00092E09983888388E090E09B838A8381E0EE
:1035E0009FEF9D838C838FEF90E09F838E8319865E
:1035F0001886188E4FEE53E16DE0CE0149960E9479
:103600000F6187E993E0D7CF89E190E00E942CAB6E
:10361000FC0188E090E09383828381E09FEF9583B3
:1036200084838FEF90E09783868311861086108EB7
:1036300083EA93E091838083F0931709E09316095E
:103640001092E60865C08CE190E00E942CABEC0182
:1036500083E592E09983888385E090E09B838A8369
:1036600081E09FEF9D838C838FEF90E09F838E831B
:1036700019861886188ECE010E94FC5F87EC93E0B5
:103680003FC089E190E00E942CABFC0113821282C2
:10369000158214821782168211861086108E8FE58D
:1036A00092E091838083F0931709E093160930C06C
:1036B0008CE0809378114CE050E06AE171E08AE19F
:1036C00092E10E942F9489E190E00E942CABEC01E2
:1036D00083E592E09983888385E090E09B838A83E9
:1036E00081E09FEF9D838C838FEF90E09F838E839B
:1036F00019861886188ECE010E94FC5F8BEB93E032
:1037000099838883D0931709C09316091092EF0804
:103710008091160990911709DC01ED91FC910280CE
:10372000F381E02D199560918011643630F4809119
:103730001609909117090E94225B809179119927AF
:1037400087FD9095A92FB92FFC013897E830F10536
:1037500008F0F0C0E658FF4F0C94C2AD82E290E052
:103760000E942CABEC0183E592E09983888389E089
:1037700090E09B838A8381E09FEF9D838C838FEF12
:1037800090E09F838E8319861886188E4FEE53E142
:1037900064E8CE0149960E9427628FE793E09983FF
:1037A00088838CEF91E199A388A323C080E290E005
:1037B0000E942CABEC0183E592E09983888389E039
:1037C00090E09B838A8381E09FEF9D838C838FEFC2
:1037D00090E09F838E8319861886188E4FEE53E1F2
:1037E00067E8CE0149960E947D608BE893E099835B
:1037F0008883D0931509C0931409CCC080E290E06F
:103800000E942CABEC0183E592E09983888389E0E8
:1038100090E09B838A8381E09FEF9D838C838FEF71
:1038200090E09F838E8319861886188E4FEE53E1A1
:103830006DE0CE0149960E940F6187E993E0D7CFF2
:1038400089E190E00E942CABFC0189E090E0938339
:10385000828381E09FEF958384838FEF90E097834D
:10386000868311861086108E83EA93E0918380838D
:10387000F0931509E09314091092E5088BC08CE1D0
:1038800090E00E942CABEC0133E5832E32E0932EC6
:103890009982888244E0A42EB12CBB82AA82CC24D7
:1038A000C394DD24DA94DD82CC82EE24EA94F12CF8
:1038B000FF82EE8219861886188E0E94FC5F07EC44
:1038C00013E019830883D0931509C09314098CE180
:1038D00090E00E942CABEC0199828882BB82AA8284
:1038E000DD82CC82FF82EE8219861886188E0E94B5
:1038F000FC5F19830883D0931309C0931209CE018A
:103900000E94075C45C089E190E00E942CABFC015D
:1039100013821282158214821782168211861086F3
:10392000108E8FE592E091838083F0931509E093E8
:10393000140930C08CE0809379114CE050E06BE1C9
:1039400071E08AE192E10E942F9489E190E00E9467
:103950002CABEC0183E592E09983888384E090E0CE
:103960009B838A8381E09FEF9D838C838FEF90E020
:103970009F838E8319861886188ECE010E94FC5F65
:103980008BEB93E099838883D0931509C093140936
:103990001092EE088091140990911509DC01ED91C7
:1039A000FC910280F381E02D199560917F116436BE
:1039B00030F480911409909115090E94225B809146
:1039C00079118C50823000F560917A1170917B11E1
:1039D00084E00E94585E60917C1170917D1184E0BA
:1039E0000E94755E80917E11E0911409F091150995
:1039F000808F809179118D3039F480917E11E09122
:103A00001209F0911309808F8EE190E00E942CAB97
:103A1000EC01B0908511E0908911F0908A11C0906E
:103A20008711D090881183E592E09983888383E0A1
:103A300090E09B838A8381E09FEF9D838C830FEFCF
:103A400010E01F830E8319861886188ECE010E94FF
:103A5000FC5F83ED93E099838883DA8EC98EFC8EB8
:103A6000EB8EBD8ED0931109C093100960918B111C
:103A700070918C1183E00E94585E60918D1170915D
:103A80008E1183E00E94755E80918511E09110098E
:103A9000F0911109808F6091851183E00E94685F29
:103AA0008091100990911109DC01ED91FC91028047
:103AB000F381E02D199580918F118823D1F083E255
:103AC00090E00E942CABFC01809192119091931197
:103AD0002091901130919111409194115091951134
:103AE00068E070E073836283158214825783468393
:103AF00015C083E290E00E942CABFC0180919211F2
:103B000090919311209190113091911148E050E0E3
:103B1000538342831582148217830683118610868D
:103B2000108E4FEA53E051834083328F218F948F60
:103B3000838FF0930F09E0930E0980910E09909105
:103B40000F090E9426588091E6088823F9F089E140
:103B500090E00E942CABFC0188E090E0938382838C
:103B6000158214828FEF93E0978386838FEF91E025
:103B700091878087108E83EA93E091838083F0930E
:103B8000EA08E093E908CF010E94E8578091E50830
:103B9000882359F189E190E00E942CABFC0189E077
:103BA00090E093838283158214828FEF93E0978352
:103BB00086838FEF91E091878087108E83EA93E070
:103BC00091838083F093E808E093E708CF01DF91C9
:103BD000CF911F910F91FF90EF90DF90CF90BF900A
:103BE000AF909F908F900C94E857DF91CF911F91E9
:103BF0000F91FF90EF90DF90CF90BF90AF909F908C
:103C00008F9008952F923F924F925F926F927F9282
:103C10008F929F92AF92BF92CF92DF92EF92FF92DC
:103C20000F931F93CF93DF9300D0CDB7DEB7809172
:103C3000F108811119C08091F008811115C080919F
:103C4000EF08811111C08091EE0881110DC08091A3
:103C5000ED08811109C08091EC08811105C08091A7
:103C6000EB08882309F492C271E0472E71E1572EC8
:103C70001B82612C712C812C912C1A8219820FEFDE
:103C800013E0EE24EA94FF24F394F7ECAF2EF3E074
:103C9000BF2EABEB2A2EA3E03A2EF20180818823BF
:103CA00009F46BC2329720813181232B09F465C25C
:103CB00090E0FC01F797EB32F10508F05EC2EE5799
:103CC000FF4F0C94C2AD8091F108882309F455C2CE
:103CD000F981F11152C289E190E00E942CAB6C0194
:103CE00083E592E0F6019183808387E090E09383FF
:103CF00082831582148217830683F186E086108EF4
:103D0000C6010E94FC5FF60131822082D0920D092B
:103D1000C0920C09C6010E94485826C18091F00843
:103D2000882309F42AC28A81811127C289E190E09F
:103D30000E942CAB6C0183E592E0F60191838083B5
:103D400086E090E093838283158214821783068332
:103D5000F186E086108EC6010E94FC5FF60131827A
:103D60002082D0920B09C0920A09C6010E944858CD
:103D700028C18091EF08882309F4FFC19110FDC18B
:103D800089E190E00E942CAB6C0183E592E0F601A2
:103D90009183808385E090E09383828315821482EF
:103DA00017830683F186E086108EC6010E94FC5FB1
:103DB000F60131822082D0920909C0920809C60119
:103DC0000E9448582AC18091EE08882309F4D5C181
:103DD0008110D3C189E190E00E942CAB6C0183E596
:103DE00092E0F6019183808384E090E09383828364
:103DF0001582148217830683F186E086108EC60131
:103E00000E94FC5FF60131822082D0920709C092A5
:103E10000609C6010E9448582CC18091ED088823EC
:103E200009F4ABC17110A9C189E190E00E942CABEB
:103E30006C0183E592E0F6019183808382E090E05B
:103E4000938382831582148217830683F186E0862A
:103E5000108EC6010E94FC5FF60131822082D09252
:103E60000509C0920409C6010E9448582EC18091DC
:103E7000EC08882309F481C161107FC189E190E0D9
:103E80000E942CAB6C0183E592E0F6019183808364
:103E900081E090E0938382831582148217830683E6
:103EA000F186E086108EC6010E94FC5FF601318229
:103EB0002082D0920309C0920209C6010E9448588C
:103EC00030C18091EB08882309F457C1FB81F111BF
:103ED00054C189E190E00E942CAB6C0183E592E033
:103EE000F6019183808313821282158214821783D4
:103EF0000683F186E086108EC6010E94FC5FF60103
:103F000031822082D0920109C0920009C6010E942C
:103F1000485831C18091F108882309F42EC1898164
:103F200081112BC18CE190E00E942CAB6C0183E5E8
:103F300092E0F6019183808387E090E0938382830F
:103F40001582148217830683F186E086108EC601DF
:103F50000E94FC5FF601B182A082D092FF08C0925D
:103F6000FE08C6010E94075CF1E0F98306C180915A
:103F7000F008882309F401C18A818111FEC08CE117
:103F800090E00E942CAB6C0183E592E0F6019183F6
:103F9000808386E090E09383828315821482178366
:103FA0000683F186E086108EC6010E94FC5FF60152
:103FB000B182A082D092FD08C092FC08C6010E9486
:103FC000075CF1E0FA83D9C08091EF08882309F4F7
:103FD000D4C09110D2C08CE190E00E942CAB6C0157
:103FE00083E592E0F6019183808385E090E09383FE
:103FF00082831582148217830683F186E086108EF1
:10400000C6010E94FC5FF601B182A082D092FB083B
:10401000C092FA08C6010E94075C99249394ADC02F
:104020008091EE08882309F4A8C08110A6C08CE115
:1040300090E00E942CAB6C0183E592E0F601918345
:10404000808384E090E093838283158214821783B7
:104050000683F186E086108EC6010E94FC5FF601A1
:10406000B182A082D092F908C092F808C6010E94DD
:10407000075C8824839481C08091ED08882309F42B
:104080007CC071107AC08CE190E00E942CAB6C0176
:1040900083E592E0F6019183808382E090E0938350
:1040A00082831582148217830683F186E086108E40
:1040B000C6010E94FC5FF601B182A082D092F7088F
:1040C000C092F608C6010E94075C7724739455C01D
:1040D0008091EC08882309F450C061104EC08CE137
:1040E00090E00E942CAB6C0183E592E0F601918395
:1040F000808381E090E0938382831582148217830A
:104100000683F186E086108EC6010E94FC5FF601F0
:10411000B182A082D092F508C092F408C6010E9434
:10412000075C6624639429C08091EB08882329F1F9
:10413000FB81F11122C08CE190E00E942CAB6C015C
:1041400083E592E0F60191838083138212821582C7
:10415000148217830683F186E086108EC6010E94C2
:10416000FC5FF601B182A082D092F308C092F208FF
:10417000C6010E94075CF1E0FB8383E0480E511CFE
:1041800099E7491691E1590609F087CD0F900F90F4
:104190000F90DF91CF911F910F91FF90EF90DF90E3
:1041A000CF90BF90AF909F908F907F906F905F90D7
:1041B0004F903F902F9008958091FB109091FC10AC
:1041C0008093330990933409813039F461E08FE3AF
:1041D0000E9420A10E94EB110CC080913409882319
:1041E00011F062E001C060E08FE30E9420A10E9414
:1041F00011128091FD109091FE1080933A099093D6
:104200003B09813039F461E08EE30E9420A10E94D5
:104210005F120CC080913B09882311F062E001C05D
:1042200060E08EE30E9420A10E94851260E085E498
:104230000E9420A162E08CE30E9420A162E08BE357
:104240000E9420A162E080E40E9420A162E081E45B
:104250000E9420A162E082E40E9420A162E081E24B
:104260000E9420A162E084E40E9420A161E089E331
:104270000E9420A161E08AE30E9420A10E9488158B
:104280000E947C1561E085E30E9420A161E085E049
:104290000E9420A161E070E085E00E9408A061E03A
:1042A00084E00E9420A161E088E00E9420A161E0FA
:1042B00087E00E9420A161E089E20E9459A161E0AB
:1042C00089E20E9420A16A9A60E085E30E9459A1D8
:1042D00060E085E00E9459A160E084E00E9459A15D
:1042E00060E088E00E9459A160E087E00E9459A147
:1042F000729861E08BE20E9420A160E08BE20C9456
:1043000059A180918F098823D9F010928F090E94BA
:104310002B1680919309882399F06BE67DE08091BC
:104320009109909192090E9438A60E9449510E94D9
:10433000344DBC0180919109909192090C9474A61E
:10434000089585E999E00E94D9630E9457540E941C
:1043500050690E94E1698091AE118230C1F01CF475
:104360008130A9F02FC0833011F1843059F580914C
:104370001C0990911D09DC01ED91FC910680F781EB
:10438000E02D1995809118099091190914C0809118
:10439000200990912109DC01ED91FC910680F781C3
:1043A000E02D199580911E0990911F0904C08091FC
:1043B0001C0990911D09DC01ED91FC910680F781AB
:1043C000E02D19958091160990911709DC01ED9166
:1043D000FC910680F781E02D199580911409909148
:1043E0001509DC01ED91FC910680F781E02D19950E
:1043F00080910E0990910F09DC01ED91FC910680EE
:10440000F781E02D199483E898E00E945F8F0E9465
:104410001C1097CFBC0185E999E00C9489638091C9
:104420008F11882359F080910E0990910F09DC01BA
:10443000ED91FC910480F581E02D199408959091FF
:104440008F11992339F0682F80910E0990910F09EF
:104450000C94C55B08950E949587811150C00E94FD
:1044600099690E94066A882311F081E001C080E00A
:10447000E6DF0E94266A8091230990912409DC01DD
:10448000ED91FC910480F581E02D19958091AE119C
:104490008230C1F01CF48130A9F02FC0833011F1BB
:1044A000843059F580911C0990911D09DC01ED9132
:1044B000FC910480F581E02D199580911809909167
:1044C000190914C08091200990912109DC01ED9116
:1044D000FC910480F581E02D199580911E09909141
:1044E0001F0904C080911C0990911D09DC01ED9108
:1044F000FC910480F581E02D19950C9465110895C7
:104500000E947569882369F0A6DF80919409882349
:1045100041F069EE7FE080919109909192090C94AD
:1045200074A608958091AE118230C1F01CF48130E0
:10453000A9F02FC0833011F1843059F580911C0906
:1045400090911D09DC01ED91FC910480F581E02D35
:104550001995809118099091190914C0809120092A
:1045600090912109DC01ED91FC910480F581E02D11
:10457000199580911E0990911F0904C080911C0912
:1045800090911D09DC01ED91FC910480F581E02DF5
:1045900019958091230990912409DC01ED91FC91FA
:1045A000EC5BFF4F0190F081E02D1995809123097C
:1045B00090912409DC01ED91FC910084F185E02DBE
:1045C00019950E94138B0E947569811144DF8091B7
:1045D000140990911509DC01ED91FC910480F5819D
:1045E000E02D19958091160990911709DC01ED9144
:1045F000FC910480F581E02D199511CF80918F09F0
:10460000811112C08FDF81E080938F090E94F11524
:1046100080919409882341F06AE77DE080919109B7
:10462000909192090C9474A6089515CF8091180268
:104630008823A9F01092180280919409882341F0F0
:104640006DE47CE080919109909192090E9474A69A
:104650000E947569882319F00E94066AF0CE0895B9
:10466000E5CF80918F11882351F080911802882323
:1046700031F080910E0990910F090C94775B0895A9
:104680000E947569882339F00E949587811103C0C3
:10469000E8DF0C940A6A0895F3CF80918F11882384
:1046A00051F080911802882331F080910E09909189
:1046B0000F090C949E5B08950E949587811123C079
:1046C0000E9479698823F9F0809123099091240947
:1046D000DC01ED91FC910280F381E02D1995409170
:1046E000A9115091AA114115510551F060E070E0F7
:1046F00020E433E285E999E00E946D63CEDF01C0DA
:10470000BFDF0C94651108950E9475698111A3CED5
:10471000D3CFFACFD1CF0E947569882319F0BDDFBE
:104720000C94266A08950E943786882381F10E949E
:10473000A685882349F00E949587811128C0809121
:104740009508882399F008950E94958781111FC0CC
:1047500080919409882341F06AE371E18091910985
:10476000909192090E9474A60C94828A82E08093B0
:10477000950880919409882341F066E471E1809165
:104780009109909192090E9474A6C5DFEDCF08951A
:10479000CACF0E94066A8111BECF72CFFACFBBCFBB
:1047A00080911802811118C081E0809318028091D5
:1047B0009409882341F06DE57CE080919109909106
:1047C00092090E9474A60E947569882329F00E94AC
:1047D000066A811146CF61CF089580911802811138
:1047E00025CFDECFFACFDCCF20918F11222389F0A5
:1047F00020911802222369F0A0910E09B0910F09AF
:10480000ED91FC9111970190F081E02DBC01CD015B
:104810001994089580918F11882351F08091180286
:10482000882331F080910E0990910F090C945E0F4E
:10483000089580918F11882301F1809118028823B7
:10484000E1F0809196119091971118161906ACF429
:1048500080910E0990910F090E945E0F80910E09C0
:1048600090910F09DC01ED91FC916091961170918E
:1048700097110190F081E02D19940895CF93DF9363
:104880008091C011843050F01092C01140E050E08F
:1048900062E671E08AE192E10E942F94C091C0111A
:1048A000C13041F1D8F0C230E9F1C33009F45CC045
:1048B0001092C01140E050E062E671E08AE192E1BE
:1048C0000E942F9485E090E00E942CABEC012BE637
:1048D00032E0FC0121933193CF013AC085E090E0B2
:1048E0000E942CABEC012BE632E0DC012D933D93D2
:1048F000CD012EC08AE090E00E942CAB23E036E090
:10490000FC01318320832FEE33E1318720879093A0
:10491000240980932309C093ED08C093EC08C09349
:10492000EB0828C086E090E00E942CAB21E736E03F
:10493000DC012D933C93909324098093230980E01C
:104940000E94D65C81E08093ED088093EC0810C053
:1049500065E979E00E94B68089ED92E099838883C9
:10496000D0932409C09323091092ED081092EC080B
:104970001092EB088091230990912409DC01ED91BC
:10498000FC910190F081E02DDF91CF9119948091FD
:10499000230990912409DC01ED91FC91EA59FF4F24
:1049A0000190F081E02D1994F2CF8091230990912C
:1049B0002409DC01ED91FC91EA59FF4F0190F0814F
:1049C000E02D1994F2CF68EB7BE0809191099091F2
:1049D00092090C9438A68091230990912409DC0156
:1049E000ED91FC9102A4F3A5E02D19958091940915
:1049F000882349F0E8DF6EE37CE080919109909193
:104A000092090C9474A60895E6CF809123099091A1
:104A10002409DC01ED91FC9104A4F5A5E02D199584
:104A200080919409882349F0CEDF6AE27CE080918E
:104A30009109909192090C9474A60895E6CF809103
:104A4000230990912409DC01ED91FC9106A4F7A5BE
:104A5000E02D199580919409882349F0B4DF61E233
:104A60007CE080919109909192090C9474A608952C
:104A7000E6CF8091230990912409DC01ED91FC910E
:104A800000A8F1A9E02D199580919409882349F097
:104A90009ADF6FE17CE080919109909192090C94EA
:104AA00074A60895E6CF8091230990912409DC0132
:104AB000ED91FC9102A8F3A9E02D1995809194093C
:104AC000882349F080DF6BE07CE080919109909130
:104AD00092090C9474A60895E6CF809123099091D1
:104AE0002409DC01ED91FC9104A8F5A9E02D1995AC
:104AF00080919409882349F066DF62E07CE0809130
:104B00009109909192090C9474A60895E6CF809132
:104B1000230990912409DC01ED91FC9106A8F7A9E5
:104B2000E02D199580919409882349F04CDF60E0CD
:104B30007CE080919109909192090C9474A608955B
:104B4000E6CF8091230990912409DC01ED91FC913D
:104B500000ACF1ADE02D199580919409882349F0BE
:104B600032DF6CEE7BE080919109909192090C9478
:104B700074A60895E6CF8091230990912409DC0161
:104B8000ED91FC9102ACF3ADE02D19958091940963
:104B9000882349F018DF63EE7BE0809191099091C2
:104BA00092090C9474A60895E6CF80912309909100
:104BB0002409DC01ED91FC9104ACF5ADE02D1995D3
:104BC00080919409882349F0FEDE61EE7BE08091BC
:104BD0009109909192090C9474A60895E6CF809162
:104BE000230990912409DC01ED91FC9106ACF7AD0D
:104BF000E02D199580919409882349F0E4DE6DEC4D
:104C00007BE080919109909192090C9474A608958B
:104C1000E6CF8091230990912409DC01ED91FC916C
:104C2000E05CFF4F0190F081E02D1995809194098F
:104C3000882349F0C8DE64EC7BE080919109909173
:104C400092090C9474A60895E4CF2F923F924F924C
:104C50005F926F927F928F929F92AF92BF92CF920C
:104C6000DF92EF92FF920F931F93CF93DF931F92E8
:104C70001F92CDB7DEB7A1E0B1E18DE399E09A8351
:104C8000898319EA612E14E3712E06E5802E0CE368
:104C9000902E29E53CE347E55CE36DE574E30CEE1B
:104CA0001BE38AEEE82E8BE3F82E95EBC92E9DE0F0
:104CB000D92E2C90222009F4BAC25D0192E0A91AE3
:104CC000B108F501A080B180AB2809F4B0C2312C45
:104CD000C10101978336910508F0A9C283559F4F02
:104CE000FC010C94C2AD89E893E2E981FA819183D9
:104CF00080839DC28AE893E2E981FA81918380836F
:104D000096C285E193E2E981FA81918380838FC223
:104D10008EEC93E2E981FA819183808388C28CE4EE
:104D200093E2E981FA819183808381C28FEC93E2DF
:104D3000E981FA81918380837AC288EC93E2E981E8
:104D4000FA819183808373C282EA9FE0E981FA81CC
:104D5000918380836CC28DEE9FE0E981FA8191831B
:104D6000808365C28DEF9FE0E981FA819183808322
:104D70005EC28BE79FE0E981FA819183808357C20D
:104D80008BE89FE0E981FA819183808350C28AEBAE
:104D90009FE0E981FA819183808349C282ED9FE09F
:104DA000E981FA819183808342C288ED9FE0E981A5
:104DB000FA81918380833BC28FE993E1E981FA8193
:104DC0009183808334C283E793E1E981FA819183FF
:104DD00080832DC280E993E1E981FA819183808308
:104DE00026C282ED93E1E981FA81918380831FC21B
:104DF00081EB93E1E981FA819183808318C283EC8E
:104E000093E1E981FA819183808311C28BE294E17D
:104E1000E981FA81918380830AC284E094E1E98187
:104E2000FA819183808303C28CE194E1E981FA8164
:104E300091838083FCC18FE894E1E981FA819183B9
:104E40008083F5C181E494E1E981FA8191838083D3
:104E5000EEC185EA9CE0E981FA8191838083E7C114
:104E60008AEB9CE0E981FA8191838083E0C183EA47
:104E700094E1E981FA8191838083D9C182EC94E144
:104E8000E981FA8191838083D2C18FE794E1E9813E
:104E9000FA8191838083CBC18BEE94E1E981FA8121
:104EA00091838083C4C18AE195E1E981FA8191838C
:104EB0008083BDC185E495E1E981FA819183808396
:104EC000B6C183EF93E3E981FA8191838083AFC117
:104ED00084E095E2E981FA8191838083A8C18EE123
:104EE00095E2E981FA8191838083A1C188E395E20B
:104EF000E981FA81918380839AC182E595E2E98113
:104F0000FA819183808393C18CE695E2E981FA81ED
:104F1000918380838CC186E895E2E981FA8191834F
:104F2000808385C180EA95E2E981FA81918380835B
:104F30007EC18AEB95E2E981FA819183808377C112
:104F400084ED95E2E981FA819183808370C18EEED0
:104F500095E2E981FA819183808369C188E096E2D4
:104F6000E981FA819183808362C184E296E2E981DA
:104F7000FA81918380835BC180E192E1E981FA81CA
:104F80009183808354C18AEE91E1E981FA81918312
:104F900080834DC181E092E1E981FA819183808330
:104FA00046C184E892E1E981FA81918380833FC11F
:104FB0008EE592E1E981FA819183808338C185E7AA
:104FC00092E1E981FA819183808331C18DE29AE295
:104FD000E981FA81918380832AC18CE59AE2E98193
:104FE000FA819183808323C18AEF9EE0E981FA816F
:104FF000918380831CC186EE9EE0E981FA819183D2
:10500000808315C182ED9EE0E981FA8191838083DE
:105010000EC18FE39EE0E981FA819183808307C10D
:1050200087EC9DE0E981FA819183808300C189ED5D
:105030009DE0E981FA8191838083F9C08BEE9DE048
:10504000E981FA8191838083F2C087EF9DE0E98155
:10505000FA8191838083EBC083E09EE0E981FA814D
:1050600091838083E4C08FE09EE0E981FA8191839F
:105070008083DDC08BE19EE0E981FA8191838083AA
:10508000D6C087E29EE0E981FA8191838083CFC018
:1050900083E39EE0E981FA8191838083C8C089E43B
:1050A0009DE0E981FA8191838083C1C08BE59DE019
:1050B000E981FA8191838083BAC08DE69DE0E98120
:1050C000FA8191838083B3C08FE79DE0E981FA8103
:1050D00091838083ACC081E99DE0E981FA8191836D
:1050E0008083A5C083EA9DE0E981FA819183808372
:1050F0009EC0E981FA81D182C08299C0E981FA819A
:10510000F182E08294C0E981FA81118300838FC02B
:1051100089EE9BE3E981FA819183808388C0E981EC
:10512000FA817183608383C0E981FA81518340836E
:105130007EC0E981FA813183208379C0E981FA81D7
:105140009182808274C0E981FA81718260826FC02D
:105150008CEE9AE2E981FA819183808368C08AEFBC
:105160009AE2E981FA819183808361C08EE09FE0B9
:10517000E981FA81918380835AC086E39FE0E981C7
:10518000FA819183808353C083EB9BE4E981FA81A8
:10519000918380834CC080EB9EE0E981FA8191830A
:1051A000808345C08CE99EE0E981FA819183808308
:1051B0003EC088EC9EE0E981FA819183808337C00C
:1051C00081E491E1E981FA819183808330C083E4B5
:1051D00091E1E981FA819183808329C08DE491E195
:1051E000E981FA819183808322C083EF93E2E98190
:1051F000FA81918380831BC080E393E2E981FA8185
:105200009183808314C082EF93E2E981FA819183D4
:1052100080830DC084ED94E2E981FA8191838083DB
:1052200006C082EE94E2E981FA819183808313962D
:10523000E981FA813296FA83E983F1E1A937BF0760
:1052400009F037CD0F900F90DF91CF911F910F9103
:10525000FF90EF90DF90CF90BF90AF909F908F9096
:105260007F906F905F904F903F902F900895E1E076
:10527000F1E180E09081992339F0DF0112972D91BF
:105280003C91232B09F08F5F339691E1E937F907C1
:1052900089F7089589508C3130F4E82FF0E0ED5C07
:1052A000FD4F8081089580E008959C01019784322C
:1052B000910508F18356910984389340D0F0283E37
:1052C00083E03807C0F0C90168EE73E00E945DAD6D
:1052D00048E15CEF649FC001659F900D749F900D45
:1052E0001124820F931F6AE070E00E9471AD862F37
:1052F000089582E0089580E008959C0101978497C5
:1053000010F4822F0895C90184569109843893407E
:1053100040F4C90164E670E00E945DAD822F94E61E
:105320001BC0283E43E03407D8F0C90168EE73E0A3
:105330000E945DAD88E19CEF689FA001699F500DC0
:10534000789F500D1124420F531FCA016AE070E08C
:105350000E9471AD842F9AE0699F801911240895ED
:1053600080E00895AF92BF92CF92DF92EF92FF92CA
:105370000F931F9327E0289FF001299FF00D112420
:10538000E955F34F828193810580F681E02D2181DB
:105390003281E380F4808217930734F0B7018E15D1
:1053A0009F051CF4BC0101C0B901882777FD8095D9
:1053B000982F0027F7FC0095102F442737FD4095C4
:1053C000542F1F921F92E3E0EF93EFEFEF93A12C86
:1053D000B12C65010E94BDA80F900F900F900F9007
:1053E000CB011F910F91FF90EF90DF90CF90BF9076
:1053F000AF900895AF92BF92CF92DF92EF92FF925B
:105400000F931F93811524E0920710F08FEF93E024
:10541000BC0180E090E01F921F921F922EE02F931C
:10542000A12CB12C6501A394EE24EA9413E0F12E93
:1054300000E010E020E030E0A9010E94BDA8862F26
:105440000F900F900F900F901F910F91FF90EF9082
:10545000DF90CF90BF90AF900895CF932091170227
:10546000213019F42091981104C0223019F52091AF
:105470009E112223F9F0BEDFC82F0E947A65C8175B
:10548000C9F08C2F0E94746580919409882391F053
:105490006AEE7AE080919109909192090E9438A673
:1054A0004AE050E06C2F8091910990919209CF9140
:1054B0000C9460A7CF910895CF93209117022130CB
:1054C00019F420919B1104C0223019F52091A111EB
:1054D0002223F9F08FDFC82F0E947D65C817C9F01D
:1054E0008C2F0E94776580919409882391F063ED59
:1054F0007AE080919109909192090E9438A64AE041
:1055000050E06C2F8091910990919209CF910C9469
:1055100060A7CF9108950E94E5678093AD11482F51
:105520006FE471E08AE192E10E941B94809117027E
:10553000813099F40E947A6580939911482F6BE32A
:1055400071E08AE192E10E941B940E947D65809344
:105550009C11482F6EE371E012C00E947A6580931F
:105560009F11482F61E471E08AE192E10E941B944F
:105570000E947D658093A211482F64E471E08AE166
:1055800092E10E941B9440919E084093BB116DE5EF
:1055900071E08AE192E10E941B9440919D08409342
:1055A000BD116FE571E08AE192E10E941B94409188
:1055B000101262EB71E08AE192E10C941B948091ED
:1055C0009409882341F063E97AE0809191099091F0
:1055D00092090C9474A60895F2CF809194098823BF
:1055E00041F063E87AE080919109909192090C94DE
:1055F00074A60895F2CFCF93CDE26DE47AE0809166
:105600009109909192090E9438A6C150B1F78091FA
:105610009109909192090E9471A6809191099091AF
:105620009209DC01ED91FC910284F385E02DCF918C
:10563000199469E47AE080919109909192090C940F
:1056400038A667E47AE080919109909192090C94D0
:1056500038A61F93CF93DF931F92CDB7DEB710E02C
:10566000181729F08983EDDF1F5F8981F9CF0F902B
:10567000DF91CF911F9108958111EBCF0895CF92C3
:10568000DF92FF920F931F93CF93DF931F921F928E
:10569000CDB7DEB76B0143E658E761E07727480FE7
:1056A000511D611D711D6BBFFA014791FF24F394D9
:1056B000411101C0F12CC6010197849758F565E7A7
:1056C0007BE080919109909192090E9438A68C2DDF
:1056D0000E94224DBC0180919109909192090E94F3
:1056E00038A68C2DD7DD90E081559D4EAA2797FDD9
:1056F000A095BA2FABBFFC0187919EE0981B892F24
:105700000F900F90DF91CF911F910F91FF90DF903D
:10571000CF90B2CFC601845691098438934008F0E7
:105720004FC065E67BE080919109909192090E94BB
:1057300038A6C60164E670E00E945DAD6130710577
:1057400031F06230710559F461E67BE002C063E636
:105750007BE080919109909192090E9438A669DFBF
:10576000FF2021F1C601C9DD81110AC06DE57BE092
:1057700080919109909192090E9438A687E00CC00F
:10578000813009F097C06AE57BE0809191099091A2
:1057900092090E9438A688E00F900F90DF91CF9178
:1057A0001F910F91FF90DF90CF9053CF61E57BE089
:1057B00080919109909192090E9438A682E0ECCFE5
:1057C00088EEC81683E0D80608F474C0C60168EEF7
:1057D00073E00E945DAD8B0164E47BE080919109F0
:1057E000909192090E9438A60A3011050CF429DF25
:1057F0004AE050E0B80180919109909192090E948D
:1058000038A717DF0091910910919209FF2009F440
:105810003DC0C60172DD282FC6012A8346DD382F20
:105820006FE37BE0C80139830E9438A639812A8161
:10583000333069F03530D1F03230E1F580919109A3
:1058400090919209243048F566E37BE028C023302C
:1058500018F464E27BE015C0233019F46BE17BE0BF
:1058600010C0243038F162E17BE00BC04AE050E028
:10587000622F80919109909192090E945AA76AE043
:105880007BE0809191099091920909C061E07BE0F1
:10589000C8010E9438A684E07FCF6DE27BE00F90C4
:1058A0000F90DF91CF911F910F91FF90DF90CF90DC
:1058B0000C9438A60F900F90DF91CF911F910F910C
:1058C000FF90DF90CF900895809191099091920977
:1058D0000C9471A68F929F92AF92BF92CF92DF925B
:1058E000EF92FF920F931F93CF93DF93CDB7DEB765
:1058F00062970FB6F894DEBF0FBECDBF0E94DF9354
:1059000026E040E052EC61E070E085EB92E10E941D
:10591000C2A24091F8115091F9116091FA11709161
:10592000FB1126E082E593E10E94C2A24091FC11A6
:105930005091FD116091FE117091FF1126E08FEEE4
:1059400093E10E94C2A24091001250910112609115
:1059500002127091031226E08CE894E10E94C2A228
:1059600060E979E083ED9BE00E94B9940E941C10ED
:105970008091151280939309109294090E94DC2063
:105980000E947C1583E898E00E945F8F44E75EE008
:1059900060E070E083E898E00E94D98F882309F4E2
:1059A00038C00E94EF9390DF8FDF25DE6FE972E150
:1059B00080919109909192090E9438A601E010E02F
:1059C0000E9484150E947C156EEE72E080E090E0EB
:1059D0000E94499F6CE972E180919109909192092E
:1059E0000E9438A60E9488150E9480150530110576
:1059F00031F064EF71E080E090E00E94499F0F5F1A
:105A00001F4F06301105E1F65FDFF5DD5DDF5CDF7E
:105A100006C083E898E00E94BD8F8111B3CF109239
:105A2000800082E0809381008FE286BB10926F003D
:105A300010928500109284009BE29093A0009AE05F
:105A40009093A10089BB109272001092A500109251
:105A5000A4001092A9001092A8001092AB0010921E
:105A6000AA001092AD001092AC0099EA9093200128
:105A700091E0909321018ABB10927300109225014E
:105A800010922401109229011092280110922B01EA
:105A900010922A0110922D0110922C010E94AA5CF2
:105AA0000E94D11685E999E00E94764D4091AB1194
:105AB0006091AD118091AE110E9433658091170203
:105AC0000E94FE10409191095091920960919309B2
:105AD0008091A7119091A8110E9425696091910968
:105AE00070919209809193090E94B4690E943E24AA
:105AF0000E94021E0E94AA10898386E0EAEEF1E16C
:105B0000DE01129601900D928A95E1F78091E311E2
:105B100088878091F31189878091E4118A87809129
:105B2000E5118B878091E6118C878091E7118D8735
:105B30008091E8118E878091E9118F878091F01113
:105B4000888B8091F1119091F2119A8B898B85E964
:105B500099E09F938F93809124098F9380912309DB
:105B60008F93809111098F93809110098F93809169
:105B700011128F9380910B128F9380910A128F9341
:105B8000809114128F93809113128F9380918411BE
:105B90008F93809183118F93809186118F93809141
:105BA00081118F93809182118F9389809A80AB802D
:105BB000BC80CD80DE80EF80F88409851A852B8536
:105BC0003C854D855E856F85788989899A890E9493
:105BD000AB884DDB80933C0938D80E949D118091A1
:105BE000230990912409DC01ED91FC91E85BFF4FC2
:105BF0004091C3115091C4116091C1117091C211B3
:105C00000190F081E02D199580912309909124094C
:105C1000DC01ED91FC91E65BFF4F4091C711509183
:105C2000C8116091C5117091C6110190F081E02DED
:105C300019958091230990912409DC01ED91FC9143
:105C4000E45BFF4F4091CB115091CC116091C91191
:105C50007091CA110190F081E02D1995809123096E
:105C600090912409DC01ED91FC91E25BFF4F4091A2
:105C7000D6115091D7116091D4117091D511019026
:105C8000F081E02D19958091230990912409DC0180
:105C9000ED91FC91E05BFF4F4091DA115091DB11E7
:105CA0006091D8117091D9110190F081E02D199572
:105CB0008091230990912409DC01ED91FC91EE5A29
:105CC000FF4F4091DE115091DF116091DC11709116
:105CD000DD110190F081E02D1995809123099091BB
:105CE0002409DC01ED91FC91EC5AFF4F0190F08109
:105CF000E02D6091CD11199580912309909124098F
:105D0000DC01ED91FC91EA5AFF4F0190F081E02D0A
:105D10006091CE1119958091230990912409DC019D
:105D2000ED91FC91E85AFF4F0190F081E02D6091D8
:105D3000CF1119958091230990912409DC01ED91EF
:105D4000FC91E65AFF4F0190F081E02D6091E01147
:105D500019958091230990912409DC01ED91FC9122
:105D6000E45AFF4F0190F081E02D6091E111199507
:105D70008091230990912409DC01ED91FC91E25A74
:105D8000FF4F0190F081E02D6091E2111995809113
:105D9000230990912409DC01ED91FC9100A4F1A567
:105DA000E02D6091D11119958091230990912409DA
:105DB000DC01ED91FC91068CF78DE02D6091D21104
:105DC00019958091230990912409DC01ED91FC91B2
:105DD00004A0F5A1E02D6091D31119950FB6F894A8
:105DE000DEBF0FBECDBF8091BA11882331F0809104
:105DF00079118D3011F01092BA1110929F08109203
:105E0000A0088091BB1180939E088091BD11809362
:105E10009D086091081270E080E090E01F921F9250
:105E20001F922FEF2F93A12CB12C650114E6E12EC8
:105E3000F12C00E010E020E030E0A9010E94BDA8B4
:105E400060932B090F900F900F900F908091071285
:105E500081110E94EA130E94FE220E941A9F6B0188
:105E60007C0110E011110FC080919309882359F033
:105E70002BE83EE040ED57E060E070E085E999E016
:105E80000E946D6311E00E94D594882341F00E9426
:105E90002B160E947C150E944E9D0E94F1150E94B7
:105EA0004B53029711F00E947B4D0E9403220E94E7
:105EB0004B530297B9F60E941A9F6C197D098E09FF
:105EC0009F096C3B72408105910560F20E9481211F
:105ED0000E947C150E944651811104C08EE590E11C
:105EE0000E9480510E944C5186E30E94E39FBC01B6
:105EF000882777FD8095982F0E9479A82DEE3BE0AA
:105F000048EE53E060E070E085E999E062960FB6F4
:105F1000F894DEBF0FBECDBFDF91CF911F910F91DF
:105F2000FF90EF90DF90CF90BF90AF909F908F90B9
:105F30000C946D632091910930919209882319F096
:105F400062E47AE002C06CE37AE0C9010C9438A6FE
:105F5000F1DF80919109909192090C9471A62F9292
:105F60003F924F925F926F927F928F929F92AF92E9
:105F7000BF92CF92DF92EF92FF920F931F93CF9336
:105F8000DF9300D0CDB7DEB7782E192F0E94922272
:105F90000E9488150E947C15809191099091920928
:105FA0000E9471A628DBC72CD12E23E0C216D10493
:105FB00009F449C084E0C816D10409F089C08CE115
:105FC00090E00E942CAB9B838A8383E592E0AA81B8
:105FD000BB8111969C938E931396DC92CE9212976E
:105FE00081E09FEF15969C938E9314978FEF90E02E
:105FF00017969C938E93169719961C921E9218973B
:1060000058961C925897CD010E94FC5F87EC93E054
:10601000EA81FB8191838083E0911409F091150955
:10602000608C84E00E94925E8C0184E00E94A25EFB
:106030007C016AE47DE080919109909192090E942F
:1060400074A6212C62C08CE190E00E942CAB9B8353
:106050008A8383E592E0AA81BB8111969C938E93FB
:106060001396DC92CE92129781E09FEF15969C9347
:106070008E9314978FEF90E017969C938E931697BC
:1060800019961C921E92189758961C925897CD01FB
:106090000E94FC5F87EC93E0EA81FB81918380831F
:1060A000E0911009F0911109608C83E00E94925EEA
:1060B0008C0183E00E94A25E7C0167E37DE0809119
:1060C0009109909192090E9474A6222423941DC0E4
:1060D0006EE17DE080919109909192090F900F906F
:1060E0000F90DF91CF911F910F91FF90EF90DF9074
:1060F000CF90BF90AF909F908F907F906F905F9068
:106100004F903F902F900C9474A675DA61E17DE07A
:1061100080919109909192090E9474A665E07DE0BA
:1061200080919109909192090E9438A64AE050E02E
:10613000B80180919109909192090E943FA769EF5F
:106140007CE080919109909192090E9438A64AE0E2
:1061500050E0B70180919109909192090E943FA768
:106160006DEE7CE080919109909192090E9438A691
:10617000862DEEDE80919109909192090E9471A680
:10618000AA81BB81ED91FC9111970280F381E02DF2
:10619000CD011995872D0E94485E8D3D954090F464
:1061A00064E378E0872D0E94755EB7018A819B8148
:1061B0000E94F05B6CED75E0872D0E94585E6110C7
:1061C00012C013C064E873E0872D0E94585EB801C6
:1061D0008A819B810E94F05B6CED75E0872D0E94A7
:1061E000755E611002C0512C02C0552453943324B3
:1061F0003394412C21E029830E947C538091100D1F
:10620000882369F1AA81BB81ED91FC91119760917E
:10621000150D7091160D0190F081E02DCD011995AD
:10622000872D0E94485E8D3DB5E09B0764F484385D
:10623000E3E09E0794F08C018D3DF5E09F077CF034
:106240000CED15E00CC07C01853328E092073CF092
:1062500054E3E52E58E0F52E02C004E813E029814E
:1062600021111FC08091060D8823C9F1E0910D0D09
:10627000F0910E0D858196814091090D50910A0D86
:106280009C0121533109421753074CF1C1968417E1
:1062900095072CF10E941A9F681579058A059B05C0
:1062A000F0F08091060D8823C1F04091090D5091C6
:1062B0000A0DE0910D0DF0910E0D858196819C01E6
:1062C000285C3109421753072CF088539F4F8417DD
:1062D00095071CF481E0582605C021E0298344205D
:1062E00009F468C05520D9F16620E9F064E873E04C
:1062F000872D0E94585E222009F448C060918911C0
:1063000070918A1141E0872D0E94B25E0E940322A3
:106310008A819B810E94F55B08171907BCF3872DC2
:106320000E94DF5F33C064E378E0872D0E94755ED2
:106330002220E1F06091891170918A1140E0872D4F
:106340000E94B25E0E9403228A819B810E94F55BBB
:106350008E159F05BCF3872D0E94DF5F07C0662066
:1063600081F064E378E0872D0E94755EB7018A8131
:106370009B810E94F05B6CED75E0872D0E94585E5A
:106380000FC064E873E0872D0E94585EB8018A81CF
:106390009B810E94F05B6CED75E0872D0E94755E1D
:1063A0000E941A9F4B015C0188EC880E911CA11C75
:1063B000B11C19823320D9F18091FC0C8823A9F1FA
:1063C0004091FF0C5091000DE091030DF091040DF0
:1063D000858196819C01285C3109421753072CF076
:1063E00088539F4F8417950704F581E068268091B4
:1063F000910990919209662039F06EED7CE00E943F
:1064000074A682E090E006C06CEC7CE00E9474A66A
:1064100081E090E00E94B1150E941A9FAA81BB8181
:1064200058966C924424439403C0412C1EC0412CC6
:106430008091FC0C882309F491C1E091030DF09147
:10644000040D258136814091FF0C5091000DC9014A
:10645000C197481759070CF481C12F5C3F4F332473
:106460003394241735070CF479C10E94575483E8FC
:1064700098E00E945F8F85E999E00E94D96383E8E4
:1064800098E00E94C58F882309F4B6CE83E898E08F
:106490000E945F8F83E898E00E94CF8F8823B1F33A
:1064A000B3E0CB16D10409F480C0E4E0CE16D104E9
:1064B00009F0E6C010937B1100937A11F0927D11E0
:1064C000E0927C1160927E11A8016CE171E08AE19A
:1064D00092E10E942F94A7016EE171E08AE192E1BE
:1064E0000E942F94462D60E271E08AE192E10E94C1
:1064F0001B94B80184E00E94585EB70184E00E94BA
:10650000755EE0911409F0911509608E8091791102
:106510008D3029F4E0911209F0911309608E6CED31
:1065200075E0872D0E941F5E66E970E080E090E0D4
:106530000E94499F809179118D3059F5872D0E94D5
:10654000485EA0911409B09115098D3D95404CF01D
:10655000ED91FC9111970190F081E02D6FEF7FEFAD
:1065600008C0ED91FC9111970190F081E02D61E060
:1065700070E0CD0119958091140990911509DC0105
:10658000ED91FC910190F081E02D60E070E01995B3
:1065900077C08091140990911509DC01ED91FC916F
:1065A0000480F581E02D19956BC010938C11009338
:1065B0008B11F0928E11E0928D1160928511A801DD
:1065C0006DE271E08AE192E10E942F94A7016FE2EF
:1065D00071E08AE192E10E942F94462D67E271E01A
:1065E0008AE192E10E941B94B80183E00E94585E08
:1065F000B70183E00E94755E80918511E0911009DA
:10660000F0911109808F6091851183E00E94685F8D
:10661000872D0E94485E5C0180918511811105C023
:106620008091851181112CC007C0872D0E94925E38
:10663000A816B90639F4F4CF872D0E94A25EA816D9
:10664000B906F1F080918511882309F489C0609121
:10665000891170918A1141E0872D0E94B25E0E94DB
:1066600003228A819B810E94F55B08171907BCF3FE
:10667000872D0E94DF5FB8018A819B810E94F05BB9
:1066800080919109909192090E9471A60E94FB2A23
:10669000B3E0CB16D10439F0E4E0CE16D10459F4BE
:1066A00062EB7CE002C06BE97CE080919109909103
:1066B00092090E9474A60E94FB2A60E97CE0809106
:1066C0009109909192090E9474A664E87CE08091FF
:1066D0009109909192090E9438A64AE050E0B801D1
:1066E00080919109909192090E943FA768E77CE010
:1066F00080919109909192090E9438A64AE050E059
:10670000B70180919109909192090E943FA76CE690
:106710007CE080919109909192090E9438A6862D83
:1067200017DC80919109909192090E9471A60F90B7
:106730000F900F90DF91CF911F910F91FF90EF90ED
:10674000DF90CF90BF90AF909F908F907F906F9091
:106750005F904F903F902F900C948015312C85CEF8
:106760006091891170918A1140E0872D0E94B25E7C
:106770000E9403228A819B810E94F55B8E159F05F2
:10678000BCF3872D0E94DF5FB70176CF209191097E
:1067900030919209882319F068E37AE002C065E33A
:1067A0007AE0C9010C9438A6F1DF809191099091AB
:1067B00092090C9471A64AE050E0682F80919109EB
:1067C000909192090E945AA763E37AE0809191091F
:1067D000909192090C9438A6EEDF809191099091E6
:1067E00092090C9471A6AF92BF92CF92DF92EF9272
:1067F000FF920F931F93CF93BC0180E090E01F9214
:106800001F921F9224E62F93A12CB12C6501EE2438
:10681000EA9413E0F12E00E010E020E030E0A9015E
:106820000E94BDA8C62F262F30E080911408281B97
:10683000310937FF03C03195219531090F900F9031
:106840000F900F902330310574F1C33020F0C23621
:1068500018F0C4E601C0C0E080912309909124099A
:10686000DC01ED91FC91EC59FF4F0190F081E02D9E
:106870006C2F1995C093140880919409882399F07E
:1068800060E47CE080919109909192090E9438A681
:106890008C2FCF911F910F91FF90EF90DF90CF90B1
:1068A000BF90AF9099CFCF911F910F91FF90EF9034
:1068B000DF90CF90BF90AF900895AF92BF92CF92EC
:1068C000DF92EF92FF920F931F93CF93BC0180E072
:1068D00090E01F921F921F9224E62F93A12CB12CBF
:1068E0006501A394EE24EA9413E0F12E00E010E099
:1068F00020E030E0A9010E94BDA8C62F0F900F90A4
:106900000F900F9080919E088C17C9F0C0939E083D
:1069100080919409882399F06AEB7AE0809191093B
:10692000909192090E9438A68C2FCF911F910F91C0
:10693000FF90EF90DF90CF90BF90AF904DCFCF9171
:106940001F910F91FF90EF90DF90CF90BF90AF908D
:106950000895AF92BF92CF92DF92EF92FF920F9382
:106960001F93CF93BC0180E090E01F921F921F9273
:1069700024E62F93A12CB12C6501A394EE24EA9474
:1069800013E0F12E00E010E020E030E0A9010E94C9
:10699000BDA8C62F0F900F900F900F9080919D086B
:1069A0008C17C9F0C0939D0880919409882399F0B1
:1069B00063EA7AE080919109909192090E9438A649
:1069C0008C2FCF911F910F91FF90EF90DF90CF9080
:1069D000BF90AF9001CFCF911F910F91FF90EF909B
:1069E000DF90CF90BF90AF900895CF93DF9300D00A
:1069F00000D0CDB7DEB780919109909192090E94A5
:106A000071A60E94FB2A6AE07AE080919109909138
:106A100092090E9438A669E272E0CE0101960E94B6
:106A20006AA9BE016F5F7F4F809191099091920991
:106A30000E9484A6CE0101960E9403A926960FB655
:106A4000F894DEBF0FBECDBFDF91CF910895809146
:106A50009109909192090E9471A60E94FB2A6CEF05
:106A600079E080919109909192090E9438A60E9444
:106A700049510E94344DBC01809191099091920935
:106A80000E9474A60E94FB2A66EC79E0809191092D
:106A9000909192090E9474A60E94FB2A6AEB79E009
:106AA00080919109909192090E9438A6E091030D7E
:106AB000F091040D81819281883E934014F40E94EC
:106AC000212BE091030DF091040D618172814AE068
:106AD00050E080919109909192090E9438A784E03A
:106AE0000E94292BE091030DF091040D65817681C0
:106AF0004AE050E080919109909192090E9438A754
:106B000085E00E94292BE091030DF091040D638133
:106B100074814AE050E080919109909192090E941D
:106B200038A784E00E94292BE091030DF091040D19
:106B30004AE050E0678180919109909192090E940A
:106B40005AA788E00E94292BE091030DF091040DD3
:106B50008085FED96EEA79E0809191099091920941
:106B60000E9438A6E0910D0DF0910E0D8181928169
:106B7000883E934014F40E94212BE0910D0DF0917A
:106B80000E0D618172814AE050E0809191099091EF
:106B900092090E9438A784E00E94292BE0910D0DF4
:106BA000F0910E0D658176814AE050E08091910967
:106BB000909192090E9438A785E00E94292BE091CC
:106BC0000D0DF0910E0D638174814AE050E08091CB
:106BD0009109909192090E9438A784E00E94292B84
:106BE000E0910D0DF0910E0D4AE050E0678180912B
:106BF0009109909192090E945AA788E00E94292B3E
:106C0000E0910D0DF0910E0D8085A2D962EA79E038
:106C100080919109909192090E9438A6E091170DF8
:106C2000F091180D81819281883E934014F40E9466
:106C3000212BE091170DF091180D618172814AE0CE
:106C400050E080919109909192090E9438A784E0C8
:106C50000E94292BE091170DF091180D6581768126
:106C60004AE050E080919109909192090E9438A7E2
:106C700085E00E94292BE091170DF091180D63819A
:106C800074814AE050E080919109909192090E94AC
:106C900038A784E00E94292BE091170DF091180D80
:106CA0004AE050E0678180919109909192090E9499
:106CB0005AA788E00E94292BE091170DF091180D3A
:106CC000808546D966E979E0809191099091920991
:106CD0000E9438A6E091210DF091220D81819281D0
:106CE000883E934014F40E94212BE091210DF091F5
:106CF000220D618172814AE050E08091910990916A
:106D000092090E9438A784E00E94292BE091210D6E
:106D1000F091220D658176814AE050E080919109E1
:106D2000909192090E9438A785E00E94292BE0915A
:106D3000210DF091220D638174814AE050E0809131
:106D40009109909192090E9438A784E00E94292B12
:106D5000E091210DF091220D4AE050E06781809191
:106D60009109909192090E945AA788E00E94292BCC
:106D7000E091210DF091220D8085EAD88091910952
:106D8000909192090C9471A6CF92DF92EF92FF92AC
:106D90000F931F93CF93DF930E944C51C82E65E74A
:106DA00079E080919109909192090E9474A60E94C5
:106DB000FB2AC7EADCE000E010E0D12C78012FEFDD
:106DC000E21AF20A4AE050E0B701809191099091ED
:106DD00092090E9438A70930110514F48BE001C014
:106DE0008AE00E94292B2881809191099091920933
:106DF000222391F1ED81FE81618172814AE050E0B0
:106E00000E9438A7ED81FE8181819281883E934066
:106E100014F40E94212B84E00E94292BED81FE8135
:106E2000638174814AE050E08091910990919209C8
:106E30000E9438A784E00E94292BED81FE812781E2
:106E40008091910990919209222319F06DE679E0E1
:106E50000BC066E679E008C00C151D051CF46EE554
:106E600079E002C061E579E00E9474A627968CE083
:106E7000E816F10411F08701A1CFDF91CF911F91A6
:106E80000F91FF90EF90DF90CF900C94FB2A6DE371
:106E900079E080919109909192090E9438A60E9410
:106EA0004C514AE050E0682F8091910990919209ED
:106EB0000E9460A769E279E080919109909192091E
:106EC0000E9438A66091250D7091260D4AE050E091
:106ED00080919109909192090C943FA7B8DD54DFFD
:106EE000D6CF80919109909192090E9471A60E943B
:106EF000FB2A6DE179E080919109909192090E94BD
:106F000074A60E94FB2A69E079E080919109909132
:106F100092090E9438A6809177110E94955ABC016F
:106F200080919109909192090E9474A665EF78E092
:106F300080919109909192090E9438A680917811D0
:106F40000E94955ABC0180919109909192090E94EA
:106F500038A62091781180919109909192092B3057
:106F60003CF4293054F4283069F464EE78E007C02A
:106F70002B3041F460EF78E002C06AEE78E00E94C6
:106F800074A602C00E9471A660ED78E0809191091C
:106F9000909192090E9438A6809179110E94955A89
:106FA000BC0180919109909192090E9438A620918C
:106FB000791180919109909192092B303CF42930FC
:106FC00054F4283069F46FEB78E007C02B3041F4BB
:106FD0006BEC78E002C065EC78E00E9474A602C019
:106FE0000E9471A66BEA78E08091910990919209D4
:106FF0000E9438A620918111809191099091920967
:10700000222319F063EA78E002C061E978E00E9487
:1070100038A680919109909192090C9471A61F93C2
:10702000CF93DF9380911702823009F470C21091E0
:107030009811D0919B11C1E0809191099091920992
:107040000E9471A60E94FB2A62E878E08091910973
:10705000909192090E9474A60E94FB2A69E678E04A
:1070600080919109909192090E9438A68091AE1169
:107070000E94E764BC0180919109909192090E945D
:1070800074A660E578E080919109909192090E9440
:1070900038A64AE050E060911702809191099091E2
:1070A00092090E9460A767E378E08091910990912E
:1070B00092090E9438A6812F69DB112309F44EC082
:1070C0006DE278E080919109909192090E9438A632
:1070D00080919109909192094AE050E0CC2339F0D7
:1070E000609199110E945AA71091991106C0609160
:1070F0009F110E945AA710919F110E947A65181340
:107100000CC261E178E080919109909192090E940E
:1071100038A68091910990919209CC2339F0609121
:107120009A1161110CC06CE078E006C06091A0116A
:10713000611105C067E078E00E9438A607C0772794
:1071400067FD70954AE050E00E9438A765E078E05E
:1071500080919109909192090E9438A6809191099D
:10716000909192090E9471A66CEE77E0809191094E
:10717000909192090E9438A68D2F08DBDD2309F437
:107180004EC062EE77E080919109909192090E9441
:1071900038A680919109909192094AE050E0CC2361
:1071A00039F060919C110E945AA7D0919C1106C0A1
:1071B0006091A2110E945AA7D091A2110E947D65F0
:1071C000D813C7C166EC77E080919109909192093C
:1071D0000E9438A68091910990919209CC2339F0B0
:1071E00060919D1161110CC061EC77E006C0609167
:1071F000A311611105C06CEB77E00E9438A607C0AF
:10720000772767FD70954AE050E00E9438A76AEB47
:1072100077E080919109909192090E9438A680911F
:107220009109909192090E9471A661EA77E080919C
:107230009109909192090E9438A68091B71181110D
:1072400002C0B2DA36C068E37AE080919109909189
:1072500092090E9438A66EE977E080919109909199
:1072600092090E9438A64AE050E06091B7118091DF
:107270009109909192090E945AA76EE877E0809157
:107280009109909192090E9438A66091B81170916D
:10729000B9114AE050E080919109909192090E94C1
:1072A00075A769E877E080919109909192090E9411
:1072B00074A660E777E080919109909192090E940D
:1072C00038A68091AF118436D8F469E677E08091D2
:1072D0009109909192090E9438A64AE050E060918D
:1072E000AF1180919109909192090E945AA767E687
:1072F00077E080919109909192090E9474A602C052
:1073000080E052DA6EE477E08091910990919209E1
:107310000E9438A68091B0118436D8F467E477E0F3
:1073200080919109909192090E9438A64AE050E01C
:107330006091B01180919109909192090E945AA791
:1073400065E477E080919109909192090E9474A67A
:1073500002C080E029DA6CE277E080919109909197
:1073600092090E9438A66091A5117091A6118827F4
:1073700077FD8095982F0E9433AC20E030E04AE7FB
:1073800054E40E9498ABAB01BC0121E030E0809155
:107390009109909192090E9468A867E277E0809134
:1073A0009109909192090E9474A66EE077E0809115
:1073B0009109909192090E9438A66091A71170914D
:1073C000A811882777FD8095982F0E9433AC20E084
:1073D00030E04AE754E40E9498ABAB01BC0121E0E5
:1073E00030E080919109909192090E9468A869E02B
:1073F00077E080919109909192090E9474A660EFC4
:1074000076E080919109909192090E9438A660914E
:10741000A9117091AA11882777FD8095982F0E9455
:1074200033AC20E030E04AE754E40E9498ABAB0173
:10743000BC0121E030E080919109909192090E9475
:1074400068A86BEE76E080919109909192090E9474
:1074500074A662ED76E080919109909192090E9464
:1074600038A68091AE11813011F08430E1F4809122
:10747000AB118CD98091AB118823E9F06EEC76E0EA
:1074800080919109909192090E9438A64AE050E0BB
:107490006091AC1180919109909192090E945AA734
:1074A0006CEC76E002C067EB76E0809191099091F8
:1074B00092090E9438A680919109909192090E94A8
:1074C00071A66EE976E080919109909192090E94EF
:1074D00038A68091AE118150823070F40E94E56729
:1074E0004AE050E0682F8091910990919209DF91D4
:1074F000CF911F910C9460A769E876E08091910983
:1075000090919209DF91CF911F910C9474A61091E4
:107510009E11D091A111C0E08FCD6EE178E08091F5
:107520009109909192090E9438A60E947A654AE0DA
:1075300050E0682F80919109909192090E945AA77A
:107540006CE178E080919109909192090E9438A6AF
:10755000D8CD63ED77E080919109909192090E94D6
:1075600038A60E947D654AE050E0682F809191091D
:10757000909192090E945AA761ED77E0809191095C
:10758000909192090E9438A61DCE80919109909108
:1075900092090E9471A60E94FB2A69E776E0809119
:1075A0009109909192090E9474A60E94FB2A68E5B5
:1075B00076E080919109909192090E9438A680917D
:1075C00080118436D8F461E576E08091910990913C
:1075D00092090E9438A64AE050E0609180118091A3
:1075E0009109909192090E945AA76FE476E08091E8
:1075F0009109909192090E9474A602C080E0D4D8AB
:107600006EE276E080919109909192090E9438A6ED
:1076100080917F118436D8F467E276E080919109F9
:10762000909192090E9438A64AE050E060917F1143
:1076300080919109909192090E945AA765E276E0A3
:1076400080919109909192090E9474A602C080E0F5
:10765000ABD864E076E080919109909192090E9404
:1076600038A6609183117091841116161706F4F4F0
:10767000882777FD8095982F0E9433AC20E030E07A
:107680004AE754E40E9498ABAB01BC0122E030E031
:1076900080919109909192090E9469A86FEF75E01D
:1076A00080919109909192090C9474A680E07CC815
:1076B00080919109909192090E9471A60E94FB2AE3
:1076C00064EF75E080919109909192090E9474A6EF
:1076D0000E94FB2A67EE75E08091910990919209D2
:1076E0000E9438A68091C0110E94BD7CBC0180918F
:1076F0009109909192090C9474A669E475E08091C7
:107700009109909192090E9438A64AE050E0609158
:10771000BB1180919109909192090E945AA7909172
:10772000BB1180919E08981791F069E375E08091F4
:107730009109909192090E9438A64AE050E0609128
:107740009E0880919109909192090E945AA767E33F
:1077500075E080919109909192090C9438A69091CE
:1077600094098823F1F080919F088823D1F08091BB
:1077700079118D30B1F481E08093BA118093A00823
:10778000992309F16EE97FE0809191099091920926
:107790000E9438A6B2DF80919109909192090C94D1
:1077A00071A61092BA11992341F06DE77FE08091A4
:1077B0009109909192090E9474A68091BC11811147
:1077C00002C01092A00808959091BA1181E0892713
:1077D000C6CFFACF81E0C3CF80E0C1CF68E275E0C9
:1077E00080919109909192090E9438A64AE050E058
:1077F0006091BD1180919109909192090E945AA7C0
:107800009091BD1180919D08981791F068E175E005
:1078100080919109909192090E9438A64AE050E027
:1078200060919D0880919109909192090E945AA7B8
:1078300066E175E080919109909192090C9438A6C7
:10784000909194098823D1F080919F088823B1F00A
:1078500081E08093BC118093A008992309F165E62B
:107860007FE080919109909192090E9438A6B6DF3D
:1078700080919109909192090C9471A61092BC117B
:10788000992341F06CE47FE08091910990919209F5
:107890000E9474A68091BA11811102C01092A008B2
:1078A00008959091BC1181E08927CACFFACF81E079
:1078B000C7CF80E0C5CF80919109909192090E9435
:1078C00071A60E94FB2A6DEC75E080919109909160
:1078D00092090E9474A60E94FB2A20919F08809121
:1078E0009109909192092223B1F16BEA75E00E940F
:1078F00038A680919109909192090E9471A66CE836
:1079000075E080919109909192090E9438A680912A
:10791000BA110E94C6338091BA118111EEDE8091B6
:107920009109909192090E9471A66DE675E080918F
:107930009109909192090E9438A68091BC110E94F1
:10794000C6338091BC11811149DF809191099091DA
:1079500092090C9471A668E575E00C9474A6809168
:107960009109909192090E9471A60E94FB2A6AE0F7
:1079700075E080919109909192090E9474A60E94ED
:10798000FB2A20914C108091910990919209222319
:1079900009F475C167EF74E00E9438A60E94A685BD
:1079A0000E94D4330E94A6852091910930919209BA
:1079B000882389F064EE74E0C9010E9438A68091A2
:1079C0004F100E94FA72BC01809191099091920926
:1079D0000E9474A635C061ED74E0C9010E9438A60A
:1079E00080914C100E94FA72BC0180919109909193
:1079F00092090E9438A680914D108823D9F069EC35
:107A000074E080919109909192090E9438A680912A
:107A10004D100E945373BC0180919109909192097D
:107A20000E9438A667EC74E08091910990919209C8
:107A30000E9438A680919109909192090E9471A6A6
:107A400064EB74E080919109909192090E9438A6AC
:107A500080914E10882321F00E94FA72BC0102C06E
:107A600060EB74E080919109909192090E9474A654
:107A70006DE974E080919109909192090E9438A675
:107A800080914F10882321F00E94FA72BC0102C03D
:107A900069E974E080919109909192090E9474A61D
:107AA00066E874E080919109909192090E9438A64D
:107AB000809151108823E1F060E874E08091910991
:107AC000909192090E9438A6809150100E94FA72FB
:107AD000BC0180919109909192090E9438A661E3BE
:107AE00072E080919109909192090E9494A603C03E
:107AF00080E00E94D4336DE674E08091910990910A
:107B000092090E9438A6809152108823E1F067E61E
:107B100074E080919109909192090E9438A6809119
:107B200050100E94FA72BC018091910990919209C3
:107B30000E9438A661E372E08091910990919209C8
:107B40000E9494A603C080E00E94D43364E574E0F0
:107B500080919109909192090E9438A680915310CA
:107B60000E946585BC0180919109909192090E94C3
:107B700074A661E474E080919109909192090E9449
:107B800038A6809145100E943485BC0180919109EE
:107B9000909192090E9474A66FE374E0809191091C
:107BA000909192090E9438A64AE050E060914A10F4
:107BB00080919109909192090E945AA760E374E024
:107BC00080919109909192090E9438A68091451068
:107BD000811112C04AE050E060914B1080919109F0
:107BE000909192090E945AA765E274E080919109F0
:107BF000909192090E9438A66091461070914710AA
:107C0000882777FD8095982F0E9433AC20E030E0E4
:107C10004AE754E40E9498ABAB01BC0121E030E09C
:107C200080919109909192090E9468A867E174E09F
:107C300080919109909192090E9438A66091481014
:107C400070914910882777FD8095982F0E9433AC5A
:107C500020E030E04AE754E40E9498ABAB01BC015D
:107C600021E030E080919109909192090E9468A8EA
:107C700068E074E0809191099091920902C06CEEE5
:107C800073E00C9474A680919109909192090E94DE
:107C900071A60E94FB2A61EE73E080919109909198
:107CA00092090E9474A60E94FB2A6DEC73E08091F9
:107CB0009109909192090E9438A64091F411509137
:107CC000F5116091F6117091F7112AE030E0809182
:107CD0009109909192090E948EA769EB73E08091BF
:107CE0009109909192090E9438A64091FC115091FF
:107CF000FD116091FE117091FF112AE030E080913A
:107D00009109909192090E948EA765EA73E0809193
:107D10009109909192090E9438A64091F8115091D2
:107D2000F9116091FA117091FB112AE030E0809115
:107D30009109909192090E948EA761E973E0809168
:107D40009109909192090E9438A640910012509199
:107D5000011260910212709103122AE030E08091CA
:107D60009109909192090C948EA7609105127091DF
:107D7000061280E090E00E9431AC20E030E04AE75B
:107D800054E40E9498ABAB01BC0121E030E080914B
:107D90009109909192090C9468A880911602882309
:107DA00051F00E943813811143C01092160281E0F5
:107DB00080939B0808950E94431390919A0888230A
:107DC00001F191111EC081E080939A0810929B08E6
:107DD00080919409882389F069ED7EE08091910972
:107DE000909192090E9438A6C0DF66ED7EE08091F6
:107DF0009109909192090E9474A60E9492220C947B
:107E0000BA169923A9F00E944313811111C0109250
:107E10009A0881E080939B0880919409882341F01F
:107E20006AEB7EE080919109909192090C9474A67E
:107E3000089580919109909192090E9471A60E94E3
:107E4000FB2A69E873E080919109909192090E9460
:107E500074A60E94FB2A66E773E0809191099091D5
:107E600092090E9438A60E943813209191093091FE
:107E70009209882321F063E773E0C9011FC06FE610
:107E800073E0C9010E9474A66CE573E080919109CA
:107E9000909192090E9438A60E94CF12AB01BC01BA
:107EA00022E030E080919109909192090E9468A8A7
:107EB0006AE573E080919109909192090E9474A6FD
:107EC00067E473E080919109909192090E9438A62D
:107ED000809104120E94C63320910412809191096E
:107EE00090919209222369F064E473E00E9438A61D
:107EF0003CDF6AE373E080919109909192090C94C0
:107F000074A60C9471A6FF920F931F93CF93DF93E7
:107F1000CDB7DEB7E6970FB6F894DEBF0FBECDBF84
:107F20002FE538E641E055272BAB3CAB4DAB5EABC4
:107F300080919109909192090E9471A60E94FB2A5A
:107F400068E273E080919109909192090E9474A671
:107F50000E94FB2A6FE073E0809191099091920951
:107F60000E9438A62091240D809191099091920948
:107F7000222319F06BE073E002C066E073E00E9418
:107F800074A68091240D882351F16DEE72E08091EA
:107F90009109909192090E9438A66091BE1170914A
:107FA000BF11882777FD8095982F0E9433AC20E081
:107FB00030E04AE754E40E9498ABAB01BC0122E0F8
:107FC00030E080919109909192090E9468A868EE32
:107FD00072E080919109909192090E9474A601E04B
:107FE00011E189E2F82ED8018C91882309F466C04A
:107FF000F8013297608171816115710509F45EC0E5
:108000000E943F2B63EE72E080919109909192095A
:108010000E9438A668ED72E08091910990919209D2
:108020000E9438A6F801608170E04AE050E080913B
:108030009109909192090E9438A7D8018C918A30B9
:1080400010F40E94212B0E94192BF8018081F89EC8
:10805000C0011124AA2797FDA095BA2F2BA93CA9EE
:108060004DA95EA9820F931FA41FB51F9E012F5F0C
:108070003F4FAC01BD014F5F5F4F6F4F7F4FABBFB5
:10808000FC018791D9018D939D01882319F0DB01B3
:10809000CA01EFCFBE016F5F7F4F80919109909130
:1080A00092090E9494A68091910990919209DC0115
:1080B000ED91FC910284F385E02D19950D5F1F4F22
:1080C000B1E109371B0709F08ECFE6960FB6F89499
:1080D000DEBF0FBECDBFDF91CF911F910F91FF90FB
:1080E00008950E94F5340E94032280919109909195
:1080F0009209DC01ED91FC910284F385E02D199544
:108100000E946E370E9403228091910990919209FA
:10811000DC01ED91FC910284F385E02D19950E941C
:1081200071370E9403228091910990919209DC019C
:10813000ED91FC910284F385E02D19950E940F3892
:108140000E9403228091910990919209DC01ED91A6
:10815000FC910284F385E02D199517DA0E94032221
:108160008091910990919209DC01ED91FC9102843A
:10817000F385E02D1995F3DB0E940322809191098C
:1081800090919209DC01ED91FC910284F385E02D40
:1081900019958EDA0E94032280919109909192099B
:1081A000DC01ED91FC910284F385E02D199583DBD0
:1081B0000E9403228091910990919209DC01ED9136
:1081C000FC910284F385E02D19959DDE0E94032227
:1081D0008091910990919209DC01ED91FC910284CA
:1081E000F385E02D199525DE0E94032280919109E7
:1081F00090919209DC01ED91FC910284F385E02DD0
:10820000199541DD0E940322809191099091920974
:10821000DC01ED91FC910284F385E02D19958091AC
:108220009109909192090E9471A60C94FB2A4F9299
:108230005F926F927F929F92AF92BF92CF92DF92A6
:10824000EF92FF920F931F93CF93DF9380917B0860
:1082500081110DC0E091030DF091040D8181928197
:1082600090936A088093690881E080937B088091ED
:10827000730881110DC0E091030DF091040D83810D
:108280009481909368088093670881E080937308D5
:108290000E941A9F60936308709364088093650836
:1082A0009093660880911502882309F4DCC06091E0
:1082B000AC1170E080E090E00E9431AC20E030E052
:1082C00048EC52E40E9498AB20E030E04FE753E4E2
:1082D0000E94E7AC0E9400AC709362086093610852
:1082E0006091B11170E080E090E00E9431AC20E03C
:1082F00030E048EC52E40E9498AB20E030E04FE7D9
:1083000053E40E94E7AC0E9400AC70936008609355
:108310005F086091AF116436C0F470E080E090E0D7
:108320000E9431AC20E030E048EC52E40E9498AB6F
:1083300020E030E04FE753E40E94E7AC0E9400AC3D
:1083400070935E0860935D0806C08FEF90E0909395
:108350005E0880935D086091B0116436C0F470E0EF
:1083600080E090E00E9431AC20E030E048EC52E444
:108370000E9498AB20E030E04FE753EC0E94E7AC5E
:108380000E9400AC70935C0860935B0806C081E0BB
:108390009FEF90935C0880935B086091B711611127
:1083A00003C010925A0818C081E080935A0870E008
:1083B00080E090E00E9431AC20E030E048EC52E4F4
:1083C0000E9498AB20E030E04FE753E40E94E7AC16
:1083D0000E9405AC609359086091D01170E080E074
:1083E00090E00E9431AC20E030E048EC52E40E9482
:1083F00098AB20E030E04FE753E40E94E7AC0E94E6
:1084000005AC6093580880910412882319F00E94EB
:10841000C01205C010929A0881E080939B08809159
:108420009309882351F021E730E44CED55E060E0FA
:1084300070E085E999E00E946D630E941A9F609345
:10844000630870936408809365089093660860934E
:1084500054087093550880935608909357081092CB
:1084600015020E9480150E940322809153088823E0
:1084700021F0813009F446C04CC083E898E00E94A6
:10848000CF8F882321F00E948B2A2BDE42C048E048
:1084900057E060E070E083E898E00E94D98F88237D
:1084A000C1F10E94D510813029F0843081F583E03C
:1084B00090E025C0809179118C50823018F484E0CE
:1084C00090E01DC080919409882341F061E672E13B
:1084D00080919109909192090E9474A66AE070E0DF
:1084E00080E090E00E94499F83E898E00E945F8FBF
:1084F00083E898E00E94CF8F882381F308C00E9410
:10850000AF2F05C083E898E00E94CF8F81111092B1
:1085100053080E94D594882321F00E9492220E9441
:108520004E9D0E947C538091230D882389F00E94E8
:10853000FE220EC00E947C530E94D594882331F005
:108540000E942B160E944E9D0E94F1150E9403224C
:108550008091230D8111EECF0E9481210E94B712DC
:1085600080919B08882309F46DC0809114028823B0
:1085700009F468C0809179118F3081F18091100DDC
:10858000882361F18091120D811128C08091140916
:1085900090911509DC01ED91FC916091150D7091A0
:1085A000160D0190F081E02D19958091D31188234B
:1085B000A9F02091150D3091160D8091230990910D
:1085C0002409DC01ED91FC91232B21F402A0F3A1FD
:1085D000E02D03C000A0F1A1E02D19958091781144
:1085E0008F3081F180911A0D882361F180911C0DEB
:1085F000811128C08091160990911709DC01ED9135
:10860000FC9160911F0D7091200D0190F081E02D83
:1086100019958091D2118823A9F020911F0D3091D6
:10862000200D8091230990912409DC01ED91FC91AA
:10863000232B21F4048CF58DE02D03C0028CF38DE7
:10864000E02D19950E947569882309F4FEC7809171
:108650009B08882309F4F9C78091FC0C811105C09F
:108660008091060D882309F4EEC08091010D909150
:10867000020D909352088093510890935008809374
:108680004F0880910B0D90910C0D90934E088093A4
:108690004D0880914C08811103C081E080934C0803
:1086A0000E94066A81113CC08091130280931202DD
:1086B000823019F0833071F01BC080914F08909187
:1086C000500897FD05C01092500810924F0834C012
:1086D00083E007C080914F089091500897FDF3CF39
:1086E00082E080931202109252081092510824C026
:1086F0001092500810924F0810924E0810924D0898
:1087000081E08093120210924B0810924A08109256
:1087100049081092480810924708109246080CC069
:1087200060914D0870914E0880914F0890915008CB
:108730000E946B6780931202609112028091130273
:10874000681709F473C0813041F0843009F059C0D2
:108750001092500810924F086DC0909145089F5F8D
:1087600090934508933018F48093120263C02091CF
:10877000A5113091A611232B21F18091440881117C
:1087800022C00E941A9F4090540850905508609053
:108790005608709057086419750986099709409022
:1087A000A5115090A611612C712C641575058605D4
:1087B000970530F49091110280911202981303C032
:1087C00081E08093440880914408882399F1809146
:1087D00012028093130280915A08882359F181E094
:1087E000809343088093E2084091B8115091B911E9
:1087F00060E070E02AEE3BE085E999E00E946D635D
:1088000019C00E947E6780934208882399F0809166
:10881000A5119091A611892B69F48091950E811173
:1088200009C08091960E811105C078C71092420848
:108830001092450880914208882319F00E94D313B2
:1088400002C00E94DA138091AE1160914D087091C0
:108850004E08813009F045C080911302843009F040
:108860004FC0409161085091620885E299E00E94F2
:108870008B679093470880934608209143082223F2
:10888000A9F01816190624F42091590830E008C000
:10889000009751F02091590830E031952195310928
:1088A0003093410820934008109243082091E20839
:1088B000222351F1181619063CF42091590830E092
:1088C00082179307C4F40BC00097F1F02091590868
:1088D00030E03195219531092817390764F4C90131
:1088E0000AC0823069F440915F085091600885E2C7
:1088F00099E00E948B67909347088093460804C0D4
:10890000709347086093460820911302243009F4BD
:10891000ADC0213009F4AAC040904F0850905008D3
:108920002230F9F48091AF11843608F049C0B201C9
:10893000882777FD8095982F20915D0830915E08FB
:108940008901222717FD2095322F3F932F931F93E4
:108950000F93A12CB12C6501E12CF12C8701EA9435
:1089600021C0233069F58091B011843648F5B201F9
:10897000882777FD8095982F20915B0830915C08BF
:108980008901222717FD2095322F3F932F931F93A4
:108990000F93A12CB12C6501EE24E394FF24FA94EB
:1089A0000FEF1FEF20E030E0A9010E94BDA87093F7
:1089B0004B0860934A080F900F900F900F9004C0DF
:1089C00050924B0840924A08809143088823B1F0A6
:1089D00080911302823021F48091590890E008C000
:1089E000833051F48091590890E0919581959109D7
:1089F00090933F0880933E08109243088091E208CC
:108A00008823F9F02091130280914A0890914B0835
:108A1000223039F42091590830E0281739076CF4D6
:108A20000BC0233071F42091590830E03195219525
:108A30003109821793070CF49C0130934B08209363
:108A40004A0840913E0850913F0860914A08709151
:108A50004B08009142082091130285E299E00E94A0
:108A6000DE6590934B0880934A0816C010924B081D
:108A700010924A0840914008509141086091460880
:108A8000709147080091420885E299E00E94DE65F6
:108A9000909347088093460880911302843069F4CC
:108AA00060914D0870914E0840913C0850913D08EE
:108AB000E090420804E09B0118C00E94066A2091E1
:108AC0004A0830914B08882321F02115310509F41B
:108AD0002CC640913C0850913D086091510870911E
:108AE0005208E09042080091130285E299E00E944A
:108AF000EE66909349088093480860914808709109
:108B0000490880913C0890913D086817790789F0E1
:108B10008091230990912409DC01ED91FC9106805C
:108B2000F781E02D199580914808909149080E949D
:108B3000F42380911302843029F480914D089091A0
:108B40004E0804C080914A0890914B08892B09F087
:108B500062C081E08093130280911002813009F499
:108B600045C080931102109244080E941A9F60939E
:108B70005408709355088093560890935708809135
:108B8000AE118230C1F01CF48130A9F02FC08330C7
:108B900011F1843059F580911C0990911D09DC0177
:108BA000ED91FC910480F581E02D199580911809D3
:108BB0009091190914C08091200990912109DC013C
:108BC000ED91FC910480F581E02D199580911E09AD
:108BD00090911F0904C080911C0990911D09DC012E
:108BE000ED91FC910480F581E02D19958091230988
:108BF00090912409DC01ED91FC91EC5BFF4F019019
:108C0000F081E02D199580910912882309F4F0C0B4
:108C10000E94D313EDC08091AE11833009F45AC085
:108C20001CF481302CF492C0843009F463C08EC0EF
:108C3000409146085091470860914A0870914B084E
:108C400008E318E02AE338E085E299E00E94EE6745
:108C500060913A0870913B088091360890913708EE
:108C60008617970761F42091340830913508809178
:108C70003808909139082817390709F467C080919E
:108C8000200990912109DC01ED91FC910190F08186
:108C9000E02D199580911E0990911F09DC01ED913D
:108CA000FC9160913808709139080190F081E02DB5
:108CB000199580913A0890913B08909337088093DA
:108CC0003608809138089091390890933508809340
:108CD00034083CC060914A0870914B0880913E086E
:108CE00090913F088617970789F180911C09909110
:108CF0001D0925C060914A0870914B0880913E087B
:108D000090913F088617970759F080911C09909120
:108D10001D09DC01ED91FC910190F081E02D199588
:108D200060914D0870914E088091320890913308FF
:108D30008617970759F08091180990911909DC015D
:108D4000ED91FC910190F081E02D1995809123091E
:108D500090912409DC01ED91FC91EA5BFF4F0190B9
:108D6000F081E02D1995A0912309B091240981117A
:108D700019C080914A0890914B0897FF03C09195C4
:108D8000819591092091580830E08217930754F09B
:108D9000ED91FC911197EE5BFF4F0190F081E02D7A
:108DA000CD01DCC4ED91FC911197EA5BFF4F01907E
:108DB000F081E02DCD011995882381F080914A083A
:108DC00090914B0897FF03C091958195910920914F
:108DD000580830E0281739070CF0B4C48091091204
:108DE0008111A8C480911302813011F00E94651195
:108DF00080919B088823A1F08091AE11825082302F
:108E000078F480911A0990911B09DC01ED91FC9195
:108E100060910B0D70910C0D0190F081E02D199572
:108E200080911402882309F401C180919B08882352
:108E300009F4FCC0912C80913C09981608F0E6C01A
:108E40008091240D8823F9F08091A60C8823D9F015
:108E5000E92DF0E0CF01880F991FE80FF91FE150CD
:108E6000FF4E408151812091A40C3091A50C4217F6
:108E7000530749F4FC01E35CF64F0190F081E02DCB
:108E800080E090E01995C8EADCE03BEA432E3CE044
:108E9000532E08EE13E0612C712CA92CB12CC501C6
:108EA000880F991FA80EB91EF501E150FF4E5F0112
:108EB0009C01235C364F7901EC81FD8187818823F9
:108EC000D9F088818823C1F08085D801EAE08E9F9F
:108ED000A00DB11D1124CD01D2012C91820F911D45
:108EE000F501208131812817390731F4D701ED913F
:108EF000FC9180E090E01995EC81FD8187818111E2
:108F000011C08881882371F0F501808191818017DB
:108F1000910741F4D701CD90DC90C3010E94B229A2
:108F2000F6011995FFEF6F1A7F0A279608511C4F1B
:108F300027E0420E511C3CE06316710409F0BCCFDF
:108F4000F3E3CF2EF9E0DF2EA4E3EA2EA9E0FA2E18
:108F50000FE219E0C1E3D9E0B4E64B2E512C692CA5
:108F6000712CC301880F991F680E791ED301A1507F
:108F7000BF4E3D01FC01E35CF64F5F01D6018C91D1
:108F8000811118C0F70180818823A1F0888188238E
:108F900089F0D8018D919C91840D951DF30120815C
:108FA00031812817390731F4D501ED91FC9180E02A
:108FB00090E01995F6018081811114C0D7018C9140
:108FC000811110C08881882369F0F301808191812B
:108FD0008415950539F4D501ED91FC91D8018D9159
:108FE0009C911995B7E0CB0ED11CE7E0EE0EF11C79
:108FF000095F1F4FF4E64F0E511C27962CE24216D4
:1090000021E0520609F0BACF939415CF8091B211A6
:10901000882361F00E947569811108C08091010D5B
:109020009091020D8F3791050CF09AC380919B08A7
:10903000882309F439C180911402882309F434C1CA
:109040000E94DA8CC82F882309F42EC18230E1F106
:10905000833009F46BC0813009F094C08091940989
:10906000882309F45CC063E572E1809191099091D5
:1090700092090E9438A60E948F870E94FA72BC0152
:1090800080919109909192090E9438A60E9492873E
:10909000882359F00E9492870E945373BC018091EB
:1090A0009109909192090E9438A661E572E1809140
:1090B0009109909192090E9474A680919508882345
:1090C00071F166E372E125C080919409882339F13A
:1090D00063E272E180919109909192090E9438A611
:1090E0000E948F870E94FA72BC0180919109909131
:1090F00092090E9438A661E272E1809191099091F3
:1091000092090E9474A680919508882341F066E038
:1091100072E180919109909192090E9474A68091C8
:109120009508882379F1109295082CC080919508B4
:10913000811128C00E949587882321F181E08093C6
:109140009508809194098823D9F06DEE71E18091A2
:109150009109909192090E9438A60E948F870E94DF
:10916000FA72BC0180919109909192090E9438A6EF
:109170006BEE71E180919109909192090E9474A621
:109180000E948B238091AE119FEF980F9230C0F414
:1091900000910E0910910F092091140930911509C1
:1091A000409116095091170960911E0970911F098D
:1091B000C82EE0908F1180912009909121092FC035
:1091C000833099F400910E0910910F092091140930
:1091D00030911509409116095091170960911A09AB
:1091E00070911B09E3E0CE2E14C08430D1F40091BD
:1091F0000E0910910F092091140930911509409121
:10920000160950911709609118097091190994E095
:10921000C92EE0908F1180911C0990911D090E9428
:10922000F187109237081092360810923508109284
:109230003408809194098823E9F0C330D9F06CEDAB
:1092400071E180919109909192090E9438A60E9443
:1092500098874AE050E0682F809191099091920997
:109260000E945AA76AED71E180919109909192094B
:109270000E9474A68091ED0F8823B1F080911402B2
:10928000882391F080919409882341F06BEC71E17F
:1092900080919109909192090E9474A610921402F3
:1092A0000E9492220E941924809195088823D1F16E
:1092B0000E949587811136C080919409882319F105
:1092C00063EB71E180919109909192090E9474A6DB
:1092D00064EA71E180919109909192090E9438A607
:1092E0000E9498874AE050E0682F80919109909100
:1092F00092090E945AA762EA71E1809191099091C6
:1093000092090E9474A61092950880912309909169
:109310002409DC01ED91FC910484F585E02D19957B
:109320000E9440238091140281115CC08091ED0F56
:10933000811158C080919B08882309F453C081E0B3
:10934000809314028091AE1181508230A8F48091F4
:109350002009909121090E945E0F80911E09909131
:109360001F090E945E0F8091AE118230F9F4809146
:109370001A0990911B0918C080911C0990911D0930
:109380000E945E0F8091AE11833031F480911A09F2
:1093900090911B090E945E0F8091AE11843031F4D0
:1093A00080911809909119090E945E0F8091160909
:1093B000909117090E945E0F8091140990911509F0
:1093C0000E945E0F0E940A240E945C2380919409EF
:1093D000882341F064E971E18091910990919209AB
:1093E0000E9474A680919B08882309F4EAC08091AA
:1093F0004208882329F00E947C150E94841504C02D
:109400000E9480150E94881580919409882381F01C
:1094100080914208882361F080913108811108C051
:109420006CE871E180919109909192090E9474A673
:1094300080911302823051F024F4813009F48BC002
:10944000A4C08330D1F0843079F19FC0809142086C
:1094500081119BC00E9480150E94841580919409FF
:10946000882309F492C090911302809110029817FA
:1094700009F48BC06DE771E182C0809142088111CF
:1094800084C00E947C150E948815809194098823CD
:1094900009F47BC09091130280911002981709F48F
:1094A00074C06EE671E16BC08091460890914708E8
:1094B000181619061CF580912F0890913008009716
:1094C00031F00E940A221092300810922F080E9458
:1094D000801580912D0890912E08892B89F523ED18
:1094E00035E140E951E060E070E085E999E00E94F3
:1094F000656390932E0880932D0822C080912D08DB
:1095000090912E08009731F00E940A2210922E08A6
:1095100010922D080E94881580912F089091300894
:10952000892B71F42EEA35E140E951E060E070E00A
:1095300085E999E00E9465639093300880932F0835
:1095400080919409882309F1809110028430E9F018
:1095500061E671E114C080914208811116C00E9439
:1095600080150E94881580919409882371F090914C
:10957000130280911002981741F069E571E1809122
:109580009109909192090E9474A6809113028430EF
:10959000C1F080912D0890912E08009731F00E9423
:1095A0000A2210922E0810922D0880912F08909177
:1095B0003008009731F00E940A2210923008109271
:1095C0002F088091120280930F02809113028093E2
:1095D000100280914A0890914B0890933F08809325
:1095E0003E088091460890914708909341088093E7
:1095F00040088091420880933108809151089091F1
:10960000520890932C0880932B08809148089091E1
:10961000490890933D0880933C0880914D089091B3
:109620004E089093330880933208DF91CF911F91B9
:109630000F91FF90EF90DF90CF90BF90AF909F90F1
:109640007F906F905F904F90089580914C08882391
:1096500009F4CECB10924B0810924A081092490898
:1096600010924808109247081092460810923B0842
:1096700010923A0810923908109238088091AE1171
:109680008230C1F01CF48130A9F02FC0833011F179
:10969000843059F580911C0990911D09DC01ED91F0
:1096A000FC910480F581E02D199580911809909125
:1096B000190914C08091200990912109DC01ED91D4
:1096C000FC910480F581E02D199580911E099091FF
:1096D0001F0904C080911C0990911D09DC01ED91C6
:1096E000FC910480F581E02D199581E080931302AF
:1096F000109242080E94DA1310924C0880912309BC
:1097000090912409DC01ED91FC91EC5BFF4F0190FD
:10971000F081E02D19950E944E116ACB10924208FB
:10972000809112028093130285C810925208109201
:109730005108CFC980912D09882309F453CB0E9489
:10974000DA1350CB8091230990912409DC01ED912B
:10975000FC91EC5BFF4F0190F081E02D19953ECB21
:109760000E945C2363CC0C947140EF92FF920F93A4
:109770001F9383ED9BE00E94F58F85E999E00E949D
:10978000946280E999E09DD186E299E00E94FC5FB5
:1097900085E299E00E94186582E299E00E948A853C
:1097A00028E24FEF5FEFBA0181EA98E00E949D9DA9
:1097B0008CE998E00E94B89419E1E12EF12C00E0C8
:1097C00010E021E041E064E483E898E00E94278F04
:1097D0001F910F91FF90EF900895089580E090E021
:1097E000FC01EE0FFF1FE452F44F1182108201962C
:1097F00088309105A9F71092ED0B1092EC0B0895AB
:10980000CF93DF93EC0162E083E00E9420A11092ED
:10981000DB0B1092D90B1092D80B1092D40BCE0107
:10982000DDDFEAE6F0E080818C608083ED9A2FB77F
:10983000F89480918400909185009093D60B80934A
:10984000D50B2FBFDF91CF910895ED98E59A109237
:10985000DB0B1092D70B1092D90B1092D80B1092F1
:10986000D40BBCCF80918400909185002091D50BC2
:109870003091D60B821B930B209184003091850090
:109880003093D60B2093D50B803727E1920770F1E8
:109890009093DD0B8093DC0B8091D80B9091D90BCA
:1098A000029751F49091DB0B8091D70B98133CC039
:1098B00081E08093D40B3EC08091D80B9091D90B5E
:1098C000892B49F481E090E09093D90B8093D80BD9
:1098D0001092DA0B2FC08091D80B9091D90B019781
:1098E00061F58091DB0B8430D8F527C02091DB0B2C
:1098F000283008F047C09C012C5D3540293B3B4097
:1099000068F4E091DB0BEF5FE093DB0BF0E0EE0F30
:10991000FF1FE452F44F9183808308958091D80B08
:109920009091D90B029771F583E090E09093D90B59
:109930008093D80B1092DB0B08958091D80B9091F7
:10994000D90B0397B9F79091DB0B8091D70B981344
:10995000F1CF8091D70B843068F382E090E0E6CFBE
:109960008091DA0B8F5F8093DA0B863018F382E0F8
:1099700090E09093D90B8093D80B8091DB0B809370
:10998000D70BD8CF08951F920F920FB60F921124C4
:109990000BB60F922F933F934F935F936F937F93E9
:1099A0008F939F93AF93BF93EF93FF935BDFFF91F1
:1099B000EF91BF91AF919F918F917F916F915F9147
:1099C0004F913F912F910F900BBE0F900FBE0F90B4
:1099D0001F9018958091D80B9091D90B0895809184
:1099E000D70B0895BFB7F894A0E08A2F90E08417B2
:1099F000950794F4FC01EE0FFF1FE252F44F208113
:109A00003181FC01EE0FFF1FE60FF71F36952795FA
:109A100031832083AF5FE9CFBFBF1092D40B08958D
:109A200081E080939D0C089581E080939C0C0895C3
:109A300081E080939B0C08951092120D089510926E
:109A40001C0D0895853208F080E089508C3148F46F
:109A5000E82FF0E0EE0FFF1FED5BFC4F808191815E
:109A6000089581E493E10895CF93DF93CDB7DEB7F6
:109A700028970FB6F894DEBF0FBECDBF84300CF030
:109A800080E027EC32E13A83298323EC32E13C8306
:109A90002B832EEB32E13E832D8329EB32E1388795
:109AA0002F83E82FEE0FFF0BEC0FFD1F81819281BA
:109AB00028960FB6F894DEBF0FBECDBFDF91CF91D1
:109AC000089510929A0C1092270D1092260D109264
:109AD000250D1092970C1092240D1092230D1092C8
:109AE0009D0C10929C0C10929B0C08959093990CD5
:109AF0008093980C08951F93CF93DF938091F20B7E
:109B00001091190281115BC0123021F11330A9F1BB
:109B1000113009F087C080919D0C811183C081E0D4
:109B200090E00E942CABEC0158DED093A30CC093C4
:109B3000A20CCE0165DE20E13DE44AEF50E060E09A
:109B400070E08091980C9091990C0E946D63109335
:109B5000F20B68C080919C0C811164C081E090E0A0
:109B60000E942CABEC01C7D6D093A10CC093A00CE3
:109B7000CE01C2D624E13DE414C080919B0C81113A
:109B800051C081E090E00E942CABEC010E94F055A6
:109B9000D0939F0CC0939E0CCE010E94F15528E1FA
:109BA0003DE44AEF50E060E070E08091980C9091C5
:109BB000990C0E946D6381E08093F20B33C01230E8
:109BC00071F01330D9F0113069F580919D0C81113D
:109BD00029C08091A20C9091A30CFCDE1FC0809143
:109BE0009C0C81111FC08091A00C9091A10C28D7D2
:109BF0008091A00C9091A10CE4D710C080919B0C97
:109C0000811110C080919E0C90919F0C0E944B5628
:109C100080919E0C90919F0C0E943F57029711F4E7
:109C200010939A0C809119028230D9F0833071F12F
:109C3000813009F041C080919D0C882309F43CC01B
:109C40008091A20C9091A30C00DE8091A20C9091C7
:109C5000A30C0E942DAB1092F20B10929C0C82E090
:109C600029C080919C0C882339F18091A00C90919F
:109C7000A10C89D68091A00C9091A10C0E942DABD3
:109C80001092F20B10929B0C83E014C080919B0CFD
:109C9000882391F080919E0C90919F0CEBD780913E
:109CA0009E0C90919F0C0E942DAB1092F20B109283
:109CB0009D0C81E0809319028091980C9091990CF1
:109CC000DF91CF911F910C94D963E091170DF09122
:109CD000180D8181928183969283818383819481FF
:109CE000839794838383E091210DF091220D8181EC
:109CF00092818396928381838381948183979483D5
:109D0000838308956091F30B7091F40B8091980C0C
:109D10009091990C0E94D564811110C020EF32E51A
:109D20004CE251E060E070E08091980C9091990CC9
:109D30000E946D639093F40B8093F30B08956091F0
:109D4000F30B7091F40B8091980C9091990C0E94F8
:109D5000D564882351F06091F30B7091F40B8091DE
:109D6000980C9091990C0C94B864CCCFEF92FF9220
:109D70000F931F93CF93DF93CDB7DEB7EDB6FEB64B
:109D80004091250D5091260DCA01880F991F2DB7BE
:109D90003EB7281B390B0FB6F8943EBF0FBE2DBF40
:109DA0000DB71EB70F5F1F4F80919A0C823079F06C
:109DB0008330A1F0813009F04CC0B8018091A20C31
:109DC0009091A30C0FDE40E05AE061E01CC0B801A6
:109DD0008091A00C9091A10CDAD6F5CFB8018091BA
:109DE0009E0C90919F0C0E942557EDCF589FF0013B
:109DF000599FF00D1124E950F44FA085B1858C9145
:109E000081110BC04F5F842F90E02091250D309180
:109E1000260D8217930754F31CC0A081B1818C9149
:109E2000D801A80FB11DA80FB11D12978D919C915B
:109E3000A281B3812D913C9111970480F581E02D91
:109E40002817390711F41082DDCF60838D939C931E
:109E5000D9CF0FB6F894FEBE0FBEEDBEDF91CF9105
:109E60001F910F91FF90EF9008956F927F928F92C4
:109E70009F92AF92BF92CF92DF92EF92FF920F9399
:109E80001F93CF93DF93CDB7DEB72D970FB6F8941E
:109E9000DEBF0FBECDBF4C01762E5A01622ECDB66D
:109EA000DEB68091970C2DB73EB792E0899F2019BE
:109EB000310911240FB6F8943EBF0FBE2DBFEDB788
:109EC000FEB731967F0161E078E0CE0107960E94EF
:109ED0006AA9F501108280919A0C823081F083305A
:109EE000C1F0813009F060C04091970C50E0B7019B
:109EF0008091A20C9091A30C75DD00E013C04091FD
:109F0000970C50E0B7018091A00C9091A10C3FD626
:109F100009C04091970C50E0B70180919E0C909140
:109F20009F0C93D76DE270E0CE0107960E9431A995
:109F30002091970C293038F0002321F0013029F0CE
:109F400020E004C028E010E001C018E0121700F57E
:109F5000F701E10FF11DE10FF11D608171814AE010
:109F6000CE0101962D870E9406AABE016F5F7F4F2A
:109F7000CE0107960E94DAAACE0101960E9403A99B
:109F8000662DCE0107960E94E0AA1F5F2D85DECFC9
:109F9000472D50E020E030E0B401CE0107960E944A
:109FA000F3AA8B85F5018083CE0107960E9403A951
:109FB0000FB6F894DEBE0FBECDBE0FB6F894DEBE6F
:109FC0000FBECDBE2D960FB6F894DEBF0FBECDBF2F
:109FD000DF91CF911F910F91FF90EF90DF90CF9085
:109FE000BF90AF909F908F907F906F9008959F92B9
:109FF000AF92BF92CF92DF92EF92FF920F931F9397
:10A00000CF93DF93EC01992493948E819F81892BC8
:10A0100009F4912C6C817D81E885F9852581368153
:10A02000878190E0A901480F591F6417750704F153
:10A03000A085E380F480442737FD4095542F88277E
:10A0400077FD8095982F0027F7FC0095102FAA2305
:10A0500031F0EFEFEF93EF93EF93E1E004C01F9245
:10A060001F921F92EFEFEF93A12CB12C650120C03E
:10A07000A901481B590B4617570794F140857901F0
:10A080000027F7FC0095102F882777FD8095982FE3
:10A09000218132814423A9F0442737FD4095542F74
:10A0A0001F921F921F921F92A12CB12C6501AA949E
:10A0B0000E94BDA87F836E830F900F900F900F902A
:10A0C00014C0442737FD4095542F1F921F921F92B2
:10A0D0001F92AA24A394BB24BA94CB2CDB2CE8CFE8
:10A0E0001F821E82911001C019828E819F8100976C
:10A0F00089F08F3F910519F014F08FEF90E08130D7
:10A100005FEF950714F481E09FEF9F838E8381E0DA
:10A1100089258A83DF91CF911F910F91FF90EF9056
:10A12000DF90CF90BF90AF909F900895FC018091F9
:10A13000130D9091140DA091170DB091180D139659
:10A140002D913C911497281739072CF418968C916F
:10A15000882361F011C011962D913C9112978217BE
:10A1600093073CF418968C91882331F020E230E07C
:10A1700005C020E130E002C028E030E080911D0DF4
:10A1800090911E0DA091210DB091220D13964D912D
:10A190005C911497481759072CF418968C918823D2
:10A1A00061F00DC011964D915C911297841795073F
:10A1B00044F418968C91882311F0216003C0246028
:10A1C00001C02260808191818217930711F412826D
:10A1D00004C03183208381E08283C901089527E090
:10A1E000289FF001299FF00D1124E955F34F22819A
:10A1F000338141E040832A3347E0340794F4A901D6
:10A2000041545640493F510570F047535F4F493C18
:10A21000510558F02F573440293F310540F422E0D2
:10A2200007C025E005C024E003C023E001C021E011
:10A2300037E0389FF001399FF00D1124E955F34FB5
:10A240000580F681E02D3185332379F0213041F00E
:10A25000223041F0243041F0253039F421E005C0AE
:10A2600025E003C024E001C022E037E0389FF00180
:10A27000399FF00D1124E955F34F8481821302C0F8
:10A280001182089581E08183248308958091270DB0
:10A29000089580919A0C089580919A0C823051F023
:10A2A000833081F08130A1F48091A20C9091A30CB5
:10A2B00096DB05C08091A00C9091A10C87D480936F
:10A2C000970C08C080919E0C90919F0CDDD5F7CF24
:10A2D0001092970C8091970C08951092FC0C10929C
:10A2E000060D1092100D10921A0D1092A60CE8EAAD
:10A2F000FCE0108237968CE0EC3FF807D1F7089528
:10A30000CF93DF93EC01C8DF84E090E09093260DBB
:10A310008093250DCE0101969093040D8093030D3B
:10A320001092FE0C2091970C8981281718F081E07B
:10A330008093FB0CCE010A9690930E0D80930D0D29
:10A340001092080D8A85281718F081E08093050D7A
:10A35000CE0143969093180D8093170D1092120D15
:10A360008B89281718F081E080930F0DCE014C9651
:10A370009093220D8093210D10921C0D8C8D281727
:10A3800018F081E08093190D1092240D80E090E088
:10A39000FE01E80FF91FEF55FF4F20813181215059
:10A3A00031092432310520F481E08093240D04C06A
:10A3B00003968837910561F78091240D811185DC22
:10A3C000FE01E65EFE4F80818F3049F43196808138
:10A3D0008F3029F41092F60B1092F50B09C0FE0194
:10A3E000E05AFE4F808191819093F60B8093F50B9C
:10A3F00082E190E09093A50C8093A40C3091970C8F
:10A400008091250D9091260DA596E7EAFCE041E0AC
:10A41000D683C5832881222321F0321710F0408390
:10A4200001962A9637962CE0EB3FF20789F7909336
:10A43000260D8093250D419734F080E190E09093B4
:10A44000260D8093250D49DF8FEF9CE09093FA0B4A
:10A450008093F90B8091030D9091040D9093F80B6C
:10A460008093F70B8CEF9CE09093FC0B8093FB0B9D
:10A470008DEF9CE09093FE0B8093FD0B8BEF9CE0A7
:10A480009093000C8093FF0B89E09DE09093040C67
:10A490008093030C80910D0D90910E0D9093020C02
:10A4A0008093010C86E09DE09093060C8093050C50
:10A4B00087E09DE09093080C8093070C85E09DE079
:10A4C00090930A0C8093090C83E19DE090930E0C0D
:10A4D00080930D0C8091170D9091180D90930C0C9A
:10A4E00080930B0C80E19DE09093100C80930F0CF7
:10A4F00081E19DE09093120C8093110C8FE09DE020
:10A500009093140C8093130C8DE19DE09093180CA4
:10A510008093170C8091210D9091220D9093160C31
:10A520008093150C8AE19DE090931A0C8093190C8E
:10A530008BE19DE090931C0C80931B0C89E19DE0C6
:10A5400090931E0C80931D0C8091250D9091260DEB
:10A55000049760E07AE0C7E0262F30E0281739073B
:10A560002CF5A9014C5F5F4F749FF001759FF00DB2
:10A570001124E950F44FC29FA001C39F500D112434
:10A580009A012755334F33832283DA01A955B34FFC
:10A5900015962D913C911697318320834855534F42
:10A5A00055834483B187A0876F5FD6CF81E08093C6
:10A5B000270DDF91CF91089581E08093FC0C80936B
:10A5C000060D8093100D80931A0D8093A60CE8EA77
:10A5D000FCE0808337969CE0EC3FF907D1F70895C3
:10A5E0008091230D811142C0E091030DF091040D83
:10A5F000858196819093000D8093FF0C1092020D3F
:10A600001092010DE0910D0DF0910E0D8581968156
:10A6100090930A0D8093090D10920C0D10920B0D62
:10A62000E091170DF091180D858196819093140D8E
:10A630008093130D1092160D1092150DE091210DBF
:10A64000F091220D8581968190931E0D80931D0DB2
:10A650001092200D10921F0D82E190E09093A50CB6
:10A660008093A40CA9DF81E08093230D089580914D
:10A670009A0C823029F48091A00C9091A10CE0C139
:10A68000089580919A0C833029F480919E0C9091CA
:10A690009F0C01C3089580919A0C823049F0833059
:10A6A00069F0813089F48091A20C9091A30C92C939
:10A6B000DEDF8091A00C9091A10C83C2E2DF80913B
:10A6C0009E0C90919F0CDBC381E090E008958091F7
:10A6D0009A0C823039F0833049F0813059F48091FE
:10A6E000D40B0895C4DF80912A0D0895CADF8091AC
:10A6F0006C0D089580E008950F931F93CF93DF931F
:10A70000B6DFBFDFC8DF029709F0C8C0E0DF8823EB
:10A7100009F4C1C014DB1092230D28DB8091FC0CDE
:10A72000882319F08BEF9CE062DC8091060D882372
:10A7300019F085E09DE05BDC8091100D882319F015
:10A740008FE09DE054DC80911A0D882319F089E197
:10A750009DE04DDC8091240D882359F08091100DEF
:10A76000811104C080911A0D882319F084EA9CE0BD
:10A77000DDDC8091240D882309F473C08091A40C42
:10A780009091A50C429731F081E080931C0D80934D
:10A79000120D67C08091F50B9091F60B18161906F3
:10A7A0000CF05BC02091110D6091F00B7091F10BDA
:10A7B0008091980C9091990C2223E1F021E0209354
:10A7C000120D0E94D56481111BC04091F50B509170
:10A7D000F60B662757FD6095762F2CE13DE48091BE
:10A7E000980C9091990C0E946D639093F10B80935B
:10A7F000F00B06C00E94D564811102C01092120DA8
:10A8000020911B0D8091980C9091990C6091EE0B0A
:10A810007091EF0B2223E1F021E020931C0D0E94A8
:10A82000D56481111EC04091F50B5091F60B66273F
:10A8300057FD6095762F2FE13DE48091980C909123
:10A84000990C0E946D639093EF0B8093EE0B09C0FF
:10A850000E94D564811105C002C01092120D1092A1
:10A860001C0DC8EADCE000E010E0FE0131978081B9
:10A87000882351F0EC81FD818781882329F088812C
:10A88000882311F0C801ABDC0F5F1F4F27960C30F7
:10A89000110559F706C021DD35DA03C01EDD80E061
:10A8A00001C081E0DF91CF911F910F910895DFDE0C
:10A8B000E8CE80919A0C823019F0833031F00895FF
:10A8C0008091A00C9091A10C83C180919E0C9091DD
:10A8D0009F0CDCC280919A0C823019F0833031F0E9
:10A8E00008958091A00C9091A10C76C180919E0C4E
:10A8F00090919F0CCFC20895809104018E7F809328
:10A900000401809105018160809305018CE894E148
:10A910009093690D8093680D2EE240EA56E861E05D
:10A9200070E00E94C2A2809165008B7F80936500D9
:10A930001092350189E0809334018EE280933201D8
:10A940008CEF8093300180E98093310180916F001A
:10A95000886080936F0010922C0D10922B0D109236
:10A960002D0D1092290D10922A0DEEE2FDE08CEDD6
:10A9700095E0819391932DE0EE34F207D1F781E0D9
:10A980008093280D08958091680D9091690D0E9423
:10A9900024A3E1E3F1E080818F77808380818F7E43
:10A9A00080831092300108950F931F93CF93DF930C
:10A9B000CEE2DDE0E0E5FDE080E090E0DC0110E0EB
:10A9C00005E09F01F9011B30A0F42F5F3F4F40814C
:10A9D00050E060E070E0012E04C0440F551F661F78
:10A9E000771F0A94D2F7842B952BA62BB72B185FD1
:10A9F000E9CFAC015770405E5340049F9001059F22
:10AA0000300D112437FF02C0295F3F4F43E03595D9
:10AA100027954A95E1F724523A4F299339931B50D1
:10AA20005BE0B695A795979587955A95D1F72DE058
:10AA3000CE34D20731F6DF91CF911F910F91089557
:10AA4000CF92DF92EF92FF920F931F93CF93DF93FA
:10AA5000DD24D394C2E0D0E003E010E0EE24E394E0
:10AA6000F12C8091680D9091690DDC01ED91FC91C4
:10AA70000480F581E02D1995892B09F47FC0C090E1
:10AA800030018091680D9091690DDC01ED91FC9190
:10AA90000680F781E02D199596B3B39A2091840032
:10AAA000309185002059384E30938D0020938C00D2
:10AAB0002C2D2C7139F010924E0D10932C0D00930B
:10AAC0002B0DCFCF93FB992790F9E0914E0DE1111B
:10AAD00016C0992331F28F3021F6D0924E0D80931B
:10AAE0004F0D80912B0D90912C0D892B09F0B9CF32
:10AAF000F0922C0DE0922B0D10922D0DB2CF9111F2
:10AB0000DACF91E09E0F90934E0DF0E0E15BF24FB3
:10AB10008083993109F0A5CF81112DC08091660DF8
:10AB200082FF05C010932C0D00932B0D24C083FDD4
:10AB3000F9CF80912B0D90912C0D019739F48091D4
:10AB40002D0D8F5F80932D0D843020F0D0932C0D30
:10AB5000C0932B0D8091290D8F5F8093290D9091CB
:10AB6000280D981730F4D0922A0D1EDF1092290D6F
:10AB700002C010922A0D10924E0D73CFDF91CF912B
:10AB80001F910F91FF90EF90DF90CF9008953FB706
:10AB9000F89420E0822F90E08417950774F4880FD2
:10ABA000991FFB01E80FF91FDC01A25DB24F8D91E7
:10ABB0009C91918380832F5FEDCF3FBF10922A0D30
:10ABC000089580912B0D90912C0D089580E10895AA
:10ABD00081E08093280D089581E08093280D0895E9
:10ABE0000895809104018E7F809304018091050176
:10ABF0008160809305018CE894E19093AE0D809381
:10AC0000AD0D26E040E052EC61E070E00E94C2A28F
:10AC1000809165008B7F809365001092350180E103
:10AC20008093340186E0809332018EEF809330016F
:10AC300080E98093310180916F00886080936F007C
:10AC400010926E0D10926D0D10926F0D10926B0D93
:10AC500010926C0DE0E7FDE08CED95E0819391930F
:10AC60002DE0EC38F207D1F710928C0D81E0809343
:10AC70006A0D08958091AD0D9091AE0D0E9424A3B0
:10AC8000E1E3F1E080818F77808380818F7E808314
:10AC9000109230010895BF92CF92DF92EF92FF920F
:10ACA0000F931F93CF93DF93DD24D394C2E0D0E0C2
:10ACB00003E010E072E0C72EEE24E394F12C8091C3
:10ACC000AD0D9091AE0DDC01ED91FC910480F5810C
:10ACD000E02D1995892B09F4AEC0B0903001809118
:10ACE000AD0D9091AE0DDC01ED91FC910680F781E8
:10ACF000E02D199596B3B39A209184003091850088
:10AD0000285A344E30938D0020938C002B2D2C71BB
:10AD100019F010928C0D4DC093FB992790F9E0919A
:10AD20008C0DE11109C0992351F2803241F6D09285
:10AD30008C0D80938D0D0BC09111EBCFE130A9F4F8
:10AD4000803409F0BCCFC0928C0D80938E0D809121
:10AD50006D0D90916E0D892B09F0B1CFF0926E0DB3
:10AD6000E0926D0D10926F0DAACF91E09E0F90931F
:10AD70008C0DF0E0E357F24F8083903209F09FCFC3
:10AD800010928C0DEDE8FDE02FEF3FEF8191281B35
:10AD90003109BDE0EB3AFB07C9F74091AB0D80915B
:10ADA000AC0D90E0982F8827840F911D2817390744
:10ADB00029F010936E0D00936D0D81CF80916D0D74
:10ADC00090916E0D019739F480916F0D8F5F809394
:10ADD0006F0D843020F0D0936E0DC0936D0D809177
:10ADE0006B0D8F5F80936B0D90916A0D981700F536
:10ADF000D0926C0D80E090E0FC01E357F24F42816D
:10AE0000238130E0322F2227240F311DA9014F5E0C
:10AE100052404B3D554028F4FC01E059F24F31833C
:10AE2000208302968C31910539F710926B0D47CF34
:10AE300010926C0D44CFDF91CF911F910F91FF9035
:10AE4000EF90DF90CF90BF9008953FB7F89420E047
:10AE5000822F90E08417950774F4880F991FFB01E7
:10AE6000E80FF91FDC01A059B24F8D919C9191839D
:10AE700080832F5FEDCF3FBF10926C0D08958091BE
:10AE80006D0D90916E0D08958EE0089582E080938F
:10AE90006A0D089581E080936A0D089508950895DC
:10AEA00008950895FC01828193818830910529F4E9
:10AEB00010922B0110922A010895099721F4109203
:10AEC000290110922801089508950895CF93DF93E2
:10AED000EC011F8A1E8A49960E9488620E941A9F6E
:10AEE0006C8F7D8F8E8F9F8FDF91CF9108950F9301
:10AEF0001F93CF93DF93EC018091B00D8E01075E1D
:10AF00001F4F811107C061E0C8010E94A96081E064
:10AF10008093B00D4AE06EE0C8010E94AD6021E868
:10AF20003FEF3B872A878FE790E09D878C871F86BE
:10AF30001E86398B288B9B8B8A8B1D8A1C8ADF91FE
:10AF4000CF911F910F910895CF93DF93EC011F8A4A
:10AF50001E8A49960E9403610E941A9F6C8F7D8F02
:10AF60008E8F9F8FDF91CF910895CF93DF93EC0168
:10AF70008091AF0D811108C061E0CE0149960E9419
:10AF80003B6181E08093AF0D21E83FEF3B872A874B
:10AF90008FE790E09D878C871F861E86398B288BD4
:10AFA0009B8B8A8B1D8A1C8ADF91CF910895CF934A
:10AFB000DF93EC011F8A1E8A49960E947B610E94E2
:10AFC0001A9F6C8F7D8F8E8F9F8FDF91CF91089509
:10AFD000CF93DF93EC0121E03FEF3B872A878FEF90
:10AFE00090E09D878C871F861E86398B288B9B8BD4
:10AFF0008A8B1D8A1C8A61E08AE00E9420A161E0A0
:10B0000086E00E9420A161E08DE20E9420A161E023
:10B010008DE00E9420A161E08BE00E9420A161E010
:10B020008EE20E9420A18A819B818830910529F4BB
:10B0300010922B0110922A0106C0099721F4109258
:10B04000290110922801DF91CF910895CF93DF93CA
:10B05000EC011B861A868FEF90E09D878C871F86F8
:10B060001E86198A188A9B8B8A8B1D8A1C8A61E02E
:10B070008CE20E9420A18A819B81089721F4109282
:10B080002D0110922C011AA219A2DF91CF910895DF
:10B09000CF93DF93EC018A816DD448EE53E05B8758
:10B0A0004A8720ED37E03D872C878CED95E09F8720
:10B0B0008E87598B488B3B8B2A8B9D8B8C8BDF919A
:10B0C000CF910895FC01178A168A6CED75E0828194
:10B0D000B6C50F931F93CF93DF93EC018A814AD4B7
:10B0E00021E08D8D811101C020E04B8D5C8D698D3B
:10B0F0007A8D8A8178D68D8D8823A1F08A8112D6A7
:10B100008C016B8D7C8D41E08A812CD661E070E0F2
:10B1100080E090E00E94499F8A81BAD508171907FC
:10B12000A8F313C08A810ED68C016B8D7C8D40E014
:10B130008A8118D661E070E080E090E00E94499F2B
:10B140008A81A6D580179107A8F38A8138D7B801DC
:10B150008A81DF91CF911F910F9171C5CF93DF93BA
:10B16000EC011F8A1E8A8A812AD78B8D882329F0B9
:10B170008A818ED59A8F898F1B8EDF91CF9108950A
:10B18000CF93DF93EC0189A19AA1892B11F01AA228
:10B1900019A2888999899B878A878A899B899D8733
:10B1A0008C878C899D899F878E8710922D011092A4
:10B1B0002C011F8A1E8A0E941A9F6D8F7E8F8F8F8F
:10B1C00098A3DF91CF9108954F925F926F927F92F3
:10B1D0008F929F92AF92BF92CF92DF92EF92FF92A7
:10B1E0000F931F93FC017B01A085B1858684978412
:10B1F0006A177B0719F4282D992D42C0D08C9D0128
:10B20000442737FD4095542F882777FD8095982F48
:10B21000AE15BF052CF446805780DD2029F012C002
:10B2200044805580DD2071F05401CC24B7FCC094DB
:10B23000DC2C72010027F7FC0095102F0484F585A3
:10B24000E02D0DC05401CC24B7FCC094DC2C72015D
:10B250000027F7FC0095102F0284F385E02D2F01C5
:10B26000662457FC6094762C7F926F925F924F9287
:10B270000E94BDA8262F972F0F900F900F900F9030
:10B28000822F1F910F91FF90EF90DF90CF90BF9092
:10B29000AF909F908F907F906F905F904F900895A8
:10B2A000CF93DF93EC017F8B6E8B8EDFAC018A81B5
:10B2B0009B818830910511F461E003C0099729F45E
:10B2C00062E0CE0149960E9478620E941A9F6C8FBC
:10B2D0007D8F8E8F9F8FDF91CF9108950F931F9356
:10B2E000CF93DF93EC010E941A9F0C8D1D8D2E8D44
:10B2F0003F8D601B710B820B930B653F7140810585
:10B30000910540F06E897F89CE01DF91CF911F9129
:10B310000F91C6CFDF91CF911F910F910895CF93D9
:10B32000DF93EC017F8B6E8B4FDFAC018A819B81B9
:10B330008830910511F461E003C0099721F462E0BF
:10B34000CE01499650D70E941A9F6C8F7D8F8E8FA9
:10B350009F8FDF91CF9108950F931F93CF93DF932A
:10B36000EC010E941A9F0C8D1D8D2E8D3F8D601B50
:10B37000710B820B930B653F71408105910540F085
:10B380006E897F89CE01DF91CF911F910F91C7CF39
:10B39000DF91CF911F910F910895CF93DF93EC012F
:10B3A0007F8B6E8B11DFAC018A819B818830910588
:10B3B00011F461E003C0099721F462E0CE014996DF
:10B3C00089D70E941A9F6C8F7D8F8E8F9F8FDF9100
:10B3D000CF9108950F931F93CF93DF93EC010E94B9
:10B3E0001A9F0C8D1D8D2E8D3F8D601B710B820B56
:10B3F000930B653F71408105910540F06E897F890F
:10B40000CE01DF91CF911F910F91C7CFDF91CF91E7
:10B410001F910F9108950F931F93CF93DF938C018A
:10B42000FC01778B668BD0DEEC01F8018281938181
:10B4300088309105D1F4D7FF06C060E08AE00E9411
:10B4400059A161E005C061E08AE00E9459A160E075
:10B4500086E00E9459A1D7FF03C0D195C195D109BB
:10B46000D0932B01C0932A011BC00997C9F4D7FFC1
:10B4700006C060E08DE00E9459A161E005C061E076
:10B480008DE00E9459A160E08BE00E9459A1D7FF96
:10B4900003C0D195C195D109D0932901C09328014A
:10B4A000DF91CF911F910F910895CF93DF93EC011E
:10B4B0007F8B6E8B888599856817790759F48A8107
:10B4C0007ED58B8D882369F08A81E2D39A8F898F0C
:10B4D0001B8E07C0CE0178DEBC018A8156D581E083
:10B4E0008B8FDF91CF910895CF93DF93EC0189A1EA
:10B4F0009AA1892B11F01AA219A29B0177FF03C010
:10B50000319521953109B901CE015EDE90932D016F
:10B5100080932C019F8B8E8B0E941A9F6D8F7E8F44
:10B520008F8F98A3DF91CF910895CF93DF93CDB7FD
:10B53000DEB7A2970FB6F894DEBF0FBECDBF803145
:10B540000CF080E128E034E13A83298320E034E103
:10B550003C832B8328EF33E13E832D8320EF33E1BF
:10B5600038872F8328EE33E13A87298720EE33E1AD
:10B570003C872B8728ED33E13E872D8720ED33E193
:10B58000388B2F8722EC33E13A8B298B20EB33E188
:10B590003C8B2B8B23E933E13E8B2D8B2EE733E164
:10B5A000388F2F8B24E733E13A8F298F2AE633E156
:10B5B0003C8F2B8F2DE533E13E8F2D8F21E533E13D
:10B5C00038A32F8F29E433E13AA329A3E82FEE0F04
:10B5D000FF0BEC0FFD1F81819281A2960FB6F894AC
:10B5E000DEBF0FBECDBFDF91CF910895EF92FF92E6
:10B5F0000F931F93CF93DF93EC016623E1F0262F87
:10B60000653608F024E60A891B89E888F988D8019C
:10B61000AE19BF0930E00E94C8AD28EC30E040E030
:10B6200050E00E9484ADE20EF31EFB86EA86021B08
:10B63000130B1D870C87DF91CF911F910F91FF9006
:10B64000EF900895653620F424E6261B622FCECFB6
:10B650000895CF93DF93EC0177FF03C07195619557
:10B660007109CE01B1DD90932D0180932C019F8B48
:10B670008E8B0E941A9F6D8F7E8F8F8F98A3DF9184
:10B68000CF9108950F931F93CF93DF93EC0189A17E
:10B690009AA1892B39F10E941A9F0D8D1E8D2F8D35
:10B6A00038A1601B710B820B930B60317105810512
:10B6B0009105C0F089A19AA10197A1F46E897F89B3
:10B6C000615071097F8B6E8BCE01161617062CF018
:10B6D000DF91CF911F910F9153CDDF91CF911F91AA
:10B6E0000F91B7CFDF91CF911F910F910895CF9315
:10B6F000DF93EC0189A19AA1892B11F01AA219A25A
:10B70000898D9A8D9B878A872FEF30E03D872C8724
:10B710009F878E87E881F9810190F081E02D60E0BC
:10B7200070E0CE0119951F8A1E8A0E941A9F6D8FA4
:10B730007E8F8F8F98A3DF91CF910895CF93DF9362
:10B74000EC0189A19AA1892B11F01AA219A28B8D63
:10B750009C8D9B878A872FEF30E03D872C879F87C2
:10B760008E87E881F9810190F081E02D60E070E042
:10B77000CE0119951F8A1E8A0E941A9F6D8F7E8F97
:10B780008F8F98A3DF91CF910895FC0180899189D3
:10B79000938782878289938995878487848995890D
:10B7A0009787868786899789892B49F4662319F0BC
:10B7B000818D928D02C0838D948D978B868B81E0D5
:10B7C00090E092A381A30895CF93DF93EC017F8B48
:10B7D0006E8BFADCBC018A81DF91CF9130C2F4CF4D
:10B7E000FC01778B668B82812AC2FC01828150C268
:10B7F0000F931F93CF93DF93EC018A018A8158D274
:10B80000B8018A81DF91CF911F910F916EC2CF93C2
:10B81000DF93EC018A81AED02EEC3FEF3B872A8785
:10B8200082E390E09D878C871F861E86398B288B4C
:10B830009B8B8A8B1D8A1C8A4AEC58E06EEE72E064
:10B84000CE01D6DF8CED95E09A8F898F1B8EDF912C
:10B85000CF9108950F931F93CF93DF93EC01E8A14D
:10B86000F9A180819181A281B3818E01075E1F4F72
:10B8700081159649A105B10509F453C026E040E0C1
:10B8800056E960E070E08FEE93E10E94C2A264E1AD
:10B8900070E080E090E00E94499FE8A1F9A140811A
:10B8A00051816281738141158BE4580761057105EF
:10B8B000E9F068F4403689E0580761057105A1F0A8
:10B8C0004038554261057105B9F442E012C0411596
:10B8D00081EE58076105710559F04115524C6140E0
:10B8E000710551F445E005C041E003C043E001C0EB
:10B8F00046E06FE0C801B0D58FEE93E10E943DA213
:10B90000E8A1F9A1408151816281738126E08FEE27
:10B9100093E10E94C2A264E170E080E090E00E94A6
:10B92000499F4AE06EE0C80197D521E83FEF3B8789
:10B930002A878FE790E09D878C871F861E86398B2C
:10B94000288B9B8B8A8B1D8A1C8ADF91CF911F913C
:10B950000F910895EFE6F0E080818260808380910E
:10B960008400909185008056904F90938900809339
:10B97000880008958930C8F49FB7F89425E1829F24
:10B98000F0011124ED54F24F21E027839FBFE09195
:10B990001C02F0911D02908121E030E0082E01C0D0
:10B9A000220F0A94EAF7922B90830895893070F45D
:10B9B0002FB7F89495E1899FF0011124ED54F24FCF
:10B9C0008CED95E09283818317822FBF0895482FD5
:10B9D00050E095E1899FF0011124ED54F24F21814F
:10B9E000328180859185280F391F83819481821748
:10B9F000930728F08581968128173907E8F485E1B7
:10BA0000849FF001859FF00D1124ED54F24F858144
:10BA100096812817390728F52581368185E1849F8D
:10BA2000F001859FF00D1124ED54F24F8285823094
:10BA300019F411861086128685E1849FF001859F96
:10BA4000F00D1124ED54F24F328321838091840054
:10BA500090918500820F931F9093890080938800B6
:10BA600008958381948182179307C0F623813481DE
:10BA7000D5CFBF92CF92DF92EF92FF920F931F9399
:10BA8000CF93DF938091B20D893048F01092B20DC0
:10BA90008091620E8823B9F090915B0E0DC0E09109
:10BAA000B20DE15085E1E89FF0011124ED54F24F11
:10BAB0008781882341F09081E0911A02F0911B0266
:10BAC000808189278083E091B20D85E1E89FF001B4
:10BAD0001124ED54F24F8781882341F09081E09149
:10BAE0001A02F0911B028081892B8083E091B20DB4
:10BAF00085E1B82EBE9EF0011124ED54F24F8085F1
:10BB00009185892B09F04DC0E091B20DBE9EF001E8
:10BB10001124ED54F24F8285813009F054C00E9407
:10BB20001A9FA091B20DBA9ED0011124AD54B24F0C
:10BB30001B96CD90DD90ED90FC901E97A091B20DDC
:10BB4000BA9ED0011124AD54B24F1F960D911C9195
:10BB500050976C197D098E099F0920E030E0061787
:10BB600017072807390778F5A091B20DC091B20DDB
:10BB7000BC9EE0011124CD54D24F8B899C89BA9E82
:10BB8000D0011124AD54B24F19969C938E931897FF
:10BB9000E091B20DBE9EF0011124ED54F24F82E00F
:10BBA00082878091B20D13DF8091B20D8F5F8093F9
:10BBB000B20DDF91CF911F910F91FF90EF90DF9029
:10BBC000CF90BF900895E091B20D20918400309104
:10BBD000850085E1E89FF0011124ED54F24F818149
:10BBE0009281820F931F9093890080938800DCCF0D
:10BBF0001F920F920FB60F9211240BB60F922F9334
:10BC00003F934F935F936F937F938F939F93AF93E4
:10BC1000BF93EF93FF932DDFFF91EF91BF91AF9112
:10BC20009F918F917F916F915F914F913F912F9154
:10BC30000F900BBE0F900FBE0F901F9018958A307B
:10BC400030F5660F771F282F30E095E1899FF001CE
:10BC50001124ED54F24F858196816817790718F405
:10BC60006581768107C0838194818617970710F4D8
:10BC7000638174818FB7F89495E1929FF001939F4F
:10BC8000F00D1124ED54F24F728361838FBF08953C
:10BC90008A3058F495E1899FF0011124ED54F24F58
:10BCA0008181928196958795089580E090E008952E
:10BCB0008A30D0F46E3E22E0720738F06B3C98E098
:10BCC000790728F06AEC78E002C06EEE72E0660F49
:10BCD000771F9FB7F89425E1829FF0011124ED545E
:10BCE000F24F768365839FBF08958A30D0F46E3E0D
:10BCF00022E0720738F06B3C98E0790728F06AEC94
:10BD000078E002C06EEE72E0660F771F9FB7F8947E
:10BD100025E1829FF0011124ED54F24F7483638377
:10BD20009FBF08958A3058F495E1899FF00111244E
:10BD3000ED54F24F858196819695879508958EEE04
:10BD400092E008958A3058F495E1899FF00111241A
:10BD5000ED54F24F838194819695879508958AECEE
:10BD600098E00895CF93DF93C82FD42F8A30C0F581
:10BD70006233710538F061368DE6780728F060E6A9
:10BD80007DE602C062E370E080E090E00E9431ACAA
:10BD900020E030E04AE754E40E9498AB20E030E035
:10BDA0004CE852E40E94E7AC9B01AC0160E070E01B
:10BDB0008AEF94E40E9498AB0E9400AC9B01DD23C3
:10BDC00021F022273327261B370B8FB7F89495E1F4
:10BDD000C99FE0011124CD54D24F398728878FBFE6
:10BDE000DF91CF9108950F931F93CF93DF93182F77
:10BDF000022F8A3008F067C06F30710540F0EB0108
:10BE000061368DE6780728F0C0E6DDE602C0CFE0B7
:10BE1000D0E04F30510540F0BA0141368DE6580769
:10BE200028F060E67DE602C06FE070E080E090E020
:10BE30000E9431AC20E030E04AE754E40E9498AB25
:10BE400020E030E04CE852E40E94E7AC9B01AC01FA
:10BE500060E070E08AEF94E40E9498AB0E9400AC2E
:10BE6000212F30E045E1429FF001439FF00D112466
:10BE7000ED54F24F002369F0A381B481AB0177FF49
:10BE800004C044275527461B570B5195419551092E
:10BE900009C0A581B681AB0177FF04C044275527AF
:10BEA000461B570B8FB7F89495E1929FF001939F33
:10BEB000F00D1124ED54F24FD08BC787B28BA18BBC
:10BEC000548B438B8FBFDF91CF911F910F910895BA
:10BED0004FB7F89490E025E1289FF001299FF00DDD
:10BEE0001124ED54F24F662351F023813481328BBB
:10BEF000218B23893489121613066CF009C0258121
:10BF00003681328B218B23893489121613061CF457
:10BF10002389348905C023893489319521953109D4
:10BF200055E1589FF001599FF00D1124ED54F24F47
:10BF3000348B238B4FBF08951F93CF93DF93282F0C
:10BF400030E095E1899FF0011124ED54F24F828594
:10BF5000811117C01FB7F89485E1829FE001839F8C
:10BF6000D00D1124CD54D24F81E08A8789899A89D6
:10BF70009A8389830E941A9F6B877C878D879E870F
:10BF80001FBFDF91CF911F9108958A30B8F49B01B4
:10BF90006333710514F022E330E02E3C4FEF340799
:10BFA00014F42EEC3FEF9FB7F89445E1849FF00125
:10BFB0001124ED54F24F318720879FBF08958A30B6
:10BFC00058F49FB7F89425E1829FF0011124ED54B5
:10BFD000F24F118610869FBF08959FB7F894660FA1
:10BFE000771F25E1829FF0011124ED54F24F7283F7
:10BFF000618310829FBF08950F931F93CF93DF93A8
:10C000008091B10D81116DC01092B20DDFB7F8941F
:10C01000C5E188EB9BE02CED35E044E951E161E0BE
:10C0200070E0E091B20DE93008F053C0E091B20D3C
:10C03000CE9FF0011124ED54F24F92838183E09161
:10C04000B20DCE9FF0011124ED54F24F36832583BB
:10C05000E091B20DCE9FF0011124ED54F24F5483C4
:10C060004383E091B20DA091B20D8B0102C0000F8D
:10C07000111FAA95E2F7CE9FF0011124ED54F24F63
:10C080000083E091B20DCE9FF0011124ED54F24FE8
:10C090001782E091B20DCE9FF0011124ED54F24FC2
:10C0A00011861086E091B20DCE9FF0011124ED545F
:10C0B000F24F1286E091B20DCE9FF0011124ED54A3
:10C0C000F24F148A138AE091B20DEF5FE093B20D44
:10C0D000A8CFDFBF60ED77E088E07FDF81E080936D
:10C0E000B10DDF91CF911F910F910895DC01ED917A
:10C0F000FC910190F081E02D1994FC016083528342
:10C10000418308951F93CF93DF93EC01162F6111A4
:10C1100006C06CED75E080E090E00E94499F6AEAFD
:10C1200070E0CE01E3DFE881F9810284F385E02D40
:10C13000CE011995111109C064EF71E080E090E023
:10C14000DF91CF911F910C94499FDF91CF911F9167
:10C150000895FC0181819281D5CF0F931F93CF93D6
:10C16000DF93EC01062F142F89819A81DC01ED9178
:10C17000FC910190F081E02D6881199589819A8167
:10C18000DC01ED91FC910190F081E02D602F19957B
:10C1900089819A81DC01ED91FC910190F081E02D83
:10C1A000612F19958881602F70E0680F711D610FF4
:10C1B000711D6F77772789819A81DF91CF911F91C8
:10C1C0000F9194CF4038510514F04FE750E04138BB
:10C1D0002FEF520714F441E85FEF57FF03C051956A
:10C1E00041955109BACF2FEF260F223058F4623013
:10C1F00011F424E001C020E0652F661F6627661F4A
:10C20000620FE0CF0895CF93DF93EC0140E060E050
:10C21000A4DF40E064E0CE01DF91CF919ECFFC012E
:10C2200060835283418308951F93CF93DF93EC0182
:10C23000162F611106C06CED75E080E090E00E9461
:10C24000499F6AEA70E0CE0151DFE881F9810284FA
:10C25000F385E02DCE011995111106C064EF71E050
:10C2600080E090E00E94499F62E870E0CE01DF919B
:10C27000CF911F913BCFFC0181819281D5CF2AEADA
:10C280002093700EDC012C912093710E6093720E3E
:10C290004093730E11968D919C911297DC01ED9154
:10C2A000FC910280F381E02D44E050E060E77EE005
:10C2B00019944F37510514F04EE750E042382FEFF4
:10C2C000520714F442E85FEF57FF03C051954195C0
:10C2D0005109D5CF613031F457FF02C06AE009C07F
:10C2E00068E007C0623031F457FF02C06EE001C061
:10C2F0006CE0DFCF0895CF93DF93EC0140E068E07E
:10C30000BEDF40E06CE0CE01DF91CF91B8CF24E8F2
:10C310002093700E6093710E4093720E25E520936A
:10C32000730E2AE22093740EDC0111968D919C917C
:10C330001297DC01ED91FC910280F381E02D45E044
:10C3400050E060E77EE0199565E070E080E090E005
:10C350000E94499F80E008951F93CF93DF93EC01E3
:10C36000162F61E088DF65E070E080E090E00E94D9
:10C37000499F42E462E4CE01CADF412F60E0CE0172
:10C38000C6DF81115FC040E061E0CE01C0DF8111F6
:10C3900059C040E062E0CE01BADF811153C046E0EF
:10C3A00062E0CE01B4DF81114DC040E063E0CE0118
:10C3B000AEDF811147C040E064E0CE01A8DF11E0AC
:10C3C000811110E040E065E0CE01A1DF811101C0E4
:10C3D0001F5F40E066E0CE019ADF811101C01F5F60
:10C3E00040E067E0CE0193DF811101C01F5F40E0B4
:10C3F00068E0CE018CDF811101C01F5F40E069E081
:10C40000CE0185DF811101C01F5F44E06AE0CE01EB
:10C410007EDF811101C01F5F44E06AE0CE0177DF5B
:10C42000811101C01F5F62E370E080E090E00E9434
:10C43000499F62E870E089819A8158DE81E0183076
:10C4400011F0111180E0DF91CF911F910895FC014F
:10C4500060835283418308950F931F93CF93DF939B
:10C46000EC01062F142F89819A81DC01ED91FC915A
:10C470000190F081E02D6881199589819A81DC0114
:10C48000ED91FC910190F081E02D602F199589814B
:10C490009A81DC01ED91FC910190F081E02D612FFA
:10C4A000199589819A81DC01ED91FC912881602F99
:10C4B00070E0620F711D610F711D6F77772701901A
:10C4C000F081E02DDF91CF911F910F9119944038A9
:10C4D000510514F04FE750E041382FEF520714F4A4
:10C4E00041E85FEF57FF03C0519541955109B4CF23
:10C4F0002FEF260F223058F4623011F424E001C0EF
:10C5000020E0652F661F6627661F620FE0CF089543
:10C51000CF93DF93EC0140E060E09EDF40E064E019
:10C52000CE01DF91CF9198CFCF93DF93EC010E94A2
:10C530001A9FFE01E65CFD4F21E030E0318320834D
:10C540009E01FE0140E050E0DE01A40FB51FAC5596
:10C55000BE4F1C92D901A858BF4F11961C921E9233
:10C560006193719381939193A051BF4F11961C9247
:10C570001E92AA56BF4F1D921C924F5F5F4F2E5FB7
:10C580003F4F4E31510501F7C45CDD4F19821882CF
:10C59000DF91CF910895FC01E45CFD4F2081318152
:10C5A0002E31310594F420E030E0FC01E858FF4FD3
:10C5B00040815181452B39F02F5F3F4F02962E313C
:10C5C000310599F702C0C90108958FEF9FEF0895D3
:10C5D0008F929F92AF92BF92CF92DF92EF92FF9293
:10C5E0000F931F93CF93DF9300D01F92CDB7DEB789
:10C5F0004C01590149835A836B837C83CCDF498189
:10C600005A816B817C8197FD4DC0A114B10409F45E
:10C6100049C07C01EE0CFF1CEE0CFF1CE80CF91C61
:10C62000F701EC54FF4F40835183628373836C01A5
:10C63000CC0CDD1CC80CD91CF601E858FF4FB182A8
:10C64000A082EC54FF4F11830083880D991DFC01DB
:10C65000EC55FE4F81E080830E941A9FF7016083B2
:10C66000718382839383F401E65CFD4F8081918125
:10C67000D601A250BE4F8D939C93D401A45CBD4FB4
:10C680002D913C9111972F5F3F4F2D933C939C012F
:10C690002F5F3F4F1216130614F021E030E0318374
:10C6A000208302C08FEF9FEF0F900F900F900F909D
:10C6B000DF91CF911F910F91FF90EF90DF90CF907E
:10C6C000BF90AF909F908F9008950F931F9300E0BD
:10C6D00010E07EDF1F910F9108950F931F9301E0EB
:10C6E00010E076DF1F910F9108959C0180E090E0AB
:10C6F000F901E250FE4F408151814617570741F042
:10C7000001962E5F3F4F8E31910591F78FEF9FEF8E
:10C710000895EF92FF920F931F93CF93DF93EC0155
:10C720008C01045C1D4FF801E080F180E114F104FC
:10C73000C9F1DBDF8F3FFFEF9F07A1F19C01220FC3
:10C74000331F2C0F3D1FF901E858FF4F40815181E5
:10C75000452B41F111821082FE01E80FF91FEC55C3
:10C76000FE4F1082F901EE53FE4F11821082FC0140
:10C77000BD96EE0FFF1FEE0FFF1FEC0FFD1F108287
:10C78000118212821382F901E859FE4F1182108240
:10C79000EA56FF4F1182108221E0E21AF108F801F7
:10C7A000F182E082DF91CF911F910F91FF90EF9086
:10C7B00008952F923F924F925F926F927F928F9245
:10C7C0009F92AF92BF92CF92DF92EF92FF920F9320
:10C7D0001F93CF93DF9300D000D0CDB7DEB79E83F9
:10C7E0008D830E941A9FED81FE81FA83E98320E008
:10C7F00030E022242394312C49815A814E535E4FDC
:10C800005C834B83DA011D921C9249815A814858FE
:10C810005F4FDA014D915C91452B09F457C0C08000
:10C82000D180E280F380AF014C545F4FDA018D90EC
:10C830009D90AD90BC902B013C014C185D086E089A
:10C840007F08481459046A047B0408F43FC0C80CEC
:10C85000D91CEA1CFB1CC082D182E282F3824D818A
:10C860005E81420F531F4C555E4FDA014C914423B9
:10C8700069F149815A81445D5E4FDA014D915C91C5
:10C880004115510529F4AB81BC812D923C921EC00B
:10C89000E980FA80B8E9EB1ABEEFFB0AD7010D91E7
:10C8A0001C910417150794F4AB81BC812D923C9226
:10C8B0000F5F1F4FD7010D931C930417150734F01A
:10C8C00042E050E0AB81BC814D935C932F5F3F4FC2
:10C8D000A981BA811296BA83A98334962E31310583
:10C8E00009F08ACFED80FE80BCE3EB0EF11C0D81D8
:10C8F0001E81F801EE53FE4F8081918181309105B8
:10C9000091F00297B9F4F801E858FF4F0190F081D7
:10C91000E02D1995F801E250FE4F608171818D8103
:10C920009E81F7DE07C0F801E858FF4F0190F081C3
:10C93000E02D19950E5F1F4F0E151F05D1F6269697
:10C940000FB6F894DEBF0FBECDBFDF91CF911F9120
:10C950000F91FF90EF90DF90CF90BF90AF909F909E
:10C960008F907F906F905F904F903F902F900895A1
:10C970000F931F93CF93DF93EC01B7DE8C010F3F32
:10C980008FEF180769F00E941A9FF801EE0FFF1F42
:10C99000EE0FFF1FEC0FFD1F608371838283938373
:10C9A000DF91CF911F910F910895CF93DF93EC0109
:10C9B0009CDE8F3F2FEF920731F0C80FD91FCC5567
:10C9C000DE4F888101C080E0DF91CF910895CF9341
:10C9D000DF93CDB7DEB72A970FB6F894DEBF0FBE50
:10C9E000CDBF85300CF080E02EE734E13A83298317
:10C9F00029E734E13C832B832FE634E13E832D830A
:10CA00002BE634E138872F832AE534E13A872987FA
:10CA1000E82FEE0FFF0BEC0FFD1F818192812A960C
:10CA20000FB6F894DEBF0FBECDBFDF91CF91089552
:10CA300082E080939F0E80919F0E8093990E1092BA
:10CA40009D0E1092970E1092A20E81E080939C0E84
:10CA500082ED90E09093900E80938F0E90938E0EC7
:10CA600080938D0E08958093A30E60938C0E409357
:10CA70008B0E1092950010929400109290008CE012
:10CA80008093910084EF90E09093990080939800B8
:10CA900081E088BB82E0809371000895EF920F934C
:10CAA0008093960E6093950E4093920E2093910E74
:10CAB0000093940EE092930E0F91EF900895E1E7AA
:10CAC000F0E080818D7F80830895E1E7F0E0808150
:10CAD0008260808308958091A20E811103C08091AD
:10CAE0009C0E8111F2CFEBCF8093940E089580932A
:10CAF000930E08958091940E08958091930E089559
:10CB0000109295001092940080919D0E8F5F8093FB
:10CB10009D0E90919E0E891784F010929D0E20918B
:10CB20009F0E8091A00E9091A10E820F911D27FD66
:10CB30009A959093A10E8093A00E8091970E8F5F8F
:10CB40008093970E9091980E891784F01092970E0B
:10CB50002091990E80919A0E90919B0E820F911DBB
:10CB600027FD9A9590939B0E80939A0E08951F929D
:10CB70000F920FB60F9211240BB60F922F933F9383
:10CB80004F935F936F937F938F939F93AF93BF93D5
:10CB9000EF93FF93B5DFFF91EF91BF91AF919F911D
:10CBA0008F917F916F915F914F913F912F910F9056
:10CBB0000BBE0F900FBE0F901F901895AF92BF92B3
:10CBC000DF92EF92FF920F931F93CF93DF931F9209
:10CBD000CDB7DEB7233039F0243041F4D72EDD1C39
:10CBE000DD24DD1C04C0DD24D39401C0D12C7B01E5
:10CBF00077FF03C0F194E194F1081092A20E213066
:10CC000009F4CEC0002309F1223029F480918D0E61
:10CC100090918E0E04C080918F0E9091900EE81628
:10CC2000F9060CF05EC081E08093A20E3091930E65
:10CC3000C70144E0959587954A95E1F78E5F1FEF10
:10CC400018160CF44AC081E048C0CA0157FF03C05F
:10CC50009195819591098E159F05D4F43091960E8A
:10CC6000332309F4A0C031E03093A20E3091940E2A
:10CC70004091920E413079F5A701481B590B4D3375
:10CC800051050CF0345011E0449734F584E025C090
:10CC9000E816F9060CF087C03091950E332309F49D
:10CCA00082C0243009F47FC031E03093A20E30916D
:10CCB000930E4091910E413009F078C042E3E416A2
:10CCC000F10414F43E5F72C08E199F09C3970CF4EF
:10CCD0006DC032506BC011E082E05701131634F082
:10CCE00004C0A12CB12C1FEF81E031E09091A20E85
:10CCF0009923C1F04FB7F894189F802D1124809389
:10CD00009F0E30939E0EAB2839F08091A00E90912B
:10CD1000A10E892B09F44CC0A090A00EB090A10EDA
:10CD20004FBF09C08FB7F89410929F0EB092A10E1A
:10CD3000A092A00E8FBF2983CEDE2981002319F097
:10CD4000B7FE28C023C0113031F4B7FC1FC0EA146D
:10CD5000FB0404F51EC01F3FE9F4223049F4AE1471
:10CD6000BF04BCF08FEFA816B104A1F09CF00AC07C
:10CD7000233081F4AE14BF0464F0EFEFAE16B104BB
:10CD800049F044F0AA24AA94B12C04C0A12CB12CDF
:10CD900001C05701DD20B1F0B194A194B10812C0D7
:10CDA000A12CB12C01C0570111E09ECF1FEF94CFF1
:10CDB00080919F0E992787FD90959093A10E809367
:10CDC000A00EAACFC5010F90DF91CF911F910F91B7
:10CDD000FF90EF90DF90BF90AF900895CF92DF92D9
:10CDE000EF920F931F93CF93DF931F92CDB7DEB7D0
:10CDF000E1100AC08B0177FF03C01195019511095D
:10CE00000417150764F402C000E010E081E080938D
:10CE10009C0E8FEF433351059CF495E012C04017F0
:10CE2000510734F010929C0E81E021E091E00AC09D
:10CE30004D335105BCF381E080939C0E93E001C01B
:10CE400094E022E030919C0E332379F03FB7F894C0
:10CE5000829F202D11242093990E9093980EC090BC
:10CE60009A0ED0909B0E3FBF0AC09FB7F8941092C5
:10CE7000990E10939B0E00939A0E9FBF68018983B1
:10CE80002ADE8981EE2019F0D7FE1BC016C0813042
:10CE900031F4D7FC12C00C151D059CF411C08F3F56
:10CEA00081F4C016D10664F08FEFC816D10449F0A2
:10CEB00044F0CC24CA94D12C04C0C12CD12C01C084
:10CEC0006801C6010F90DF91CF911F910F91EF90F4
:10CED000DF90CF9008951816190654F0892B51F45D
:10CEE000672B51F080918B0E882331F084E00895F8
:10CEF00082E0089583E0089581E00895823021F46E
:10CF000081E0633031F406C0833019F481E062308F
:10CF100009F080E00895AF92BF92CF92DF92EF9236
:10CF2000FF920F931F9377FF1AC0AA24BB24A41A61
:10CF3000B50ACC24B7FCC094DC2C882777FD8095FB
:10CF4000982F2FEF2F932F932F932F93EE24EA9464
:10CF5000FE2C870121E03FEF4FEF5FEF1CC0611512
:10CF6000710509F1882777FD8095982F8A0122277E
:10CF700017FD2095322F3F932F931F930F93A12CD2
:10CF8000B12C6501A394E12CF12C8701EA9421E0F6
:10CF900030E040E050E00E94BDA8CB010F900F9020
:10CFA0000F900F9002C080E090E01F910F91FF90D2
:10CFB000EF90DF90CF90BF90AF9008959FEF980FC4
:10CFC000933010F480938C0E089580918C0E089508
:10CFD00080938B0E089580918B0E08952F923F922F
:10CFE0004F925F926F927F928F929F92AF92BF9279
:10CFF000CF92DF92EF92FF920F931F93CF93DF9325
:10D00000CDB7DEB72A970FB6F894DEBF0FBECDBFFF
:10D010004B013A013E832D8318870F83411551053B
:10D0200009F4EBC06115710559F480918B0E8823CA
:10D0300009F4E5C088249924841A950ACA01E4C039
:10D040001B0177FF04C022243324261A370A3A86AC
:10D050002986230177FE04C0442455244618570826
:10D0600020918C0E223011F1233009F475C021304B
:10D0700009F0AEC0B201882777FD8095982F610135
:10D08000EE24D7FCE094FE2CFF92EF92DF92CF9239
:10D09000A12CB12C6501E12CF12C8701EA9420E050
:10D0A00030E0A9010E94BDA8C1014FC0B10188278D
:10D0B00077FD8095982F0E9433AC6B017C01C201F3
:10D0C000AA2797FDA095BA2F89839A83AB83BC8347
:10D0D000BC01CD010E9433AC20E030E04FE753E4C7
:10D0E0000E9498AB9B01AC01C701B6010E94E7AC5E
:10D0F0000E9400AC620D731D6F3F710519F014F0B2
:10D100006FEF70E07A87698777FF02C01A86198609
:10D11000E985FA85CF01AA2797FDA095BA2FBF937D
:10D12000AF939F938F93A12CB12C6501E12CF12C2F
:10D130008701EA9420E030E0A90169817A818B813E
:10D140009C810E94BDA889859A85861B970B0F90AC
:10D150000F900F900F903EC0B201882777FD809509
:10D16000982F6101EE24D7FCE094FE2CFF92EF9201
:10D17000DF92CF92A12CB12C6501E12CF12C87011B
:10D18000EA9420E030E0A9010E94BDA80F900F9022
:10D190000F900F90CB0195958795A101480F591FCE
:10D1A0009101281B390BC9012F3F310519F014F0EB
:10D1B0008FEF90E097FF02C080E090E04F3F510575
:10D1C00019F014F04FEF50E05A87498757FF02C01B
:10D1D0001A86198677FC06C039852A859A87898739
:10D1E000832F922F97FE0EC0919581959109898486
:10D1F0009A8491948194910807C0CB0105C080E086
:10D2000090E002C089849A84AD81BE818D929C9207
:10D21000EF81F885918380832A960FB6F894DEBF5C
:10D220000FBECDBFDF91CF911F910F91FF90EF9077
:10D23000DF90CF90BF90AF909F908F907F906F9036
:10D240005F904F903F902F90089590938A0E809317
:10D25000890E6093870E5093860E4093850E109230
:10D26000880E81E08093800E08958091890E9091C0
:10D270008A0E892B89F08091800E882381F00E948C
:10D280001A9F6093810E7093820E8093830E909309
:10D29000840E1092800E089581E08093800E089590
:10D2A0000F931F938091800E81111CC00E941A9FC2
:10D2B0000091810E1091820E2091830E3091840E88
:10D2C000601B710B820B930B0091890E10918A0EDB
:10D2D00020E030E0061717072807390718F481E027
:10D2E0008093800E1F910F910895DADF8091880E50
:10D2F0000895D6DF8091800E8823B9F08091880E42
:10D30000811113C081E08093880E1092800EADDFF2
:10D310008091870E882359F06BE474E18091850E2B
:10D320009091860E0E9474A602C080E0089581E06C
:10D330000895B6DF8091800E8823A9F08091880E31
:10D34000882389F01092880E1092800E8EDF8091D3
:10D35000870E882341F06BE374E18091850E9091F4
:10D36000860E0C9474A6089524E630E030937F0E68
:10D3700020937E0E80937C0E70937B0E60937A0ECA
:10D3800010927D0E81E08093750E089580917E0E3F
:10D3900090917F0E892B89F08091750E882381F002
:10D3A0000E941A9F6093760E7093770E8093780E8A
:10D3B0009093790E1092750E089581E08093750E0A
:10D3C00008950F931F938091750E81111CC00E94C8
:10D3D0001A9F0091760E1091770E2091780E309161
:10D3E000790E601B710B820B930B00917E0E1091D6
:10D3F0007F0E20E030E0061717072807390718F4DA
:10D4000081E08093750E1F910F910895DADF80916E
:10D410007D0E0895D6DF8091750E8823B1F080913E
:10D420007D0E811112C081E080937D0E1092750EE9
:10D43000ADDF80917C0E882341F067E274E180913A
:10D440007A0E90917B0E0C9474A60895BADF8091A9
:10D45000750E8823A9F080917D0E882389F01092A3
:10D460007D0E1092750E92DF80917C0E882341F024
:10D4700060E174E180917A0E90917B0E0C9474A619
:10D48000089580E00895FC011282138214821582AF
:10D4900016821782128608954F925F926F927F9242
:10D4A0008F929F92AF92BF92CF92DF92EF92FF92B4
:10D4B0000F931F93CF93DF937C01DC01ED91FC91DF
:10D4C000369700811181080F191FF8014284F3E09B
:10D4D000F41508F086C0C0E0D0E093E8A92E95E1ED
:10D4E000B92EC0FF7AC0D80118968D909C901997DC
:10D4F0006E01CC0CDD1CC80CD91CF601608071805B
:10D50000F5016591749180E090E00E9431AC25E8CE
:10D510003BEE41E55FE30E94E7AC0E9405AC661676
:10D52000770608F45AC0D601CD90DC90F5016591DC
:10D53000749180E090E00E9431AC2EE33AE047E93C
:10D540005FE30E94E7AC20E030E040E85FE30E9448
:10D5500030AB0E9405AC6C157D0508F43EC08C0E06
:10D56000911C8C0E911CC0E0D0E05E01A80CB91C8F
:10D57000F50160807180CE018D579A4E6C01FC01DF
:10D580006591749180E090E00E9431AC25E83BEE1B
:10D5900041E55FE30E94E7AC0E9405AC66167706A2
:10D5A00000F1D501AD90BC90F6016591749180E0D9
:10D5B00090E00E9431AC2EE33AE047E95FE30E943D
:10D5C000E7AC20E030E040E85FE30E9430AB0E942F
:10D5D00005AC6A157B0538F404C02196C41508F41F
:10D5E00080CF80E016C02296C630D10509F0BDCFAD
:10D5F00083E0F8018783D701ED91FC913697019084
:10D60000F081E02DEE0DFF1D13821482158216822B
:10D6100081E0DF91CF911F910F91FF90EF90DF900C
:10D62000CF90BF90AF909F908F907F906F905F90C2
:10D630004F9008954F925F926F927F928F929F9238
:10D64000AF92BF92CF92DF92EF92FF920F931F9310
:10D65000CF93DF937C01DC01ED91FC913697008143
:10D660001181080F191FF8014284F3E0F41508F046
:10D6700086C0C0E0D0E03BE7A32E35E1B32EC0FF6B
:10D680007AC0D80118968D909C9019976E01CC0C99
:10D69000DD1CC80CD91CF60160807180F501659114
:10D6A000749180E090E00E9431AC25E83BEE41E5CA
:10D6B0005FE30E94E7AC0E9405AC6616770608F4AB
:10D6C0005AC0D601CD90DC90F5016591749180E04F
:10D6D00090E00E9431AC2EE33AE047E95FE30E941C
:10D6E000E7AC20E030E040E85FE30E9430AB0E940E
:10D6F00005AC6C157D0508F43EC08C0E911C8C0E9B
:10D70000911CC0E0D0E05E01A80CB91CF50160805E
:10D710007180CE0185589A4E6C01FC01659174911F
:10D7200080E090E00E9431AC25E83BEE41E55FE30C
:10D730000E94E7AC0E9405AC6616770600F1D501A1
:10D74000AD90BC90F6016591749180E090E00E94EC
:10D7500031AC2EE33AE047E95FE30E94E7AC20E01A
:10D7600030E040E85FE30E9430AB0E9405AC6A15F0
:10D770007B0538F404C02196C41508F480CF80E0FE
:10D7800016C02296C630D10509F0BDCF83E0F8015E
:10D790008783D701ED91FC9136970190F081E02DC0
:10D7A000EE0DFF1D138214821582168281E0DF9137
:10D7B000CF911F910F91FF90EF90DF90CF90BF908E
:10D7C000AF909F908F907F906F905F904F90089553
:10D7D0004F925F927F928F929F92AF92BF92CF9221
:10D7E000DF92EF92FF920F931F93CF93DF93DC01B1
:10D7F000ED91FC913697A081B181A80FB91F1A96BF
:10D800007C901A97E2E3E71508F08CC042E050E004
:10D8100060E070E0C12CD12C40FD5CC01896CD9129
:10D82000DC911997FE01E60FF71F208131812C3919
:10D83000394008F44FC020813181263D3D4008F039
:10D8400049C04A01AA24A394B12C20E030E02E0163
:10D85000E2E04E0E511C460E571E2496C60FD71FEF
:10D86000F201E20FF31FE080F1801EECE11614E0FC
:10D87000F106D0F1E080F1801CEEE11616E0F10631
:10D8800098F5DD0CED2DE160DE2EFE01E20FF31FB9
:10D89000E080F1801AE9E11611E0F10608F442C0D7
:10D8A0000190F081E02DE035F240E0F5F401319691
:10D8B000F497C4F5F501E770FF27EF2BA9F12C5F72
:10D8C0003F4FEFEFAE1ABE0A12E0810E911C2036D8
:10D8D000310531F66E5F7F4F4F5F5F4F2EEF240FA4
:10D8E000271508F499CF3FC0E080F1801AE9E116CE
:10D8F00011E0F106B8F00190F081E02DE035F24042
:10D9000088F4DD0CFE01E20FF31FE080F1801EECD5
:10D91000E11614E0F10630F00190F081E02DEC3ECC
:10D92000F64020F280E01FC0EC2DF0E0ED58FA4EFA
:10D93000E491DE12F7CFC394E2E0EC1590F428E115
:10D9400017962C93DC01ED91FC9136970190F081B4
:10D95000E02DE80FF91F138214821582168281E0F0
:10D9600002C0D12CACCFDF91CF911F910F91FF90CE
:10D97000EF90DF90CF90BF90AF909F908F907F906F
:10D980005F904F9008956F927F928F929F92AF9287
:10D99000BF92CF92DF92EF92FF920F931F93CF939C
:10D9A000DF937C01DC01ED91FC913697C081D18140
:10D9B000C80FD91F8A85873008F43EC0C884D9842F
:10D9C00000E010E0B2E0CB0ED11C4601800E911EAB
:10D9D000F40160807180C8018D599A4E5C01FC0190
:10D9E0006591749180E090E00E9431AC25E83BEEB7
:10D9F00041E55FE30E94E7AC0E9405AC661677063E
:10DA0000D8F0D4018D909C90F5016591749180E0DF
:10DA100090E00E9431AC2EE33AE047E95FE30E94D8
:10DA2000E7AC20E030E040E85FE30E9430AB0E94CA
:10DA300005AC6815790510F480E016C00E5F1F4F25
:10DA40000E30110509F0C1CF87E08F83D701ED912A
:10DA5000FC9136970190F081E02DEE0DFF1D1382B1
:10DA600014821582168281E0DF91CF911F910F9170
:10DA7000FF90EF90DF90CF90BF90AF909F908F90EE
:10DA80007F906F900895DC01ED91FC9136970190A5
:10DA9000F081E02DE80FF91F2285283090F122E077
:10DAA00030E060E0A085B185A20FB31F4D915C917D
:10DAB000119760FF09C0433D514018F14D915C91B1
:10DAC000423A524048F01DC04C3F5140D0F04D9179
:10DAD0005C914D3D5240A8F46F5F2E5F3F4F673021
:10DAE00009F76783DC01ED91FC9136970190F08195
:10DAF000E02DE80FF91F138214821582168281E04F
:10DB0000089580E008950F931F93CF93DF93DC0176
:10DB1000ED91FC913697A081B181A80FB91F1A969B
:10DB20002C911A97223108F450C01896ED91FC916F
:10DB300019972281338126393A4108F446C022815F
:10DB400033812434364208F040C0349618E040E077
:10DB500050E0BA0120813181273F3440B0F120816B
:10DB600031812732374088F5EF01229622813381B7
:10DB70002E3E394000F1228133812C343E40D8F4CE
:10DB8000440F551F661F771F4160115034961111C5
:10DB9000E1CF28E017962C93DC01ED91FC913697AC
:10DBA0000190F081E02DE80FF91F438354836583D2
:10DBB000768381E011C028813981273F344028F0E5
:10DBC000288139812732374010F080E005C0440FAA
:10DBD000551F661F771FD9CFDF91CF911F910F91EE
:10DBE00008950F931F93CF93DF93DC01ED91FC9188
:10DBF0003697A081B181A80FB91F1A962C911A9758
:10DC0000223108F463C01896ED91FC911997228196
:10DC100033812432354108F459C0228133812E36B4
:10DC20003E4108F053C0369618E040E050E0BA019B
:10DC3000EF012297288139812934354078F12881F4
:10DC400039812D39374050F5440F551F661F771F16
:10DC5000416020813181233C3140C0F120813181FC
:10DC60002B38324098F5115034961111E1CF28E04D
:10DC700017962C93DC01ED91FC9136970190F08181
:10DC8000E02DE80FF91F438354836583768381E099
:10DC90004B35510561057105C9F419C028813981D9
:10DCA000233C314098F0288139812B38324070F480
:10DCB000440F551F661F771F20813181293435405D
:10DCC00028F0208131812D39374068F280E0DF91E2
:10DCD000CF911F910F910895DC01ED91FC91369742
:10DCE0000190F081E02DE80FF91F13821482158254
:10DCF000168280E008954F925F926F927F928F928A
:10DD00009F92AF92BF92CF92DF92EF92FF920F93CA
:10DD10001F93CF93DF937C01DC01ED91FC9136974B
:10DD200000811181080F191FF8014284F4E0F415F5
:10DD300008F086C0C0E0D0E04BE3A42E45E1B42E4D
:10DD4000C0FF7AC0D80118968D909C9019976E01EB
:10DD5000CC0CDD1CC80CD91CF60160807180F5016B
:10DD60006591749180E090E00E9431AC25E83BEE33
:10DD700041E55FE30E94E7AC0E9405AC66167706BA
:10DD800008F45AC0D601CD90DC90F50165917491EC
:10DD900080E090E00E9431AC2EE33AE047E95FE397
:10DDA0000E94E7AC20E030E040E85FE30E9430AB47
:10DDB0000E9405AC6C157D0508F43EC08C0E911CCC
:10DDC0008C0E911CC0E0D0E05E01A80CB91CF501DE
:10DDD00060807180CE01855C9A4E6C01FC0165917A
:10DDE000749180E090E00E9431AC25E83BEE41E583
:10DDF0005FE30E94E7AC0E9405AC6616770600F16F
:10DE0000D501AD90BC90F6016591749180E090E0F1
:10DE10000E9431AC2EE33AE047E95FE30E94E7ACB1
:10DE200020E030E040E85FE30E9430AB0E9405ACA8
:10DE30006A157B0538F404C02196C41508F480CF18
:10DE400080E016C02296C830D10509F0BDCF84E02D
:10DE5000F8018783D701ED91FC9136970190F0810D
:10DE6000E02DEE0DFF1D138214821582168281E0D3
:10DE7000DF91CF911F910F91FF90EF90DF90CF90A6
:10DE8000BF90AF909F908F907F906F905F904F90DA
:10DE900008954F925F926F927F928F929F92AF926E
:10DEA000BF92CF92DF92EF92FF920F931F93CF9387
:10DEB000DF937C01DC01ED91FC91369700811181AB
:10DEC000080F191FF8014284F4E0F41508F086C029
:10DED000C0E0D0E06BE4A62E65E1B62EC0FF7AC0AC
:10DEE000D80118968D909C9019976E01CC0CDD1C72
:10DEF000C80CD91CF60160807180F50165917491A0
:10DF000080E090E00E9431AC25E83BEE41E55FE324
:10DF10000E94E7AC0E9405AC6616770608F45AC06A
:10DF2000D601CD90DC90F5016591749180E090E090
:10DF30000E9431AC2EE33AE047E95FE30E94E7AC90
:10DF400020E030E040E85FE30E9430AB0E9405AC87
:10DF50006C157D0508F43EC08C0E911C8C0E911C36
:10DF6000C0E0D0E05E01A80CB91CF50160807180B2
:10DF7000CE01855B9A4E6C01FC016591749180E045
:10DF800090E00E9431AC25E83BEE41E55FE30E9462
:10DF9000E7AC0E9405AC6616770600F1D501AD909E
:10DFA000BC90F6016591749180E090E00E9431ACE4
:10DFB0002EE33AE047E95FE30E94E7AC20E030E07F
:10DFC00040E85FE30E9430AB0E9405AC6A157B0518
:10DFD00038F404C02196C41508F480CF80E016C040
:10DFE0002296C830D10509F0BDCF84E0F8018783BF
:10DFF000D701ED91FC9136970190F081E02DEE0D67
:10E00000FF1D138214821582168281E0DF91CF9169
:10E010001F910F91FF90EF90DF90CF90BF90AF9046
:10E020009F908F907F906F905F904F9008954F9248
:10E030005F926F927F928F929F92AF92BF92CF9298
:10E04000DF92EF92FF920F931F93CF93DF937C01A8
:10E05000DC01ED91FC91369700811181080F191FA9
:10E06000F8014284F4E0F41508F086C0C0E0D0E086
:10E07000E3E4AE2EE5E1BE2EC0FF7AC0D8011896CB
:10E080008D909C9019976E01CC0CDD1CC80CD91C8E
:10E09000F60160807180F5016591749180E090E0F7
:10E0A0000E9431AC25E83BEE41E55FE30E94E7AC1E
:10E0B0000E9405AC6616770608F45AC0D601CD90CA
:10E0C000DC90F5016591749180E090E00E9431ACA4
:10E0D0002EE33AE047E95FE30E94E7AC20E030E05E
:10E0E00040E85FE30E9430AB0E9405AC6C157D05F3
:10E0F00008F43EC08C0E911C8C0E911CC0E0D0E048
:10E100005E01A80CB91CF50160807180CE018D5BA9
:10E110009A4E6C01FC016591749180E090E00E9440
:10E1200031AC25E83BEE41E55FE30E94E7AC0E949D
:10E1300005AC6616770600F1D501AD90BC90F601EE
:10E140006591749180E090E00E9431AC2EE33AE05A
:10E1500047E95FE30E94E7AC20E030E040E85FE39E
:10E160000E9430AB0E9405AC6A157B0538F404C0F0
:10E170002196C41508F480CF80E016C02296C830DE
:10E18000D10509F0BDCF84E0F8018783D701ED9177
:10E19000FC9136970190F081E02DEE0DFF1D13826A
:10E1A00014821582168281E0DF91CF911F910F9129
:10E1B000FF90EF90DF90CF90BF90AF909F908F90A7
:10E1C0007F906F905F904F9008950F931F93CF9320
:10E1D000DF93DC01ED91FC913697A081B181A80F0E
:10E1E000B91F1A962C911A972A3108F450C0189624
:10E1F000ED91FC91199722813381203B374008F43F
:10E2000046C02281338122313B4008F040C0349621
:10E210001CE040E050E0BA01208131812C3E3140C9
:10E22000B0F120813181263C324088F5EF01229601
:10E2300022813381283D334000F1228133812A3805
:10E240003540D8F4440F551F661F771F41601150A9
:10E2500034961111E1CF2CE017962C93DC01ED914F
:10E26000FC9136970190F081E02DE80FF91F438370
:10E2700054836583768381E011C0288139812C3EE7
:10E28000314028F028813981263C324010F080E06E
:10E2900005C0440F551F661F771FD9CFDF91CF915F
:10E2A0001F910F9108951F93CF93DF93EC016EE8B8
:10E2B00074E185EB92E10E9438A6E885F9856081DA
:10E2C00071814AE050E085EB92E10E947AA711E06B
:10E2D0008A85181728F569E874E185EB92E10E94B8
:10E2E00038A64AE050E0612F85EB92E10E945AA7E0
:10E2F00066E874E185EB92E10E9438A698858985ED
:10E30000E92FF82FE10FF11DE10FF11D60817181FF
:10E310004AE050E085EB92E10E947AA71F5FD8CFD8
:10E32000DF91CF911F91089581E090E09093200FAD
:10E3300080931F0F10928C0F0E94269F6093220FD4
:10E340007093230F8093240F9093250FE49AEC9AF7
:10E350000895CF93DF93EC01E881F9813A978081AA
:10E3600091818C0F9D1F98D828813981F9018823CC
:10E3700049F036970190F081E02DEC0FFD1F81E010
:10E38000828312C13C97808191818C0F9D1F52D94D
:10E3900028813981F901882341F036970190F08175
:10E3A000E02DEC0FFD1F82E012C03E97808191812D
:10E3B0008C0F9D1F0DDA28813981F901882351F0D6
:10E3C00036970190F081E02DEC0FFD1F83E08283F2
:10E3D00081E0EAC07097808191818C0F9D1FD3DA14
:10E3E00028813981F901882341F036970190F08125
:10E3F000E02DEC0FFD1F84E0EACF729780819181C0
:10E400008C0F9D1F40DB28813981F901882341F061
:10E4100036970190F081E02DEC0FFD1F85E0D7CFFE
:10E420007497808191818C0F9D1F6DDB28813981CC
:10E43000F901882341F036970190F081E02DEC0F2F
:10E44000FD1F86E0C4CF7697808191818C0F9D1F40
:10E45000C8DB28813981F901882341F03697019082
:10E46000F081E02DEC0FFD1F87E0B1CF7897808120
:10E4700091818C0F9D1F30DC28813981F90188231F
:10E4800041F036970190F081E02DEC0FFD1F88E000
:10E490009ECFB097808191818C0F9D1F96DE288141
:10E4A0003981882391F0F90136970190F081E02DB0
:10E4B000EC0FFD1F43815481658176814031510508
:10E4C0006105710511F499E043C0F9017A978081E3
:10E4D00091818C0F9D1F0FDC28813981882349F0A1
:10E4E000F90136970190F081E02DEC0FFD1F8AE0D5
:10E4F0006ECFF9017C97808191818C0F9D1FC9DCC3
:10E5000028813981F901882341F036970190F08103
:10E51000E02DEC0FFD1F8BE05ACFB09780819181E9
:10E520008C0F9D1F52DE28813981882399F0F901D3
:10E5300036970190F081E02DEC0FFD1F438154814F
:10E5400065817681403154406105710519F49CE084
:10E5500092832AC0F9017E97808191818C0F9D1F43
:10E5600066DD28813981882349F0F90136970190C9
:10E57000F081E02DEC0FFD1F8DE029CFF901B09760
:10E58000808191818C0F9D1F20DE28813981F901C6
:10E5900036970190F081E02DEC0FFD1F882311F0DC
:10E5A0008EE015CF128280E0DF91CF910895CF9356
:10E5B000DF9300D000D0CDB7DEB796E0E3E2F2E023
:10E5C000DE01119601900D929A95E1F7863040F4A4
:10E5D000E1E0F0E0EC0FFD1FE80FF11D808101C0CC
:10E5E0008FEF26960FB6F894DEBF0FBECDBFDF913A
:10E5F000CF910895CF93DF93CDB7DEB76E970FB667
:10E60000F894DEBF0FBECDBF8F300CF080E023E367
:10E6100035E13A8329832CE235E13C832B832EE1DB
:10E6200035E13E832D8322E135E138872F8328E0D1
:10E6300035E13A87298721E035E13C872B872DEFAB
:10E6400034E13E872D8726EF34E1388B2F872BEE80
:10E6500034E13A8B298B2EED34E13C8B2B8B23ED6F
:10E6600034E13E8B2D8B27EC34E1388F2F8B25EB5B
:10E6700034E13A8F298F24EA34E13C8F2B8F2FE944
:10E6800034E13E8F2D8FE82FEE0FFF0BEC0FFD1FB7
:10E69000818192816E960FB6F894DEBF0FBECDBF1A
:10E6A000DF91CF910895CF93DF93CDB7DEB7289751
:10E6B0000FB6F894DEBF0FBECDBF84300CF080E003
:10E6C0002AE934E13A83298328E934E13C832B8326
:10E6D00026E934E13E832D8324E934E138872F8312
:10E6E000E82FEE0FFF0BEC0FFD1F81819281289622
:10E6F0000FB6F894DEBF0FBECDBFDF91CF91089566
:10E70000FC0187EE93E09183808386E29FE091870E
:10E7100080871386158614861282138214821582CE
:10E720001682178212860895CF93DF93EC01E88159
:10E73000F98136970190F081E02DE80FF91F1282E0
:10E74000862F992787FD9095A92FB92FFC01319726
:10E7500028813981EE30F10508F02EC1E05FFE4FCF
:10E760000C94C2ADF9013A97808191818C0F9D1F65
:10E770000E944C6A882309F427C1E881F981369701
:10E780000190F081E02DEC0FFD1F81E014C0F90134
:10E790003C97808191818C0F9D1F0E941A6B88236A
:10E7A00009F412C1E881F98136970190F081E02DDA
:10E7B000EC0FFD1F82E0828307C1F9013E97808143
:10E7C00091818C0F9D1F04D8882309F4FDC0E88136
:10E7D000F98136970190F081E02DEC0FFD1F83E069
:10E7E000EACFF9017097808191818C0F9D1FCBD862
:10E7F000882309F4E9C0E881F98136970190F08116
:10E80000E02DEC0FFD1F84E0D6CFF90172978081D7
:10E8100091818C0F9D1F37D9882309F4D5C0E881D9
:10E82000F98136970190F081E02DEC0FFD1F85E016
:10E83000C2CFF9017497808191818C0F9D1F63D99C
:10E84000882309F4C1C0E881F98136970190F081ED
:10E85000E02DEC0FFD1F86E0AECFF90176978081A9
:10E8600091818C0F9D1FBDD9882309F4ADC0E8812B
:10E87000F98136970190F081E02DEC0FFD1F87E0C4
:10E880009ACFF9017897808191818C0F9D1F24DAAE
:10E89000882309F499C0E881F98136970190F081C5
:10E8A000E02DEC0FFD1F88E086CFF901B097808145
:10E8B00091818C0F9D1F89DC882309F485C0E88134
:10E8C000F98136970190F081E02DEC0FFD1F438117
:10E8D000548165817681403151056105710509F0EA
:10E8E00073C080C0F9017A97808191818C0F9D1F40
:10E8F00002DA882309F468C0E881F981369701902B
:10E90000F081E02DEC0FFD1F8AE055CFF9017C97D7
:10E91000808191818C0F9D1FBCDA882309F454C03B
:10E92000E881F98136970190F081E02DEC0FFD1F11
:10E930008BE041CFF901B097808191818C0F9D1FB1
:10E9400044DC882309F440C0E881F98136970190BE
:10E95000F081E02DEC0FFD1F4381548165817681AC
:10E96000403154406105710579F53EC0F9017E974B
:10E97000808191818C0F9D1F5ADB882329F1E881CA
:10E98000F98136970190F081E02DEC0FFD1F8DE0AD
:10E9900012CFF901B097808191818C0F9D1F15DCFA
:10E9A000882391F0E881F98136970190F081E02D7C
:10E9B000EC0FFD1F8EE0FFCEF90136970190F0813C
:10E9C000E02DEC0FFD1F1282E881F981369701904E
:10E9D000F081E02DEC0FFD1F81E09281911106C0C6
:10E9E00080E004C089E0E7CE8CE0E5CEDF91CF91F6
:10E9F00008958091210F882339F080918C0F80FF3A
:10EA000002C0289A089528980895EF92FF920F93D4
:10EA10001F93CF93DF938C01EB017A01E881F98199
:10EA20000190F081E02DCB01199580918C0F8A87A0
:10EA300040E080918C0F481720F5A42FB0E0CD0165
:10EA4000880F991FE885F985E80FF91FDC01AA5D99
:10EA5000B04F2D913C912E9DC0012F9D900D3E9D5C
:10EA6000900D1124D80112962C9130E040FF03C084
:10EA7000319521953109280F391F318320834F5F4C
:10EA8000D8CF81E0DF91CF911F910F91FF90EF9050
:10EA90000895CF93DF93EC0180911E0F60E00E94F8
:10EAA00020A1E881F9810190F081E02DCE01DF9174
:10EAB000CF911994FC01862F2DEF35E0318320830F
:10EAC0001092210F92E39283638371DD80931E0F76
:10EAD000EAE6F0E080818C7F8083808181608083A2
:10EAE0000895CF92DF92EF92FF920F931F93CF93EF
:10EAF000DF93EC018B0180911F0F9091200F059700
:10EB0000F9F480911E0F0E948EA1892BC9F0C0904C
:10EB1000220FD090230FE090240FF090250F0E9439
:10EB2000269F6C197D098E099F09613E7E428105F1
:10EB3000910530F084E090E09093200F80931F0FB8
:10EB400080911F0F9091200F049741F4EC9841E0C1
:10EB500050E0B801CE0159DF81E001C080E0DF91D3
:10EB6000CF911F910F91FF90EF90DF90CF9008957C
:10EB70001F920F920FB60F9211240BB60F92CF92E5
:10EB8000DF92EF92FF921F932F933F934F935F93E8
:10EB90006F937F938F939F93AF93BF93EF93FF9365
:10EBA000CF93DF9300D01F92CDB7DEB780911E0FB9
:10EBB0000E948EA111E0892B09F010E00E94269F8F
:10EBC00069837A838B839C83C980DA80EB80FC80A5
:10EBD0008091220F9091230FA091240FB091250FC7
:10EBE000C81AD90AEA0AFB0A80911F0F9091200FD8
:10EBF0008430910509F441C08530910519F00197E1
:10EC0000A1F40BC0F6DE112381F081EEC8168EE26E
:10EC1000D806E104F10448F02AC0112371F185E01F
:10EC200090E09093200F80931F0F80911F0F909181
:10EC3000200F059711F5E0918C0FF0E0EE0FFF1F0C
:10EC4000EA5DF04FD182C08289819A81AB81BC811B
:10EC50008093220F9093230FA093240FB093250F3E
:10EC600080918C0F8F5F80938C0F833330F084E022
:10EC700090E09093200F80931F0F0F900F900F90B4
:10EC80000F90DF91CF91FF91EF91BF91AF919F9145
:10EC90008F917F916F915F914F913F912F911F9134
:10ECA000FF90EF90DF90CF900F900BBE0F900FBEB4
:10ECB0000F901F90189561E089E00E9420A160E00C
:10ECC00089E00E9459A11092110F0895CF93C82F87
:10ECD00061E089E00E9420A160E089E00E9459A1E2
:10ECE0002C2F30E040E050E060E47FE180E090E0F5
:10ECF0000E94A6AD81E08093B00089E08093B100CE
:10ED00002093B3008BEA289F212D11242695209370
:10ED1000B400CF9108958091110F811134C01092E9
:10ED20000F0F10920C0F81E08093110F8091100F44
:10ED3000CDDF80916F008B7F80936F008091B0005A
:10ED400080628093B0002091840030918500E09132
:10ED50000C0F81E08E0F80930C0F84E0E89FF00190
:10ED60001124EC55F14F80819181A281B381280F4C
:10ED7000391F30938B0020938A00B29A80916F00E4
:10ED8000846080936F000895EFE6F0E080818B7FD0
:10ED900080831092110F08959091110F81E08927BF
:10EDA00008951F93CF93DF938091120F833009F062
:10EDB0005FC08091130F8130D1F488EE93E0A0E022
:10EDC000B0E08093A40E9093A50EA093A60EB093EE
:10EDD000A70E80E797E1A0E0B0E08093A80E9093A3
:10EDE000A90EA093AA0EB093AB0EC2E001C0C0E082
:10EDF000E091130FF0E0EC5EF04FD08110E11C0FBA
:10EE000088EE93E0A0E0B0E048EB5BE060E070E00B
:10EE10002C2F30E0F901EE0FFF1FEE0FFF1FEC5516
:10EE2000F14FD7FF10C04083518362837383F90190
:10EE3000EE0FFF1FEE0FFF1FE855F14F8083918308
:10EE4000A283B3830FC080839183A283B383F9012C
:10EE5000EE0FFF1FEE0FFF1FE855F14F4083518368
:10EE600062837383CE5FDD0FC113D2CFC0930D0FCA
:10EE7000DF91CF911F91089590910C0F80910D0F0C
:10EE8000981316C010920C0F8091130F8F5F809310
:10EE9000130F9091130F8091140F891740F481E0A4
:10EEA0008093130F80910F0F8F5F80930F0F79DF87
:10EEB00090910F0F80910E0F981306C08091B000B3
:10EEC0008F7D8093B00060CF8091B00085FF04C03B
:10EED0008091B0008F7D03C08091B00080628093EC
:10EEE000B0002091840030918500E0910C0F81E00A
:10EEF0008E0F80930C0F84E0E89FF0011124EC55F5
:10EF0000F14F80819181A281B381280F391F309305
:10EF10008B0020938A0008951F920F920FB60F92D4
:10EF200011240BB60F922F933F934F935F936F93E0
:10EF30007F938F939F93AF93BF93EF93FF939CDF48
:10EF4000FF91EF91BF91AF919F918F917F916F91C1
:10EF50005F914F913F912F910F900BBE0F900FBE7D
:10EF60000F901F90189584E080930D0F8AE0809396
:10EF70000E0F86E28093100F81E08093130F809331
:10EF8000140F8093120F43E855E120E030E08091A8
:10EF90000D0F90E028173907CCF4FA018591949170
:10EFA000A0E0B0E0880F991FAA1FBB1FF901EE0F68
:10EFB000FF1FEE0FFF1FEC55F14F80839183A2835B
:10EFC000B3832F5F3F4F4E5F5F4FE1CFA4CE84E00E
:10EFD00080930D0F8AE080930E0F86E28093100FCE
:10EFE00081E08093130F8093140F82E08093120FBF
:10EFF0004BE755E120E030E080910D0F90E02817BD
:10F000003907CCF4FA0185919491A0E0B0E0880F23
:10F01000991FAA1FBB1FF901EE0FFF1FEE0FFF1F65
:10F02000EC55F14F80839183A283B3832F5F3F4FD1
:10F030004E5F5F4FE1CF6FCE84E080930E0F85E28D
:10F040008093100F81E08093130F88E08093140F5A
:10F0500083E08093120F80E090E0FC01ED58FA4EBF
:10F06000E491DC01AB5EB04FEC93019688309105E2
:10F07000A1F797DE50CE88E080930D0F86E0809355
:10F080000E0F86E28093100F81E08093130F809320
:10F09000140F84E08093120F43E655E120E030E046
:10F0A00080910D0F90E028173907CCF4FA01859173
:10F0B0009491A0E0B0E0880F991FAA1FBB1FF9012F
:10F0C000EE0FFF1FEE0FFF1FEC55F14F8083918372
:10F0D000A283B3832F5F3F4F4E5F5F4FE1CF1BCEC5
:10F0E00088E080930D0F86E080930E0F86E2809378
:10F0F000100F81E08093130F8093140F85E08093AD
:10F10000120F43E555E120E030E080910D0F90E0D3
:10F1100028173907CCF4FA0185919491A0E0B0E06A
:10F12000880F991FAA1FBB1FF901EE0FFF1FEE0FDB
:10F13000FF1FEC55F14F80839183A283B3832F5F30
:10F140003F4F4E5F5F4FE1CFE6CD0F931F93CF93BD
:10F15000DF9382E180930D0F86E080930E0F96E29D
:10F160009093100F91E09093130F9093140F80934E
:10F17000120F88ED90E4A0E0B0E08093A40E90938D
:10F18000A50EA093A60EB093A70E8CE19CE0A0E084
:10F19000B0E08093A80E9093A90EA093AA0EB0930E
:10F1A000AB0EB42FAA2799278827E2E0F0E04CE1C4
:10F1B0005CE060E070E008E318E120E030E0EF019F
:10F1C000CC0FDD1FCC0FDD1FCC55D14FB7FF05C0D5
:10F1D000088319832A833B8304C0488359836A8345
:10F1E0007B83EF01CC0FDD1FCC0FDD1FC855D14F46
:10F1F000488359836A837B83880F991FAA1FBB1F8B
:10F200003296E231F105D9F68CE199E8A0E0B0E060
:10F210008093E80E9093E90EA093EA0EB093EB0E64
:10F22000DF91CF911F910F9176CDCF92DF92EF9228
:10F23000FF920F931F93CF93DF9382E180930D0F83
:10F2400085E080930E0F82E28093100F81E080931F
:10F25000130F8093140F87E08093120F80E993E3DC
:10F26000A0E0B0E08093A40E9093A50EA093A60E0C
:10F27000B093A70EB42FAA279927882722E030E061
:10F28000E1E0F0E04CE454E060E070E0C4EECC2E4D
:10F29000CCE0DC2EE12CF12CEF01CC0FDD1FCC0FEC
:10F2A000DD1F8901000F111F000F111FCC55D14F19
:10F2B000B7FF0CC0C882D982EA82FB82E801CC5534
:10F2C000D14F488359836A837B830BC0488359831A
:10F2D0006A837B83E801CC55D14FC882D982EA8208
:10F2E000FB82880F991FAA1FBB1F32962E5F3F4FCC
:10F2F0002231310589F688E79FEFA0E0B0E08093E6
:10F30000E80E9093E90EA093EA0EB093EB0EDF9116
:10F31000CF911F910F91FF90EF90DF90CF90FBCC9A
:10F3200084E080930D0F82E380930E0F86E280933A
:10F33000100F81E08093130F8093140F8AE0809365
:10F34000120F4BE355E120E030E080910D0F90E08B
:10F3500028173907CCF4FA0185919491A0E0B0E028
:10F36000880F991FAA1FBB1FF901EE0FFF1FEE0F99
:10F37000FF1FEC55F14F80839183A283B3832F5FEE
:10F380003F4F4E5F5F4FE1CFC6CC84E080930D0FBF
:10F3900080E280930E0F86E28093100F81E08093CD
:10F3A000130F8093140F8BE08093120F4BE455E101
:10F3B00020E030E080910D0F90E028173907CCF461
:10F3C000FA0185919491A0E0B0E0880F991FAA1FDF
:10F3D000BB1FF901EE0FFF1FEE0FFF1FEC55F14FA2
:10F3E00080839183A283B3832F5F3F4F4E5F5F4F34
:10F3F000E1CF91CC84E080930D0F83E080930E0FDA
:10F4000086E28093100F81E08093130F8093140F96
:10F410008DE08093120F43E455E120E030E08091CD
:10F420000D0F90E028173907CCF4FA0185919491DB
:10F43000A0E0B0E0880F991FAA1FBB1FF901EE0FD3
:10F44000FF1FEE0FFF1FEC55F14F80839183A283C6
:10F45000B3832F5F3F4F4E5F5F4FE1CF5CCCAF92E6
:10F46000BF92CF92DF92EF92FF920F931F93CF93B1
:10F47000DF938AE180930D0F20930E0F88E2809333
:10F48000100F81E08093130F8093140F8EE0809310
:10F49000120F80EC92E1A0E0B0E08093A40E909374
:10F4A000A50EA093A60EB093A70E80EB94E0A0E06B
:10F4B000B0E08093A80E9093A90EA093AA0EB093EB
:10F4C000AB0E24E1440F551F661F771F2A95D1F715
:10F4D00032E0A32EB12CE3E0F0E000E619E020E0FA
:10F4E00030E0C0E4CC2ECCE9DC2EE12CF12CE5019F
:10F4F000CC0FDD1FCC0FDD1FCC55D14F77FF05C0E2
:10F50000088319832A833B8304C088839983AA8351
:10F51000BB83E931F10561F0EF01CC0FDD1FCC0FAA
:10F52000DD1FCC55D14F88839983AA83BB8308C044
:10F53000C092080FD092090FE0920A0FF0920B0FC1
:10F54000440F551F661F771F3296C2E0AC0EB11CE8
:10F55000EB31F10561F6DF91CF911F910F91FF9093
:10F56000EF90DF90CF90BF90AF90D5CBCF93DF934C
:10F570001F921F92CDB7DEB7CE0101969CDB83EEC2
:10F5800093E09A83898323E040E150E060E070E0FB
:10F59000CE01019664DF0F900F90DF91CF91089517
:10F5A000CF93DF931F921F92CDB7DEB7CE010196A6
:10F5B00082DB83EE93E09A83898321E040E154E08B
:10F5C00060E070E0CE0101964ADF0F900F90DF916E
:10F5D000CF9108950F931F93CF93DF93EC01062FE4
:10F5E000BA01A901112707FD1095212F312F0150D4
:10F5F00011090E30110508F0A2C0025E1E4FF8017D
:10F600000C94C2ADA881B98118978D919C918C0FF3
:10F610009D1FDF91CF911F910F91A5CCA881B9813A
:10F620001A978D919C918C0F9D1FDF91CF911F9107
:10F630000F91CDCCA881B9811C978D919C918C0F95
:10F640009D1FDF91CF911F910F91F6CCA881B981B9
:10F650001E978D919C918C0F9D1FDF91CF911F91D3
:10F660000F9109CDA881B98150978D919C918C0FF4
:10F670009D1FDF91CF911F910F9132CDA881B9814C
:10F6800052978D919C918C0F9D1FDF91CF911F916F
:10F690000F915BCDA881B98154978D919C918C0F6E
:10F6A0009D1FDF91CF911F910F91BFCDA881B9818F
:10F6B00058978D919C918C0F9D1FDF91CF911F9139
:10F6C0000F9154CFA881B9815A978D919C918C0F3D
:10F6D0009D1FDF91CF911F910F9122CEA881B981FB
:10F6E0005C978D919C918C0F9D1FDF91CF911F9105
:10F6F0000F914BCEA881B9815E978D919C918C0F13
:10F700009D1FDF91CF911F910F914ACFA881B981A1
:10F7100090978D919C918C0F9D1FDF91CF911F91A0
:10F720000F9168CEA881B98192978D919C9123E029
:10F730008C0F9D1FDF91CF911F910F9190CEDF9184
:10F74000CF911F910F910895CF93DF93EC01462F36
:10F75000552747FD5095652F752F415051094D3064
:10F76000510508F085C0445D5E4FFA010C94C2ADAE
:10F77000A881B98118978D919C918C0F9D1FDF9165
:10F78000CF91F1CBA881B9811A978D919C918C0F63
:10F790009D1FDF91CF911BCCA881B9811C978D91C2
:10F7A0009C918C0F9D1FDF91CF9146CCA881B98190
:10F7B0001E978D919C918C0F9D1FDF91CF915BCCFB
:10F7C000A881B98150978D919C918C0F9D1FDF91DD
:10F7D000CF9186CCA881B98152978D919C9140E5BB
:10F7E00050E060E070E08C0F9D1FDF91CF91ADCCB9
:10F7F000A881B98154978D919C914BE550E060E0D0
:10F8000070E08C0F9D1FDF91CF910FCDA881B98142
:10F8100058978D919C918C0F9D1FDF91CF91A6CE13
:10F82000A881B9815A978D919C918C0F9D1FDF9172
:10F83000CF9176CDA881B9815C978D919C918C0FE9
:10F840009D1FDF91CF91A1CDA881B9815E978D9148
:10F850009C918C0F9D1FDF91CF91A2CEA881B98181
:10F8600090978D919C918C0F9D1FDF91CF91C2CD70
:10F87000DF91CF910895DC01ED91FC9138972081C3
:10F880003181820F931F0C944C6ADC01ED91FC9145
:10F89000389720813181820F931F0C941A6BDC0101
:10F8A000ED91FC91389720813181820F931F0C9448
:10F8B000E86BDC01ED91FC91389720813181820F5A
:10F8C000931F0C94C36CDC01ED91FC91389720815F
:10F8D0003181820F931F0C94436DDC01ED91FC91FB
:10F8E000389720813181820F931F0C94836DDC0146
:10F8F000ED91FC91389720813181820F931F0C94F8
:10F90000F16DDC01ED91FC91389720813181820FFE
:10F91000931F0C946C6EDC01ED91FC913897208163
:10F920003181820F931F0C947B6EDC01ED91FC9171
:10F93000389720813181820F931F0C94496FDC012D
:10F94000ED91FC91389720813181820F931F0C94A7
:10F950001770DC01ED91FC91389720813181820F85
:10F96000931F0C94E570DC01ED91FC913897208198
:10F970003181820F931F0C94A971CF93DF93CDB780
:10F98000DEB72A970FB6F894DEBF0FBECDBF843026
:10F990000CF084E02BEC35E13A83298324EB35E14C
:10F9A0003C832B8322EA35E13E832D8323E935E135
:10F9B00038872F832BE835E13A872987E82FEE0F28
:10F9C000FF0BEC0FFD1F818192812A960FB6F894F0
:10F9D000DEBF0FBECDBFDF91CF910895FC016483E0
:10F9E0000895FC0166830895FC0163830895FC017A
:10F9F0008281089508950895FC0112821382148271
:10FA00001582168217820895FF920F931F93CF934A
:10FA1000DF93EC01F62E042F122F6AED70E088853B
:10FA200099850E94766088859985DC01ED91FC912D
:10FA30000190F081E02D6F2D199588859985DC0165
:10FA4000ED91FC910190F081E02D602F1995888552
:10FA50009985DC01ED91FC910190F081E02D612F01
:10FA600019956F2D70E066527F4F600F711D610F09
:10FA7000711D6F77772788859985DF91CF911F91C9
:10FA80000F91FF900C94766021E040E06DE3BCCFD5
:10FA900021E040E06EE3B8CF21E040E06FE3B4CF77
:10FAA00022E040E06DE3B0CF22E040E06EE3ACCF77
:10FAB00022E040E06FE3A8CF23E040E06DE3A4CF75
:10FAC00023E040E06EE3A0CF23E040E06FE39CCF73
:10FAD00024E040E06DE398CF24E040E06EE394CF73
:10FAE00024E040E06FE390CF462F21E064E48CCF28
:10FAF000462F22E064E488CF462F23E064E484CFDD
:10FB0000462F24E064E480CF462F25E064E47CCFD8
:10FB1000462F26E064E478CF20E076CF77FF03C05D
:10FB2000719561957109462F6EE2F6CF462F66E416
:10FB3000F3CF462F67E4F0CF20E040E065CF6CE2E2
:10FB4000FBCF6DE2F9CF6FE2F7CF60E3F5CF61E372
:10FB5000F3CF62E3F1CF63E3EFCF64E3EDCF65E38F
:10FB6000EBCF66E3E9CF67E3E7CFFC0124812223F3
:10FB700039F02581211104C021E0258368E3DCCF21
:10FB80000895FC012481222331F02581222319F0DC
:10FB9000158269E3D1CF0895FC012681222339F033
:10FBA0002781211104C021E027836AE3C5CF08958E
:10FBB000FC012681222331F02781222319F01782AC
:10FBC0006BE3BACF0895FC012381222311F06CE38B
:10FBD000B3CF0895CF93DF93EC018A81811105C0E3
:10FBE00060E4CE01A9DF81E08A83DF91CF9108959F
:10FBF000CF93DF93EC018A81882321F061E4CE0169
:10FC00009BDF1A82DF91CF91089565E495CFDF9253
:10FC1000EF92FF920F931F93CF93DF938C01D22E1D
:10FC2000643F81E0780738F0613187E2780728F097
:10FC300060E177E202C064EF71E0443F81E0580781
:10FC400040F0EA01413187E2580728F0C0E1D7E2ED
:10FC500002C0C4EFD1E0CB01845F914022E3E22EE9
:10FC6000F12CB7010E945DAD462F2D2D62E4C80135
:10FC7000CBDECE01845F9140B7010E945DAD462F7F
:10FC80002D2D63E4C801DF91CF911F910F91FF905B
:10FC9000EF90DF90B9CE21E0BACF22E0B8CF23E0D9
:10FCA000B6CF24E0B4CF25E0B2CF26E0B0CFFC0140
:10FCB00062830895FC01648308950895089508956A
:10FCC000089508950895089508950895089508954C
:10FCD000089508950895089508950895089508953C
:10FCE00080E0089508950895089508950895089569
:10FCF000089508950895089508950895089508951C
:10FD00000895089508958091940F9091950F9260B1
:10FD10009093950F8093940F8091940F9091950FED
:10FD200080649093950F8093940F089580E094E001
:10FD30009093950F8093940F0895DC01ED91FC91C1
:10FD40000680F781E02D60E070E019948091940FB7
:10FD50009091950F80629093950F8093940F0895E2
:10FD60008091940F9091950F20E282279093950FA8
:10FD70008093940F08958091940F9091950F8061D6
:10FD80009093950F8093940F08958091940F909184
:10FD9000950F80689093950F8093940F08958091AC
:10FDA000940F9091950F91609093950F8093940F7D
:10FDB0000895FC01128213821482158261E086E1AB
:10FDC0000E9420A161E086E10E9459A1E2E7F0E0F3
:10FDD0008081816080831092950F1092940F089516
:10FDE00077FF03C07195619571096F3F710519F037
:10FDF00014F06FEF70E08091940F9091950F8C7BD1
:10FE000091709093950F8093940F8091940F90919F
:10FE1000950F6F30710514F480641FC0673371054E
:10FE200014F481641AC06F3571051CF4816490610B
:10FE300014C0673871051CF4816490630EC06F3A7A
:10FE400071051CF48164906408C0673D71051CF461
:10FE50008164906502C0816490669093950F809351
:10FE6000940F0895FC018481882371F085818111AC
:10FE70000BC081E085838091940F9091950F8860ED
:10FE80009093950F8093940F0895FC0184818823AB
:10FE900071F08581882359F015828091940F90919B
:10FEA000950F28E082279093950F8093940F0895E3
:10FEB000FC018281882371F0838181110BC081E074
:10FEC00083838091940F9091950F84609093950F08
:10FED0008093940F0895FC018281882371F08381BF
:10FEE000882359F013828091940F9091950F24E00C
:10FEF00082279093950F8093940F08958091930F8C
:10FF00008F5F8093930F9091920F891708F4FFC031
:10FF10001092930F8091910F90E08730910508F037
:10FF2000F6C0FC01E75CFE4F0C94C2AD60E086E1D8
:10FF30000E9459A188E08093920F81E048C061E05F
:10FF400086E10E9459A181E08093920F36C060E063
:10FF500086E10E9459A180918F0F9091900F97FF99
:10FF600005C083E08093920F84E031C081E08093EC
:10FF7000920F83E02CC061E086E10E9459A183E0EA
:10FF800005C061E086E10E9459A181E08093920F53
:10FF900080918E0F8F5F80938E0F803120F01092B2
:10FFA0008E0F85E014C080918F0F9091900F880F75
:10FFB000991F9093900F80938F0F82E008C060E0AC
:10FFC00086E10E9459A181E08093920F86E08093A0
:10FFD000910F089561E086E10E9459A188E1809324
:10FFE000920F8091940F9091950F9093900F809322
:10FFF0008F0F8091940F9091950F91FF1DC080916C
:020000021000EC
:100000008D0F8823B1F08091940F9091950F22E08D
:1000100092279093950F8093940F8091940F9091D5
:10002000950F80649093950F8093940F10928D0F8D
:1000300003C081E080938D0F8091940F9091950F74
:1000400092FF0EC080918D0F882339F01092950F8A
:100050001092940F10928D0F03C081E080938D0F4A
:100060008091940F9091950F84FF14C080918D0F13
:10007000882369F08091940F9091950F20E1822759
:100080009093950F8093940F10928D0F03C081E091
:1000900080938D0F8091940F9091950F87FF13C0DF
:1000A00080918D0F882361F08091940F9091950F2E
:1000B00080589093950F8093940F10928D0F03C0EA
:1000C00081E080938D0F8091940F9091950F90FF18
:1000D00014C080918D0F882369F08091940F9091C6
:1000E000950F21E092279093950F8093940F109293
:1000F0008D0F03C081E080938D0F8091940F9091BC
:10010000950F9093900F80938F0F1092910F0895F9
:100110001F920F920FB60F9211240BB60F922F93CE
:100120003F934F935F936F937F938F939F93AF937F
:10013000BF93EF93FF93E2DEFF91EF91BF91AF91F9
:100140009F918F917F916F915F914F913F912F91EF
:100150000F900BBE0F900FBE0F901F90189581E06F
:100160008093B30F6CED75E00C941F5E0F931F939B
:10017000CF93DF93EC017093B90F6093B80F81E0D8
:1001800090E00E942CAB8C010E94FC5F1093B70F93
:100190000093B60F21E02093B30F2093B00F10927D
:1001A000B50F1092B40F1092B20F1092B10F1092BF
:1001B000AF0F84EF91E09093A10F8093A00F88EB95
:1001C0009BE090939F0F80939E0F80E293E090932B
:1001D0009D0F80939C0F8CEA9DE090939B0F8093E2
:1001E0009A0F88E097E09093990F8093980F84E995
:1001F00091E19093970F8093960F1092AE0F10920B
:10020000AD0F1092AC0F1092AB0F1092AA0F10927C
:10021000A90F1092A70F1092A60F1092A50F10927F
:10022000A40F1092A30F1092A20F288329832A8370
:10023000DF91CF911F910F910895AF92BF92CF920E
:10024000DF92EF92FF920F931F93882777FD80959F
:10025000982F1F921F9227E02F9320ED2F932CEDC4
:10026000A22E25E0B22EC12CD12CE12CF12C87013D
:10027000EA9420E030E0A9010E94BDA80F900F9001
:100280000F900F9080E01F910F91FF90EF90DF9003
:10029000CF90BF90AF900C941F5E6CED75E080E046
:1002A0000C941F5E1092B30F2FEA30E84EE150E03D
:1002B00060E070E08091B80F9091B90F0E946D637B
:1002C0009093B50F8093B40F08951092B30FAC01C3
:1002D000662757FD6095762F2FEA30E88091B80F9A
:1002E0009091B90F0E946D639093B50F8093B40FF6
:1002F00008958091B30F882331F060ED77E081E0BD
:100300000E941F5ECFCF08958091B30F882341F0E4
:1003100068EE73E081E00E941F5E88E99AE3D5CF22
:1003200008951DCF1092B00F25EA31E84EE150E05C
:1003300060E070E08091B80F9091B90F0E946D63FA
:100340009093B20F8093B10F089580911E0288237D
:1003500089F087EC99E7A1E0BB27ABBFFC0167916F
:10036000769182E00E941F5E1092AF0FDBDF109249
:100370001E02089587EC99E7A1E0BB27ABBFFC0103
:100380006791769182E00E941F5E81E08093B00FBA
:100390001092AF0F80931E0208956CED75E080E01F
:1003A0000E941F5E6CED75E081E00E941F5E87EC8D
:1003B00099E7A1E0BB27ABBFFC016791769182E092
:1003C0000E941F5EC2CFCF93DF93EC0180E00E94BA
:1003D000BA5C81E00E94BA5C82E00E94BA5CCE0105
:1003E000DF91CF91DACFEF92FF920F931F93CF93CC
:1003F000DF93EC01F62E87EC99E7A1E0BB278E0195
:10040000000F111F0C0F1D1F222717FD2095322FE3
:10041000B901A8014E5F5F4F6F4F7F4F480F591FC3
:100420006A1F7B1F6BBFFA01E79087EC99E7A1E099
:10043000BB274091AF0F63E0469FA00111246627C0
:1004400057FD6095762F4E5F5F4F6F4F7F4F480F80
:10045000591F6A1F7B1F6BBFFA0187918E15D0F45D
:1004600047EC59E761E07727400F511F621F731F68
:100470006BBFFA016791769182E00E941F5EC09384
:10048000AF0FFF2039F0DF91CF911F910F91FF90B7
:10049000EF9048CFDF91CF911F910F91FF90EF9098
:1004A00008958091AB0F882301F161E08CE090E02A
:1004B0009ADF20919E0F30919F0F40E050E06091B5
:1004C000A00F7091A10F80E090E00E94A2A8AB0164
:1004D000BC0121E532E88091B80F9091B90F0E94DC
:1004E0006D639093A70F8093A60F08958091AA0F34
:1004F000882301F161E08DE090E075DF20919A0F93
:1005000030919B0F40E050E060919C0F70919D0FE7
:1005100080E090E00E94A2A8AB01BC0126E732E88F
:100520008091B80F9091B90F0E946D639093A50FC1
:100530008093A40F08958091A90F882301F161E0B1
:100540008EE090E050DF2091960F3091970F40E0C1
:1005500050E06091980F7091990F80E090E00E94B8
:10056000A2A8AB01BC012BE932E88091B80F9091B1
:10057000B90F0E946D639093A30F8093A20F08950B
:1005800061E083E090E02FCF60E084E090E02BCF4B
:10059000DCCEFC0161830895FC018181882321F078
:1005A00061E081E090E01FCF0895FC01818181111D
:1005B000CCCE0895FC0162830895FC0182818823DA
:1005C00021F061E082E090E00ECF0895FC0182818D
:1005D0008111BBCE089561E086E090E004CF61E038
:1005E00085E090E000CF61E087E090E0FCCEFC0188
:1005F00060830895FC018081882321F061E088E018
:1006000090E0F1CE089561E089E090E0ECCE60E00A
:1006100089E090E0E8CE99CE61E08AE090E0E3CE18
:1006200060E08AE090E0DFCE90CE61E08BE090E089
:10063000DACE60E08BE090E0D6CE87CE61E08FE04E
:1006400090E0D1CE61E080E190E0CDCE8091A80F26
:10065000811113C026EA33E848EB5BE060E070E00C
:100660008091B80F9091B90F0E946D639093A70F7E
:100670008093A60F81E08093A80F08958091A80F22
:1006800008957093A10F6093A00F50939F0F409314
:100690009E0F08956093AE0F08958091AB0F811166
:1006A00008C08091AE0F882321F081E08093AB0FCA
:1006B000F8CE08956091A60F7091A70F8091B80FA2
:1006C0009091B90F0E9489631092AB0F08957093B7
:1006D0009D0F60939C0F50939B0F40939A0F08952A
:1006E0006093AD0F08958091AA0F811108C0809189
:1006F000AD0F882321F081E08093AA0FF7CE0895F3
:100700006091A40F7091A50F8091B80F9091B90FCF
:100710000E9489631092AA0F08957093990F6093B5
:10072000980F5093970F4093960F08956093AC0FD6
:1007300008958091A90F811108C08091AC0F882382
:1007400021F081E08093A90FF6CE08958091AE0F3D
:100750008111A3DF8091AD0F8111C5DF8091AC0FB6
:100760008111E7CF08956091A20F7091A30F80913E
:10077000B80F9091B90F0E9489631092A90F089544
:1007800099DFBEDFF0DF1092A80F089581E080931B
:10079000FA0F08951092ED0F1092E30F1092E20FEE
:1007A0001092DE0F1092DF0F1092E00F1092E10F07
:1007B00081E08093EE0F409148105091491060E025
:1007C00070E02CE134E880914310909144100C9437
:1007D0006D636091C70F7091C80F80914310909125
:1007E00044100E94D564882319F081E08093C90FDA
:1007F000089561E089E20C9459A160E088E00C94CE
:1008000059A160E08BE20E9459A16091EF0F7091B5
:10081000F00F80914310909144100E94D56488237A
:1008200051F06091EF0F7091F00F80914310909113
:1008300044100C94896308950E94CC76882391F02B
:100840008DEF9FE00E94436A8091221090912310C7
:10085000DC01ED91FC910190F081E02D1995109251
:10086000EE0F08952CE134E845E050E060E070E0E0
:1008700080914310909144100C946D6381E08093BB
:10088000EE0F6091501084E290E10E94A47BD4CFDF
:10089000CF93DF93EC0102960E948073EDE0F5E0C8
:1008A000A48DB58D16970D90BC91A02DAC0FBD1FDA
:1008B000868D978D8D939C93A0A1B1A116970D90D5
:1008C000BC91A02DAC0FBD1F82A193A152969C9309
:1008D0008E935197A4A1B5A116970D90BC91A02D10
:1008E000AC0FBD1F86A197A154969C938E935397EE
:1008F000A0A5B1A516970D90BC91A02DAC0FBD1F62
:1009000082A593A556969C938E935597A4A5B5A5BD
:1009100016970D90BC91A02DAC0FBD1F86A597A575
:1009200058969C938E935797A0A9B1A916970D90AE
:10093000BC91A02DAC0FBD1F82A993A95A969C9380
:100940008E935997A4A9B5A916970D90BC91A02D87
:10095000AC0FBD1F86A997A95C969C938E935B975D
:10096000A0ADB1AD16970D90BC91A02DAC0FBD1FE1
:1009700082AD93AD5E969C938E935D9704ACF5AD7E
:10098000E02D36970190F081E02DEC0FFD1F809156
:100990004B0590914C0590A3878FE0914D05F09108
:1009A0004E0536970190F081E02DEC0FFD1F8091F0
:1009B0004F059091500592A381A3E0915105F091CC
:1009C000520536970190F081E02DEC0FFD1F8091CC
:1009D00053059091540594A383A3E0915505F0919C
:1009E000560536970190F081E02DEC0FFD1F8091A8
:1009F00057059091580596A385A389E795E09983BB
:100A0000888385E895E09B838A8383E995E09A8BC8
:100A1000898B8DE995E09C8B8B8B87EA95E09E8B8B
:100A20008D8B81EB95E0988F8F8B8BEB95E09A8F78
:100A3000898F85EC95E09C8F8B8F8FEC95E09E8F56
:100A40008D8F89ED95E098A38F8F83EE95E09AA323
:100A500089A38DEE95E09CA38BA387EF95E09EA3E1
:100A60008DA3DF91CF910895CF93DF93CDB7DEB7FC
:100A70002A970FB6F894DEBF0FBECDBF84300CF0BE
:100A800084E028E136E13A83298322E136E13C83A0
:100A90002B832BE036E13E832D8325E036E138873A
:100AA0002F832DEF35E13A872987E82FEE0FFF0BD3
:100AB000EC0FFD1F818192812A960FB6F894DEBF5C
:100AC0000FBECDBFDF91CF910895CF93DF9300D0BC
:100AD00000D0CDB7DEB782300CF082E021EF35E1F7
:100AE0003A83298325EE35E13C832B832DED35E1D7
:100AF0003E832D83E82FEE0FFF0BEC0FFD1F81814E
:100B0000928126960FB6F894DEBF0FBECDBFDF915F
:100B1000CF910895CF93DF9381E08093FA0F1092E5
:100B200042101092D50F1092D00F8093EE0F84E0F8
:100B300090E00E942CABEC0160E00E945A75D093CB
:100B40002310C0932210DF91CF91089581E20E947B
:100B50008EA121E0892B09F420E0822F0895809353
:100B6000F90F08958091F90F089580934510813011
:100B700071F08330C1F488E293E290934710809340
:100B8000461089E080934A1080E197E217C088EB15
:100B90009BE0909347108093461083E080934A1027
:100BA00088E99AE30BC088E893E19093471080931B
:100BB000461086E080934A1080EE9EE290934910A2
:100BC0008093481008958091E90F9091EA0FDC011D
:100BD000ED91FC910684F785E02D199480914C10DD
:100BE0008823A1F181E08093EE0FB0DF882329F004
:100BF00060914F10662349F106C080914D1081111C
:100C000007C060914C1084E290E10E94A47B1DC05B
:100C100090914C109630C9F4823049F0833061F0E5
:100C2000813099F425E530E040E050E009C02AE544
:100C300030E040E050E004C02FE530E040E050E01C
:100C400066E084E290E10E94EA7AF6CD089510927F
:100C5000FA0F409146105091471060E070E026EC8A
:100C600033E880914310909144100C946D6380910F
:100C7000FA0F08956091E60F7091E70F809143108D
:100C8000909144100E94D56481113DC04091E80FBD
:100C900050E060E070E020EC36E8809143109091E5
:100CA00044100E9465639093E70F8093E60F809154
:100CB000E90F9091EA0FDC01ED91FC910488F58930
:100CC000E02D1995809151108823E9F06091E40F8F
:100CD0007091E50F80914310909144100E94D5646B
:100CE000811111C0CBDD2EE334E844E650E060E032
:100CF00070E080914310909144100E94656390933E
:100D0000E50F8093E40F0895729A089572980895FC
:100D10006091E60F7091E70F80914310909144101D
:100D20000E94D5648823A9F06091E60F7091E70FC7
:100D300080914310909144100E9489638091E90F43
:100D40009091EA0FDC01ED91FC910688F789E02D86
:100D500019956091E40F7091E50F80914310909187
:100D600044100E94D564882351F06091E40F709183
:100D7000E50F80914310909144100E948963C6CF83
:100D8000CF93C0912102CC2311F0C0DF01C0BCDFA2
:100D900081E08C2780932102CF91089561E08BE25E
:100DA0000C9459A1EE9A0895F9DFFCDF21E034E8B4
:100DB00048E853E160E070E0809143109091441066
:100DC0000E946D639093F00F8093EF0F0895E6DF1C
:100DD000E9DF21E034E848E853E160E070E0809129
:100DE0004310909144100E946D639093F00F809394
:100DF000EF0F08958091F80F8111D6CFE8CFEE98CC
:100E0000089560E089E20E9459A129EF33E842E3A6
:100E100050E060E070E080914310909144100C9499
:100E20006D6361E088E00E9459A14091F10F5091FB
:100E3000F20F60E070E02DEF33E880914310909165
:100E400044100C946D638091F40F8111DADF80916E
:100E5000F30F8111E6CF0895B6DEF5DF8091F80F2C
:100E6000882321F08091F90F811101C0B7DE8091B4
:100E7000F90F882379F08091F80F882359F0809139
:100E8000F70F882339F0E091EB0FF091EC0F82819E
:100E90000E949C5FDCCE8091F80F8823A1F06699B8
:100EA00016C0ADDFAEDC8091F90F882381F0809110
:100EB000F70F882339F0E091EB0FF091EC0F82816E
:100EC0000E949C5FC9CF669B02C099DF9ACC0895AF
:100ED0001F920F920FB60F9211240BB60F922F9301
:100EE0003F934F935F936F937F938F939F93AF93B2
:100EF000BF93EF93FF93CFDFFF91EF91BF91AF913E
:100F00009F918F917F916F915F914F913F912F9121
:100F10000F900BBE0F900FBE0F901F9018958091F1
:100F2000D20F08958091D10F08958091D50F089523
:100F30008F929F92AF92BF92CF92DF92EF92FF92E9
:100F4000C090DE0FD090DF0FE090E00FF090E10F47
:100F500020E030E0A901C701B6010E94E3AC20E027
:100F600030E040E05FE387FD0BC0C701B6010E949F
:100F700030AB4B015C010E9400AC97FD25C00EC058
:100F8000C701B6010E942FAB0E9400AC97FD1CC0A8
:100F90006536710581059105CCF413C0C501B40116
:100FA0000E9400AC65367105810591057CF420E056
:100FB00030E040E05FE3C701B6010E9430AB0E9421
:100FC00000AC24E6261B03C024E601C020E0822FEB
:100FD000FF90EF90DF90CF90BF90AF909F908F9059
:100FE00008958F929F92AF92BF92CF92EF92FF920D
:100FF0000F931F93CF93DF93EC017B0180915310EC
:10100000823008F08DC08090DE0F9090DF0FA090AE
:10101000E00FB090E10F20E030E0A901C501B4017C
:101020000E9494AB181654F520E030E0A901C501E8
:10103000B4010E94E3AC181654F420E030E048E418
:1010400052E4C501B4010E9494AB1816D4F420E018
:1010500030E048E452E4C501B4010E94E3AC181644
:101060009CF420E030E048EC52E4C501B4010E9459
:1010700094AB87FF09C00BE410E008C000E010E06B
:1010800005C002E310E002C004E610E08FEF8C0D13
:10109000823020F50115110539F0602FCE010E9434
:1010A000F65A602FC70123C0888999899B878A8750
:1010B0008A899B899D878C878C899D899F878E874C
:1010C000F70180899189938782878289938995879F
:1010D0008487848995899787868722C08DEF8C0DB8
:1010E0008230F0F40115110579F0602FCE01DF9107
:1010F000CF911F910F91FF90EF90CF90BF90AF9045
:101100009F908F900C94F65A888999899B878A873B
:101110008A899B899D878C878C899D899F878E87EB
:10112000DF91CF911F910F91FF90EF90CF90BF90E3
:10113000AF909F908F9008951092ED0F1092E30F53
:101140001092E20F1092DE0F1092DF0F1092E00F5C
:101150001092E10F71CB8F929F92AF92BF92CF927C
:10116000DF92EF92FF920F931F93CF93DF93CDB750
:10117000DEB762970FB6F894DEBF0FBECDBF89828F
:101180009A82AB82BC82CD82DE82EF82F8860987AA
:101190001A872B873C874D875E876F87788B898B73
:1011A0009A8BBAA0CBA0DCA06DA17EA1FFA008A560
:1011B00049A55AA5EBA42CA53DA58EA59FA5E8A9F8
:1011C000F9A9F0934410E093431012E1FE01319627
:1011D000A5E4B0E101900D921A95E1F7B092F90FF4
:1011E000C092F80FD092F70F7093F60F6093F50F3F
:1011F000E092E80FF092F40F0093F30F5093F20F88
:101200004093F10F3093EC0F2093EB0F9093EA0F84
:101210008093E90F80915010811102C010925110FB
:1012200090914C10911105C0811103C01092421091
:101230006DC081E080934210809122109091231024
:101240000E9449758091451081118FDC80914C106E
:101250008823E9F18091501060914A1070E0882352
:10126000C9F0809152108823A9F080E090E00E949C
:1012700031AC9B01AC0160E070E088EC92E40E942C
:1012800098AB6093DA0F7093DB0F8093DC0F909331
:10129000DD0F25C080E090E00E9431AC9B01AC01E5
:1012A00060E070E088EC92E40E9498AB6093DA0F03
:1012B0007093DB0F8093DC0F9093DD0F1092D60FAD
:1012C0001092D70F1092D80F1092D90F1FC0109202
:1012D000DA0F1092DB0F1092DC0F1092DD0F60918D
:1012E0004B1070E080E090E00E9431AC9B01AC01BB
:1012F00060E070E088EC92E40E9498AB6093D60FB7
:101300007093D70F8093D80F9093D90F15DF6E98F5
:10131000769AEE9880916A008F7C80936A00809123
:10132000F80F882321F080916A00806203C08091C9
:101330006A00806380936A0062DD62960FB6F8945B
:10134000DEBF0FBECDBFDF91CF911F910F91FF90F8
:10135000EF90DF90CF90BF90AF909F908F9051CA49
:1013600061E087E00E9459A181E08093D00F089549
:1013700060E087E00E9459A11092D00F0895CF93AA
:10138000DF9300D0CDB7DEB784E689838CE38A8310
:1013900088E28B838091C30F8330F8F480FF02C012
:1013A000E7DF01C0DDDF8091C30FE1E0F0E0EC0F8B
:1013B000FD1FE80FF11D408150E060E070E02FEB71
:1013C00039E880914310909144100E946D638091A0
:1013D000C30F8F5F8093C30F03C0CADF1092C30F88
:1013E0000F900F900F90DF91CF9108958091BF0FD4
:1013F000811110C084EF91E09093BE0F8093BD0FD8
:101400008BE290E09093BC0F8093BB0F81E08093C0
:10141000BF0F20C08091BB0F9091BC0F853291050A
:1014200014F0049709C08331910514F0029704C0A9
:10143000823091052CF001979093BC0F8093BB0FE5
:101440008091BB0F9091BC0F97FF04C01092BC0F0E
:101450001092BB0F8091BA0F882311F089DF01C071
:101460007FDF8091BA0F91E089278093BA0F409176
:10147000BD0F5091BE0F1416150654F01092BF0FF9
:1014800077DF27E63AE84AEF50E060E070E006C018
:10149000662757FD6095762F26EF39E88091431037
:1014A000909144100E946D639093C60F8093C50F76
:1014B0008091BD0F9091BE0F2091BB0F3091BC0F5A
:1014C000821B930B9093BE0F8093BD0F0895809164
:1014D000D50F81118BCF6091C50F7091C60F809190
:1014E0004310909144100E94D564882351F060917C
:1014F000C50F7091C60F80914310909144100E94C7
:10150000896336CF8091D50F811155C01FDB8823A9
:10151000E9F081E08093D50F8091E90F9091EA0F77
:10152000DC01ED91FC910284F385E02D1995CFDF6C
:101530002CED3AE848E95AE360E070E0809143100E
:10154000909144100E946D6382DB09C08091F90F75
:10155000882329F18091F80F882311F025DC3ECBF8
:1015600036DC8091F70F882339F0E091EB0FF09192
:10157000EC0F82810E949C5F4091F50F5091F60F15
:1015800014161506BCF4662757FD6095762F2CE2DD
:1015900037E880914310909144100C946D638091D2
:1015A000F70F882339F0E091EB0FF091EC0F828177
:1015B0000E949C5F51CC0895CF92DF92EF92FF92F0
:1015C0001092D50F2091DA0F3091DB0F4091DC0F94
:1015D0005091DD0F6091DE0F7091DF0F8091E00F71
:1015E0009091E10F0E942FAB6B017C0120E030E075
:1015F000A9010E9494AB87FD09C0C092DE0FD09272
:10160000DF0FE092E00FF092E10F08C01092DE0FC2
:101610001092DF0F1092E00F1092E10FFF90EF9009
:10162000DF90CF9054CF6091D30F7091D40F809101
:101630004310909144100E94D564882351F060912A
:10164000D30F7091D40F80914310909144100E9459
:1016500089638091D50F882319F01092D50F37CF69
:1016600008958091D00F811183CE7ACECF93C82F69
:10167000682F70E087E00E9408A0CC2321F081E071
:101680008093D00F02C01092D00FCF910895909107
:10169000C20F8091ED0F91112EC0882309F44EC026
:1016A0006091C00F7091C10F8091431090914410D0
:1016B0000E94D564882351F06091C00F7091C10FD2
:1016C00080914310909144100E94896349DE27E481
:1016D0003BE842EC51E060E070E080914310909173
:1016E00044100E9465639093C10F8093C00F81E006
:1016F0008093C20F08958111B4CF8091D00F8823B9
:10170000D9F36091C00F7091C10F809143109091F7
:1017100044100E94896327E43BE844E150E060E024
:1017200070E080914310909144100E946563909303
:10173000C10F8093C00F1092C20F089580911F02B5
:101740009091200202979093200280931F02181616
:1017500019060CF48BCF6091C00F7091C10F80916E
:101760004310909144100E94896302DE8FEF90E055
:101770009093200280931F0208958091CA0F909148
:10178000CB0F2091CE0F3091CF0F820F931F9093EC
:10179000CB0F8093CA0F6ADF8091CE0F9091CF0F4D
:1017A00018161906D4F52091CA0F3091CB0F8091ED
:1017B000CC0F9091CD0F281739070CF47FC0809182
:1017C000C90F882371F01092CD0F1092CC0F8CEFBF
:1017D0009FEF9093CF0F8093CE0F81E08093C40F43
:1017E000089522E830E040E050E06AE070E080E0F8
:1017F00090E00E94A2A87093CD0F6093CC0F22E3DB
:1018000030E040E050E06AE070E080E090E00E946C
:10181000A2A87195619571094DC0892B09F44EC03C
:101820002091CA0F3091CB0F8091CC0F9091CD0FAA
:10183000821793070CF442C08091C40F882311F1E2
:101840006091C70F7091C80F809143109091441020
:101850000E94D564882391F16091C70F7091C80FE1
:1018600080914310909144100E94896381DD109211
:10187000CB0F1092CA0F1092C40F8091ED0F8823E6
:10188000E9F005CF2FEF30E040E050E066E970E08E
:1018900080E090E00E94A2A87093CD0F6093CC0FDF
:1018A00022E330E040E050E06AE070E080E090E069
:1018B0000E94A2A87093CF0F6093CE0F08956091FD
:1018C000C50F7091C60F80914310909144100E94F3
:1018D000D5648823D1F06091C50F7091C60F8091B7
:1018E0004310909144100E94896329EE33E848EB3D
:1018F0005BE060E070E080914310909144100E94A2
:101900006D639093C60F8093C50F6091C70F709160
:10191000C80F80914310909144100E94D5648111AA
:1019200048C01092C90F8FEF90E09093CB0F809337
:10193000CA0F16DD22E830E040E050E06AE070E0D7
:1019400080E090E00E94A2A87093CD0F6093CC0F2E
:1019500022E330E040E050E06AE070E080E090E0B8
:101960000E94A2A87195619571097093CF0F609341
:10197000CE0F2DEB3BE844E150E060E070E0809159
:101980004310909144100E9465639093C80F809318
:10199000C70F29EE33E848EB5BE060E070E0809130
:1019A0004310909144100E946D639093C60F8093F2
:1019B000C50F0895CF938091EE0F8111E3C18091FF
:1019C000ED0F8111DFC180914210882309F4DAC143
:1019D0006DEF7FE080912210909123100E9471752D
:1019E000882309F4CFC11092D20F1092D10F6091C9
:1019F0004C10611105C060914E1061110BC00BC1FC
:101A00008BEF9FE00E949473C82F80914C10CC23E1
:101A1000B1F00EC080914C10681709F4FCC08BEF38
:101A20009FE00E949473C82F80914E10CC2389F0C0
:101A30008093D20FC1E08230B9F1C0E035C082306E
:101A400099F461E08BEF9FE00E949473882361F02A
:101A500009C08230D1F461E08BEF9FE00E94947363
:101A6000882399F081E00EC080914C10813019F6E6
:101A700062E08BEF9FE00E949473C82F882309F4E3
:101A8000BACF82E08093D20F0FC080914E10813088
:101A900009F0C1C062E08BEF9FE00E949473C82FF1
:101AA000882309F4B8C0EDCF8091D20F8630C9F5F4
:101AB000409100105091011060910210709103103C
:101AC0004535510561057105A1F040F440355105DA
:101AD0006105710531F51092D10F23C04A355105CA
:101AE0006105710571F04F3551056105710589F08A
:101AF00018C081E08093D10F80914D10813089F41E
:101B00008AC082E08093D10F80914D10823049F4D9
:101B100082C083E08093D10F80914D10833009F40F
:101B20007AC081E08093EE0F8091D50F81117BDD2B
:101B30008091E30F8F5F8093E30FCC2329F020E0A7
:101B400030E048E452E408C02091DA0F3091DB0F16
:101B50004091DC0F5091DD0F6091DE0F7091DF0F2F
:101B60008091E00F9091E10F0E9430AB6093DE0F07
:101B70007093DF0F8093E00F9093E10F20E030E04F
:101B800048EC52E46091DE0F7091DF0F8091E00F1E
:101B90009091E10F0E94E3ACA091E90FB091EA0FA0
:101BA000ED91FC91119787FD22C00288F389E02D09
:101BB000CD01199580E090E0A8ECB2E48093DE0FAF
:101BC0009093DF0FA093E00FB093E10F81E080933B
:101BD000ED0F2AEC33E848E95AE360E070E08091C9
:101BE0004310909144100E946D6369DE12C000881A
:101BF000F189E02DCD01199562DE2CE134E84CE449
:101C000054E060E070E080914310909144100E9495
